:020000040000FA
:040000006FD00400B9
:101000006F00907D00000000000000009020002094
:10101000AA220020A9BDF9F56C23002000000000E1
:10102000000000006C230020902000200000000041
:101030000000000090200020000000009020002010
:101040000000000090200020902000209020002030
:101050009020002090200020482F00208224002093
:101060000000000090200020902000200C24002090
:1010700090200020D22300209020002090200020EB
:101080009020002090200020902000209020002020
:101090009020002001A04111B7170040985F3AC688
:1010A000945F3247E39CE6FE3245410182800111A4
:1010B00013078008F337078093F787083EC20100C3
:1010C0000100B7170040930570052380B70413068D
:1010D00080FA2380C7040100010083C6B70493F699
:1010E000F60DA385D704238007049246F3A6068055
:1010F0000100010093760502D5CEF336078093F602
:10110000860836C4010001002380B7042380C70489
:1011100001000100B70614007D89558D88C70100C4
:1011200001000100010023800704A246F3A6068007
:101130000100010073370780137787083AC6010062
:1011400001002380B7042380C704010001000100CF
:1011500001003727004093061005A303D7802380A2
:101160000704B247F3A70780010001009307800836
:10117000F3B7078093F787083ECE01000100B71749
:101180000040130770052380E704130780FA2380CB
:10119000E7040100010003C7B70413670708A3852C
:1011A000E70423800704F247F3A70780010001004A
:1011B0000561828093760504BDC6F336078093F6F9
:1011C000860836C8010001002380B7042380C704C5
:1011D00001000100B7061400938606047D89558D31
:1011E00088C7010001000100010023800704C246F6
:1011F000F3A6068001000100733707801377870884
:101200003ACA010001002380B7042380C70401000B
:1012100001003727004093062005A303D7802380D1
:101220000704D24781B773370780137787083ACC12
:10123000010001002380B7042380C70401000100DE
:1012400098471367070C98C723800704E24719BF24
:101250000111814601468145114506CE97000000E7
:10126000E780405793078008F3B7078093F7870814
:101270003EC601000100B717004013077005238028
:10128000E704130780FA2380E7040100010003C785
:101290006704136717002383E70423800704B2471A
:1012A000F3A7078001000100F2400561828041112F
:1012B000814601468145114597000000E780805135
:1012C00013078008F337078093F787083EC40100AF
:1012D0000100B7170040130670052380C70493066A
:1012E00080FA2380D70401000100FD552396B70240
:1012F00023800704A245F3A5058001000100733790
:101300000780137787083AC6010001002380C704CD
:101310002380D7040100010003C767041367170087
:101320002383E70423800704B247F3A70780010063
:10133000010001A0B1473305F50201007D1575FDDF
:101340008280411122C426C206C6AA8401446317C2
:101350009400B24022449244410182800504130566
:10136000803E420497000000E78000FD4180C5B741
:101370009305000273A04580824573901534924016
:101380002242B2424243D2436244F2440255925551
:101390002256B2564257D2576258F25806499649D9
:1013A000264AB64A464BD64B664CF64C065D965DD1
:1013B000265EB65E465FD65F09617300203041113C
:1013C000B7170040985F3AC6945F3247E39CE6FE49
:1013D000324541018280B71700401307000323887C
:1013E000E7028547171700002326F74673002030D1
:1013F000411122C406C637040020976000E0E78050
:10140000204A1C408297976000E0E7806049F5B76A
:1014100037370040834747009146BD8B639ED70214
:10142000B73600401306F00F973500009385851FEF
:101430009737000083D7072F03C7A6001377F70F4E
:101440001DE3B7E70400BC4F0946894517150000A6
:101450000345C5F7829731A099466394D700834727
:1014600057007300203003C786001377F70FE3653A
:10147000F6FC13851700AE97173800002314A82A2E
:101480002380E70075B7B787004003C76700098B63
:101490006309071003C77700930600031377070358
:1014A000630DD708173800000348987717360000F7
:1014B000130606740547B30606012380E60083C5BC
:1014C0007700173700001307A774429793F5F50FBD
:1014D0002300B70003C58700973500009385457248
:1014E000C2951375F50F2380A500034707008945B2
:1014F0001377F703630CB70C63E7E50A6306071A73
:101500008545630CB7129737000083C7777133079F
:10151000F600034707001377F70F19CB850793F7FA
:10152000F70F3D476363F71A17370000A30AF76EFA
:10153000B787004009472383E700B787004083C788
:101540007700E207E18763DE07049737000083C76F
:10155000376D173700001307A7693E9785462300AC
:10156000D700173700001307A76A3E9793060003BA
:101570002300D70017370000130787683E97A1465E
:1015800085072300D70093F7F70F3D476364F714EF
:1015900017370000A306F768B78700400947238381
:1015A000E70073002030930610026300D70E930605
:1015B00020026305D70693060002E316D7F403C79B
:1015C00027021377C70F13672700D5A803C7670043
:1015D0001377070465CB03C7A70217380000130869
:1015E000A842173500001305E5391347070823857E
:1015F000E70203C7A7021377370F13678700238516
:10160000E702814713070004B305F5008C41B306D8
:10161000F80091078CC2E399E7FEF5B503C7A7026E
:10162000134707042385E70203C7A7021377C70FF1
:10163000136727002385E702F9B503C7670013770F
:10164000070449C303C76702173800001308882F2F
:10165000173500001305C526134707082383E70243
:1016600003C767021377370F136787002383E702E7
:10167000814713070004B305F5008C41B306F80059
:1016800091078CC2E399E7FEBDBD03C7670213470C
:1016900007042383E70203C767021377C70F1367A3
:1016A00027002383E70285B503C767001377070484
:1016B00011CB03C727021377370F136787002381E6
:1016C000E70291B5238006003DBD97370000A3894E
:1016D0000754B9BD97370000A384075475BD230391
:1016E000048015472303E48001002302A480828044
:1016F00083076480E3CE07FE230304808280830790
:101700006480E3CE07FE03454480828083076480C3
:10171000E3CE07FE2302A4808280411126C44AC280
:101720004EC006C61377F50BAD47AA892E8995449E
:10173000630CF700194597000000E78080FA9700D6
:101740000000E78020FB8D444E8597000000E78075
:1017500040F9FD59FD1463983401B240A244124986
:10176000824941018280135509011375F50F9700D5
:101770000000E780E0F92209F1BF011126CC06CE76
:10178000B704080097000000E780C0F615459700F1
:101790000000E78000F597000000E78080F69700E2
:1017A0000000E78000F62AC697000000E78080F47A
:1017B00032459377150089EB136515001375F50F06
:1017C000F240E24405618280FD14E9F00145CDBF9D
:1017D000397126DC4ADA4ED852D656D45AD25ED067
:1017E00006DE62CE66CCB7E700E07D5783AA07002D
:1017F00022C603AA470023A0E71823A2E718B717B9
:101800000040130770052380E704130780FA238044
:10181000E70483C74704930B75FFB684E20793FB85
:10182000FB0F8546AA892E8B328937240040E18739
:10183000015763FA76016308D50089461307000251
:101840006313D5000157D98F93F7F70FB71C0040EA
:101850002382FC0411472303E4801305F00F970053
:101860000000E78000E8094C97000000E78080E86E
:1018700063657C15B7050700DA953787070079554A
:1018800063FEE504B3879500636AF704370B08002D
:10189000A94733EB65016395F90881E88144970016
:1018A0000000E78020E5268515A8DA850945970020
:1018B0000000E780C0E605090345F9FFFD14050BAC
:1018C00097000000E780C0E481C49377FB0FE5F741
:1018D00097000000E780A0EA69F17D55B717004046
:1018E000130770052380E704130780FA2380E704B9
:1018F00003C74704418B2382E704F250B7E700E0B7
:1019000023A0571123A24711E25432445259C2591D
:10191000325AA25A125B825B724CE24C2161828085
:10192000A547639BF90685691309F00FB306990073
:10193000B3742B01B6941349F9FFB3749900856B06
:1019400033796901416B9387F9FFB3F7270199E375
:1019500063FC340193D94900C147E3E637FF3DBF3B
:101960000569C1697D19D9B71305800D63886901BF
:10197000130500026384790113051008CA859700D6
:101980000000E780C0D997000000E78040DF31D534
:101990004E99B38434416DBFDA852D459700000020
:1019A000E780E0D7CA94E30B99EE050997000000A1
:1019B000E78020D5A30FA9FEFDB79387F9FF93F722
:1019C000F70F636DFC0C83C71C0413073008631505
:1019D000F706370708006361EB06B3079B00B706FD
:1019E000100063FBD704334BEB0089476399F9067A
:1019F0008980D549E38404EADA8509459700000027
:101A0000E780E0D111090327C9FF91472320E48033
:101A100003076480E34E07FE23033481FD17EDFBCB
:101A2000FD14110B81C49377FB0FE9FF97000000B1
:101A3000E780E0D461F155B5B717004003C75704FC
:101A4000B70708001377070219E3B787070079552E
:101A5000E376FBE833079B00E3F9E7F841B58547F8
:101A6000E380F9F0DA852D4597000000E78020CB70
:101A70009389F4FFE38404E297000000E78060C8E4
:101A800093F7390091EB832604800327090093071D
:101A90004900E396E6E03E89CE84D9BFB547639915
:101AA000F9001305900B97000000E78080C3FDB399
:101AB000B1471305B00AE388F9FE99476397F90423
:101AC000B7050800B365BB002D4597000000E7800F
:101AD00000C581448D4BA14997000000E78060C29A
:101AE00063967401832704802320F9008504E3951D
:101AF00034FF8327048013172B016355070023123B
:101B0000F90069BB2322F90051BB9D47639FF9028D
:101B100081451305B00497000000E78040C0BD4434
:101B20002320090023220900FD5997000000E780C7
:101B300040BD93F77400CA9703C70700FD14398DA1
:101B40002380A700E39334FF91BBA1476397F90675
:101B500097000000E780A0C28144630D0B008D4711
:101B60009304C0036308FB009304000563048B0126
:101B7000930440041375C507E30295D219459700F5
:101B80000000E78000B697000000E780A0B605459A
:101B900097000000E780E0B4268597000000E7800A
:101BA00020B7094597000000E78080B69700000045
:101BB000E780E0BCE31405CE0DB39147639FF900C5
:101BC0001305600697000000E780A0B197000000B1
:101BD000E78040B213059009F9B5E38109CCF154CF
:101BE0007DB9BD660147173600001306E6209386CF
:101BF00006A685458347060093F7F70F91C38280B9
:101C00000507E3F9E6FE973700002387B71EDDB727
:101C10007D166206618693178601E18763D407000B
:101C200001458280931726003307F500AE971843CD
:101C30009C4363E7E7007D16E37FF7FC7D558280D8
:101C400005458280FD15E205E185139785016187D1
:101C500093F7F50F63480700FD15139725002A97A2
:101C6000584365D713851700620561858280330864
:101C7000B5021C4283A80600B335B502C29733B53E
:101C80000701AE98469585486367B5006394A50043
:101C900063E3070181480C43C6950CC388C21CC28C
:101CA000828081471397870161876343B7008280F1
:101CB000139727002A97232007008507E5B7814758
:101CC000014793968701E18663C5B6001335170077
:101CD000828093962700AA9694428507558FD5B7A0
:101CE00093D755408A07AA979C4305453315B500FD
:101CF0007D8D828017F3FFDFE702A33D2A849700E2
:101D00000000E78060F405C5931725003E94032783
:101D1000C4FF814711EB7D1516053E9542054185AF
:101D200017F3FFDF6700233D05838507E5B701450E
:101D3000C5BF81471397870161876343C7008280CE
:101D400013972700B386E50094422A97850714C3AA
:101D5000D5B77D1662066186014793178601E18734
:101D600063D5070013351700828093172600B3064A
:101D7000F500AE9794429C437D16B58F5D8FF1BF01
:101D80008A05AA9501476363B500828083A6C5FFD3
:101D9000F11593D71600D98F9CC11397F601E5B7BB
:101DA0002A830148014701456343D7008280B387F6
:101DB000050183A80700B30706019C43C697AA97AD
:101DC0006384F80033B517010507B3080301620700
:101DD00023A0F80061871108C1BF2A83014781470A
:101DE000014563C3D70082803388E500832808005B
:101DF000330EE600032E0E003388A8403308C84196
:101E00006384080133B508018507B308E300E207DE
:101E100023A00801E1871107E9B717F3FFDFE70205
:101E2000432B0111B286B2842E86AA850A859700BB
:101E30000000E780C0FA2A84A6850A859700000082
:101E4000E78020E833348000060413351500018D47
:101E5000056117F3FFDF6700032A17F3FFDFE702CF
:101E6000C3244111AA89AE8A328BB68402C202C44D
:101E700002C60144131C8401135C8C4163499C021B
:101E8000939B1400FD1B0549138CF4FFF15C330494
:101E90008901620461846340740792478E04CE9482
:101EA00023AEF4FE410117F3FFDF6700832313190C
:101EB0002400B30B2B01014A93172A00D69783A560
:101EC0000B00884378003400500097000000E78042
:101ED00040DA050A93178A01E187F11BE35EFCFCF7
:101EE00092474E9905042320F900A2473EC2B2470B
:101EF00002C63EC441B7131A8901135A8A41131D01
:101F0000240093178A01E18763CF970092470A0460
:101F10004E941CC0A24705091379F90F3EC2B2477F
:101F200002C63EC4ADB7B3079A0313152A005695EF
:101F30000841780034005000050AEA97DA978C438C
:101F400097000000E780E0D26DBF0000197106C263
:101F500012C416C61AC81ECA22CC26CE2AD02ED229
:101F600032D436D63AD83EDA42DC46DECAC0CEC2D9
:101F7000D2C4D6C6DAC8DECAE2CCE6CEEAD0EED209
:101F8000F2D4F6D6FAD8FEDA971500009385058CC0
:101F90008841E700050092402242B2424243D243C8
:101FA0006244F244025592552256B2564257D257D5
:101FB0006258F25806499649264AB64A464BD64BCD
:101FC000664CF64C065D965D265EB65E465FD65F55
:101FD0000961730020300000972100209381810265
:101FE000175100201301018217F5FFFF1305C501EA
:101FF0009705002093850501171600201306C6FDDE
:1020000063FAC5008322050023A055001105910540
:10201000E3EAC5FE17050200130545559715002094
:102020009385C5FB171600201306C66563FAC50025
:102030008322050023A0550011059105E3EAC5FEA2
:102040001715002013050564974500209385852604
:102050006377B500232005001105E36DB5FEFD4251
:10206000739002BC8D4273904280B722000093822D
:10207000828873900230970200209382A2F893E244
:1020800032007390523097520000938262A0739096
:1020900012346FB0F47673002030397101436EC68C
:1020A00019A0397141536AC866CA62CC5ECE19A0C4
:1020B000397101535AD056D252D44ED64AD826DA64
:1020C00022DC06DE33016140828241114AC026C211
:1020D00022C406C68282B24D4101024D924C224C6E
:1020E000B24B4101024B924A224AB2494101024994
:1020F00092442244B240410182803D432A87637367
:10210000C3029377F700BDEFADE5937606FF3D8AF6
:10211000BA960CC34CC30CC74CC74107E36BD7FE40
:1021200011E28280B306C3408A06970200009696A9
:102130006780A6002307B700A306B7002306B700F1
:10214000A305B7002305B700A304B7002304B70015
:10215000A303B7002303B700A302B7002302B7000D
:10216000A301B7002301B700A300B7002300B70005
:10217000828093F5F50F93968500D58D9396050192
:10218000D58D61B7939627009702000096968682B8
:10219000E78086FA9680C1171D8F3E96E374C3F8D8
:1021A000A5B73367B500FD530D8B79E7B7877F7F00
:1021B0009387F7F710419441B372F6003363F6004A
:1021C000BE92B3E262006397720C6318D606504168
:1021D000D441B372F6003363F600BE92B3E26200FC
:1021E0006398720A631BD60410459445B372F600D7
:1021F0003363F600BE92B3E262006391720A631E1B
:10220000D6025045D445B372F6003363F600BE9251
:10221000B3E26200639A72086311D60210499449CE
:10222000B372F6003363F600BE92B3E262006393CA
:1022300072085105D105E30FD6F6131706019397DF
:102240000601631CF7001357060193D706013305F7
:10225000F7409375F50F91E982804183C18333057F
:10226000F7409375F50F91E182801377F70F93F79D
:10227000F70F3305F74082800346050083C605004B
:10228000050585056313D60065FA3305D6408280BF
:1022900011059105E312D6FE014582802105A105B5
:1022A000E31CD6FC014582803105B105E316D6FC5E
:1022B000014582804105C105E310D6FC01458280BD
:1022C000B717004003C777051377E70FA38BE70421
:1022D000130700F8A38DE7043D47238CE704130799
:1022E0005003A38CE70403C7A7051377D70F238DEB
:1022F000E7048280B717004003C7E7020D89411148
:102300001377C70F498F93068008F3B6068093F6BC
:10231000860836C601000100930670052380D704A5
:10232000930680FA2380D704010001002387E70287
:1023300023800704B247F3A7078001000100410191
:10234000828041112A83014E930E407E130F0019A3
:10235000930F400663E56E129308001913034006BD
:10236000B3781503854E0D4FA14F337365020D8968
:102370001335150063EFBE121308F6FF7946729805
:102380004208135808013307C70213D61700BE07C7
:1023900032976146B3F6C60213068070B386C60252
:1023A0003697A166F58F42075D8FB716004083C749
:1023B000F60293F70708A303F1000346710083C7F1
:1023C000F60293F70708E394C7FE83477100B71638
:1023D000004093F7F70F6388071293078008F3B75D
:1023E000078093F787083EC401000100B71700403B
:1023F000930670052380D704930680FA2380D704C0
:102400000100010023AA070383C6170393E6060809
:10241000A388D70223800704A247F3A707800100FF
:1024200001001166B71700407D16D45BC85F938525
:102430004703A98EF18EF5FA93068008F3B606805D
:1024400093F6860836C601000100930670052380C6
:10245000D704930680FA2380D7040100010098C1B5
:1024600003C7170313670704A388E7022380070441
:10247000B247F3A7078001000100410182807D136C
:102480003368E3039308E016630E08003368F30330
:102490009308D016630808009378330093B81800A7
:1024A0009388D81633081E01131E0801135E0E010F
:1024B00055B56393E5030548638608000148630347
:1024C00003002A8871087298FD15131E0801C205C1
:1024D000135E0E01C18179BD13F8150063F4BF00CE
:1024E0007908D5B713381800E5BF83C7F60293F70C
:1024F0000708A303F1000346710083C7F60293F7B0
:102500000708E394C7FE8347710093F7F70FF1DFE5
:10251000E9B531714AD966CB06DF22DD26DB4ED71D
:1025200052D556D35AD15ECF62CD6AC96EC7AA8C36
:1025300002D897100000E78020B12A89930780080D
:10254000F3B7078093F787083EDA01000100B71759
:102550000040130770052380E704130780FA2380E7
:10256000E7040100010003C7F7021377770FA38781
:10257000E70203C7F70213678700A387E7022380F8
:102580000704D257F3A70780010001000545970013
:102590000000E78060D6130780C13347E902116A63
:1025A00093070AE893065002BD69930BA004814A81
:1025B000014B13048008930470057D1AB347F90298
:1025C0003307D7023EC0FD873ECC938709A6930907
:1025D000803E3347F7023AC27D873AC43347390316
:1025E0008549B399990193D93940B306D702B30B02
:1025F0007703B3C6F602B3CBFB0236C6FD8636C8F8
:1026000093D6FB4136CEB7460F0093860624334956
:10261000D9028566938606FAB3969601B389E902D4
:10262000130760553309D90293060010B389E902F4
:102630003349D902B3C9F9029316390036CA37199A
:102640000040FD8636D0930D090493D7F9413ED260
:10265000F336048093F6860836DC01000100930708
:1026600070052380FD00930680FA2380DD000100C1
:1026700001008346390593F6860FA309D9048346E2
:10268000390593E61600A309D90423800D00E2560C
:10269000F3A6068001000100130C80FA116DF336D9
:1026A000048093F6860836DE01000100930770056A
:1026B0002380FD0023808D01010001008346390540
:1026C000216693E60602A309D90483560905B3E6F9
:1026D000A6012318D90483560905D18E2318D904DD
:1026E00023800D00F256F3A6068001000100834608
:1026F000390593F606026381061A03463905218AD5
:102700006DDE081897100000E7800098733604808B
:1027100013768608B2C20100010023809D00238049
:102720008D0101000100B717004003C6370513767D
:10273000F60DA389C70403C6370513660602A389ED
:10274000C704835609052166B3E6A6012318D904F8
:1027500083560905D18E2318D90423800D0096468F
:10276000F3A60680010001008346390593F60602B0
:10277000638B061483463905A18AEDFE970000207D
:10278000E7806091AA8636D497000020E780A09069
:10279000A256E30AD5FE835609054255B3E6A601C3
:1027A0002318D90497100000E780C08F83463905AD
:1027B000A18AEDDE03560905834629058247337653
:1027C000CA00B306DA0293D5F641B296B388F64052
:1027D000E24733B8C6002E983308F840A247B3B694
:1027E00016013308D84063C70701631DF8009247FC
:1027F00063FA1701C247634FF80E63950701B247AA
:1028000063EAF80E894663E9660FF24693151800ED
:1028100013D3F8015E8613951800B365B30042D652
:1028200046D497C00100E780C0E93258050B137BFE
:10283000FB0F63470001631A0838A2586387083802
:1028400013081500B336A800B69513D6F5013298D3
:10285000B336C800AE9613581800FE06B3E606015C
:102860007336048013768608B2C601000100238007
:102870009D0023808D01010001000356C902B2961C
:10288000C206C1822316D90223800D00B646F3A6E4
:1028900006800100010021B5F336048093F6860816
:1028A000B6C00100010023809D0023808D0101003E
:1028B00001008346390593E60602A309D904238063
:1028C0000D0086460DB5F336048093F68608B6C42F
:1028D0000100010023809D0023808D010100010083
:1028E0008346390593E60602A309D90423800D0027
:1028F000A646BDB5E30B0BF0F336048093F68608CD
:10290000B6C801000100930680FA23809D00238051
:10291000DD00010001008346390593F5FC0F93F6B5
:10292000860FA309D90483463905CD8EA309D9049E
:1029300023800D00C646F3A60680010001001305A2
:1029400080FA03463905930639051D8A631C9629CA
:102950007336048013768608B2CC0100010013069A
:1029600080FA23809D002380CD000100010003C672
:1029700006001376F60D2380C60003C60600136614
:1029800006022380C600835609051166D18E2318DE
:10299000D904835609052166D18E2318D9042380D2
:1029A0000D00E646F3A6068001000100130680FA3A
:1029B0008346390593F60602638006268346390569
:1029C000130C3905A18AFDDA081897000000E7808A
:1029D000A06BF336048093F68608B6D001000100A0
:1029E000930680FA23809D002380DD000100010012
:1029F00083460C00116693F6F60D2300DC00834637
:102A00000C0093E606022300DC0083560905D18EF4
:102A10002318D904835609052166D18E2318D904B9
:102A200023800D008656F3A60680010001001306E0
:102A300080FA8346390593F60602638A06208346A8
:102A40003905A18AEDFE97F0FF1FE780C0642A8C4C
:102A500097F0FF1FE7802064E30C85FF835609058C
:102A600011664255D18E2318D90497000000E780E3
:102A700060638346390513063905A18AFDDAF3360A
:102A8000048093F68608B6D401000100930680FA0C
:102A900023809D002380DD000100010083460600A5
:102AA00093F6F60D2300D60023800D00A656F3A65C
:102AB0000680010001008356090503462905D24717
:102AC000B376DA003306CA021305800C9355F6413B
:102AD0003696330DF6408257333CD6002E9C333663
:102AE000A601330CFC40330CCC40330885039256CE
:102AF0004E86B335A5033305A503C29597C00100E3
:102B0000E78020BC63468001631E0C16630C0D1623
:102B1000130615003335A6002E959356F50136960B
:102B2000B335D600AA959396F50105828585D18E99
:102B30006346B000639D051A638B061A0356C902EB
:102B400015823305D6003336C500B2956348B00010
:102B5000639105241306F00F637DA622894663F373
:102B6000561593078008F3B7078093F78708BED6FA
:102B70000100010037170040930770052300F70498
:102B8000930780FA2300F704010001008356C7026F
:102B900089678117D58FC207C1832316F7022300E7
:102BA0000704B657F3A7078001000100FA506A54E2
:102BB000DA544A59BA592A5A9A5A0A5BFA4B6A4C59
:102BC000DA4C4A4DBA4D296182801308F5FF33353E
:102BD000A800FD152E951356F5013298B336C8009E
:102BE000AA9695B9F336048093F68608B6CA010012
:102BF000010023809D002380AD0001000100834679
:102C00003905CD8EA309D90423800D00D646F3A63D
:102C100006800100010035B3F336048093F6860880
:102C2000B6CE0100010023809D002380CD0001006D
:102C300001008346390593E60602A309D9042380DF
:102C40000D00F646F3A606800100010095B3F336A9
:102C5000048093F68608B6D20100010023809D000F
:102C60002380CD00010001008346390593E606026A
:102C7000A309D90423800D009656F3A6068001000F
:102C8000010045BB9306F5FF33B5A600FD152E9553
:102C90009355F501AE96B3B5B600AA951396F50116
:102CA000858269B5F336048093F68608B6D80100AC
:102CB0000100930680FA23809D002380DD0001003F
:102CC00001008356C9020566011693F6F60FD18EF0
:102CD000C206C1822316D90223800D00C656F3A670
:102CE000068001000100850A93FAFA0F95B233E6D7
:102CF000B60045C20356C9023305D0403338A000A0
:102D0000B305B040B385054115826345B000D1E1FC
:102D10006371A608894663F0560593078008F3B7E8
:102D2000078093F78708BEDA01000100B71700405B
:102D3000130770052380E704130780FA2380E70454
:102D40000100010003D7C7027D8B2396E702238091
:102D50000704D65781BDF336048093F68608B6DCA7
:102D600001000100930680FA23809D002380DD008E
:102D7000010001008356C9020566011693F6F60F9D
:102D8000D18EC206C1822316D90223800D00E656D9
:102D9000B9B793078008F3B7078093F78708BEDEBB
:102DA0000100010037170040930770052300F70466
:102DB000930780FA2300F704010001000356C702BD
:102DC00093975600B297C207C1832316F7022300D8
:102DD0000704F657C1BB914763EEB70217D701004E
:102DE0001307C7798A05BA959C41BA978287B717A6
:102DF000004003A7470B1345F5FF698F23AAE70A95
:102E000003A7070B698F23A8E70A03A7070A798D91
:102E100023A0A70A8280B717004083A6470B134759
:102E2000F5FFF98E23AAD70A83A6070B558D23A891
:102E3000A70A83A6070A758F23A0E70A8280B7171F
:102E4000004003A7470B498F23AAE70A03A7070BF4
:102E50001345F5FF45BFB717004083A6470B13473F
:102E6000F5FF758F23AAE70A03A7070A598D4DB707
:102E7000B717004003A7470B498FEDB7914763EEA3
:102E8000B70217D701001307A7708A05BA959C41AE
:102E9000BA978287B717004003A7470D1345F5FF80
:102EA000698F23AAE70C03A7070D698F23A8E70CF6
:102EB00003A7070C798D23A0A70C8280B7170040C9
:102EC00083A6470D1347F5FFF98E23AAD70C83A6D7
:102ED000070D558D23A8A70C83A6070C758F23A07B
:102EE000E70C8280B717004003A7470D498F23AA3C
:102EF000E70C03A7070D1345F5FF45BFB7170040C3
:102F000083A6470D1347F5FF758F23AAE70C03A788
:102F1000070C598D4DB7B717004003A7470D498FD0
:102F2000EDB7797122D43714004026D24AD0035924
:102F300024028354040206D64209C2044ECE52CC67
:102F400056CA13590901C1802DE11379F9F793F499
:102F5000F49F4209C20413590901C18093078008F4
:102F6000F3B7078093F787083EC401000100930779
:102F700070052300F404930780FA2300F404010091
:102F80000100231124032310940223000404A24708
:102F9000F3A7078001000100B25022549254025955
:102FA000F249624AD24A45618280B7F507008146FC
:102FB0003000B105194597000020E7806081A247E5
:102FC00013972701E34A07FC1369090893E40440B7
:102FD00093098008F3B7098093F787083EC0010082
:102FE0000100930A700523005405130A80FA230098
:102FF000440501000100231124032310940223003F
:1030000004048247F3A7078001000100294597F0D7
:10301000FF1FE7802032F3B9098093F989084EC277
:1030200001000100230054052300440501000100B4
:103030008357040293E707202310F40223000404BB
:103040009247B9B7B7170040884742054181937747
:10305000050491EB9377F5013755E80113050580D9
:103060003345F50282809377050C130700046397BC
:10307000E7009377F50137459C1CCDB72165130513
:1030800005D0828037E700E01C435443A183E20669
:10309000D58F1CC1FD572320F7182322F7188280F3
:1030A00013178500B7E700E023A0E710618123A292
:1030B000A7108280B7F700E08847CC47828081471D
:1030C00037370040A14663C4C7003285828003457C
:1030D000B740E38EA6FE3385F5000345050085075E
:1030E0002304A740CDB797070020938727EF9C4381
:1030F000173700201307071C3E95636EE50017374E
:103100000020130727506368A70017070020232714
:10311000A7EC3E858280FD57EDBF8280411122C41D
:1031200006C62A8497000000E78000F22947B3070B
:10313000E502B2408D83B3D7870222449507B3D707
:10314000E70237370040C207C1832316F700410169
:103150008280411137150E0006C697000000E780F7
:1031600020FCB7370040130770F82381E7000D47B4
:10317000A381E70013070004A380E7000547238726
:10318000E700B24041018280373700408347270083
:103190001A0593F7F703C98F93F7F70F2301F70089
:1031A0008280B737004003C7170019C9D98DA380A3
:1031B000B70003C70700136787002380E7008280FA
:1031C00093C5F5FFF98DA380B7008280AE872A876B
:1031D000B736004021463738004089E71703000022
:1031E0006700E3F383C8B600E30916FF05078348C9
:1031F000F7FFFD17C20723041801C183F9BF41116E
:1032000022C406C62A8497000000E780E0E329472D
:10321000B307E502B2408D83B3D7870222449507F6
:10322000B3D7E70237370040C207C1832316F74000
:1032300041018280716541111305052006C6970082
:103240000000E78000FCB7370040130770F82381C7
:10325000E7400D47A381E74013070004A380E74040
:1032600005472387E740B24041018280CC414111AC
:1032700006C6328503C6150083C5050022064D8E9D
:1032800042068D654186138875A2630C0611634B57
:10329000C804138845A26300060D634AC8009385DD
:1032A00035A26301B6082390060029464DA0138875
:1032B00055A26305060D938565A2E316B6FE8D45FE
:1032C0001D4663E6E5081146198E63F3C7003E8686
:1032D000B7E704002390C600FC4797D5010093850B
:1032E000652D9DA0138895A263030611634E060DFC
:1032F0001388A5A263000613938505A5E315B6FA06
:1033000099451D4663E5E504198E63F3C7003E86C3
:10331000B7E704002390C600FC479705002093857B
:1033200025D61DA09D451D4663E3E5022146198E65
:1033300063F3C7003E86B7E70400FC472390C6004E
:103340009705002093858534BA9582970146B2404F
:10335000328541018280AD451D46E3EAE5FE3146F6
:10336000198E63F3C7003E86B7E704002390C600BA
:10337000FC4797D5010093856526F9B7B1451D46F1
:10338000E3E7E5FC3546198E63F3C7003E86B7E7F1
:1033900004002390C600FC4797D5010093850525BE
:1033A00065B78D451D46E3E4E5FA1146198E63F3D2
:1033B000C7003E86B7E704002390C600FC4797D5B8
:1033C00001009385E51F49B78D451D46E3E1E5F80A
:1033D0001146198E63F3C7003E86B7E704002390B9
:1033E000C600FC4797D5010093850522B1BFA545CE
:1033F0001D46E3EEE5F42946198E63F3C7003E86C9
:10340000B7E704002390C600FC4797D501009385D9
:10341000E51B1DBFB5451D46E3EBE5F23946198EA8
:1034200063F3C7003E86B7E704002390C600FC475D
:1034300097D501009385051701BFB7E7040003A3E3
:103440000713970600209386A6C24146A545170597
:1034500000201305E5B802832D455DE703C505008F
:103460000947631FE50803A84500411106C6034745
:10347000180032850346080022074168518F9308DF
:1034800028FE6307170563E9E800051863030703CF
:1034900023900600294591A8130648FE630AC70435
:1034A0001518E31707FF15463E87637BF60015479F
:1034B00001A8130600023E876374F600130700029A
:1034C000B7E704002390E600FC471316070111A894
:1034D0003E8691C30546B7E70400FC472390C6002B
:1034E0004206CC45418282970145B240410182802B
:1034F000130600083E87E375F6FC13070008C9B7FA
:103500002390060005458280828041677917630415
:10351000E504411122C406C685472A84639FF5004D
:10352000B7E7040022852244B24003A3871397051E
:1035300000209385E52F4101028389476399F500B7
:10354000B7E7040083A7070B8545829771D9B2407E
:103550002244410182808280797126D252CCAE848D
:103560002A8A97D501009385250C17D501001305EC
:10357000250E06D63AC622D44AD0368432894ECE9B
:1035800097B00100E780205FA28517D501001305E1
:10359000250D97B00100E780005E294597B0010036
:1035A000E780406283C7840093F70702F9E383C989
:1035B00004008947054532476396F908D44083C71C
:1035C000160083C60600A207D58FC166138616FEB5
:1035D000638CC7028D16638FD7068D6693862690FF
:1035E00029456391D706B7E70400A286225403A3B6
:1035F0004714B250F2494A86A68502599254528520
:10360000624A8547456102832D450DEF930700020D
:10361000354563E98702B7E70400FC47C844130651
:103620000002CA8582978149970700209387072166
:103630009C43014581CB9C4391C74E852286CA8518
:1036400082970145B250225492540259F249624A7B
:10365000456182802D457DF79307700F3545E3E383
:1036600087FEB7E70400FC47C8442286CA858297D4
:1036700065BF2145C1BF411122C437E4040083273F
:10368000841326C2AA84416506C697050020938547
:10369000251A7D1582978327C40A17050000130594
:1036A00005E78588829795C0032304132244B2401E
:1036B000924497060020938626AE4146C5451705DD
:1036C00000201305659C41010283B24022449244CC
:1036D00001454101828019C59707002023A0A71644
:1036E00001458280454582801147636AA70A97D6C3
:1036F0000100938626F20A0536951841411106C647
:103700003697AE87B2850287130700026145639D35
:10371000E700B7E70400FC47130600021705002086
:10372000130545F782970145B24041018280054764
:103730006145E39BE7FEB7E70400FC470546170534
:103740000020130525F7F9BF1307700F6145E39DAE
:10375000E7FCB7E70400FC471306700F17050020CD
:10376000130585F5C1B7130700086145E39EE7FA25
:10377000B7E70400FC4713060008170500201305EF
:1037800025034DB715476145E390E7FAB7E7040015
:10379000FC471546170500201305C50961B7094503
:1037A0008280411126C2B7E4040083A7C41322C457
:1037B0004AC006C62E8497050020938565072A898E
:1037C0008297058905C5970700209387E78B83D7E4
:1037D000A70BA28503A3440D2310F4002244B2409A
:1037E00092444A850249014641010283B240224483
:1037F0009244024949454101828097070020238174
:1038000007049707002023AF0702B717004003A75C
:10381000070CB706C0FFFD16758F23A0E70C03A7A2
:10382000070DB7064000558F23A8E70C03A7070C28
:103830003D9B23A0E70C03A7070D1367070123A8EF
:10384000E70C8280B717004003A5470C83A7470CFD
:10385000598113451500C18B058999E3136525002E
:103860009707002083C7C7FD6380A7029707002042
:103870002388A7FC11C9970700209387A7FC03A3FF
:1038800007006303030002838280114517F3FFFFE3
:10389000670063C8411193962500AA852D4506C689
:1038A00097F0FF1FE780C0F2B240014541018280DE
:1038B000011122CC06CE3714004026CA4AC84EC693
:1038C00052C483447405034AB405834984050349FB
:1038D000940597F0FFFFE780E09E8347A40593F4EB
:1038E000F40F137AFA0F93E71700230DF40493F9FA
:1038F000F90F1379F90FB717004003C7A705058B18
:103900006DFF03D5C705A38D4705238C3705A38C11
:103910002705A38B9704F2406244D2444249B2493E
:10392000224A0561828041119397050122C406C68F
:1039300026C2C1872E8463DC0700B7E40400FC5470
:10394000829719C1BC5482972165218D15A893F7E0
:10395000150013C515008DE793F725009DC7970047
:103960000000E78060EEB7E70400BC4F1306000AD2
:10397000894517050020034565ED8297134524000E
:10398000B24022449244410182809397250163D83A
:103990000702B7E4040083A7C41E829797000000C3
:1039A000E780E0EEBC4C3756070013060630896509
:1039B00017050020034585E98297096579B7939734
:1039C00015010145E3DE07FA17D50100130545D1BE
:1039D00097B00100E7800032B7E70400BC4F130640
:1039E0000064916517050020034545E6829711653F
:1039F000A9BF2D71232A9110FD74E98C232C81100D
:103A000023282111232631112A84AE893289930675
:103A100000100A86A6852D45232E111097F0FF1F52
:103A2000E78000DB13154401B7E70400FC47518130
:103A30000A0513962900CA850A958297A685856688
:103A40000146254597F0FF1FE78080D80A86A685A6
:103A500093060010294597F0FF1FE78060D7832069
:103A6000C1110324811183244111032901118329E8
:103A7000C11015618280B7F7070003C70701411124
:103A800006C622C426C24AC0A547631DF700970098
:103A90000000E78040F6B2402244924402490145CA
:103AA0004101828013942500AA843289A286AA85C6
:103AB0000146254597F0FF1FE78080D1A2864A8600
:103AC000A685294597F0FF1FE78080D0E9B71D71D3
:103AD000A2CC37E404005C5C485886CE494697D5B2
:103AE0000100938565BB829711E917D50100130585
:103AF000E5BB97B00100E780E01F01A0B7F600E04A
:103B0000795798CAFD57DCCA0567B7E700E023A0DC
:103B1000E7101306F00290C223A0E718010001008D
:103B20003707002018471306000481459706002038
:103B300023ACE6D04157A38AE7403C44080882976B
:103B4000970700209387876D3EC8856713870740D6
:103B5000231AE1001D673ACC370701051307071048
:103B60003ACE938757D11307B00F2310E1022312E7
:103B7000F102054797F7FFFF938707542301E102FE
:103B80003ED817070000130727D197070000938737
:103B900067D2B7F50700BAC23EDC1707000013076B
:103BA000C7ED97070000938787CE81463000E10577
:103BB0001945BAC43EDE97F0FF1FE78060C11808C0
:103BC0008147994630003E96034606008507050763
:103BD000A30BC700E398D7FEC24791C70357410123
:103BE00085676373F70001A0B7E7040083A7470A5E
:103BF00008088297AA8511C917D50100130545AC9D
:103C000097B00100E78020F701A0F64066442561E7
:103C10008280411126C2B7E4040083A7040806C6C7
:103C200022C417050000130545D082971704002011
:103C30001304C4C12300A40097000000E7808002A1
:103C400097000000E780A0BB03450400224403A3C3
:103C50008405B24092441306003289654101028313
:103C6000797106D622D413078008F337078093F7BB
:103C700087083EC201000100B71700409305700598
:103C80002380B704130680FA2380C70401000100D3
:103C900083C6F70293F6A60FA387D70223800704F3
:103CA0009246F3A606800100010073370780137760
:103CB00087083AC4010001002380B7042380C704A9
:103CC0000100010003C7F70213672700A387E7027B
:103CD00023800704A247F3A70780010001000545E0
:103CE00097E0FFFFE780406197000000E78020BA7F
:103CF000014781468147054685451305407E97E08B
:103D0000FFFFE780406437E404003C44680051460C
:103D100081458297B707C0A83EC8B787E803938755
:103D200007D03ECA97E7FF1F938767693EC67C5856
:103D300068008297B250225445618280411197D524
:103D400001009385250017D501001305659006C66F
:103D500097B00100E78020E217D501001305451751
:103D600097B00100E78020E1B2402945410117B337
:103D70000100670023E5411197D501009385C5FD3A
:103D800017D501001305C58C06C697B00100E78062
:103D900080DE17D501001305651297B00100E7809A
:103DA00080DDB2402945410117B30100670083E17E
:103DB000411122C406C6834705002A849DC797D5B2
:103DC0000100938525FF17D501001305658897B07D
:103DD0000100E78040DA4C4017D501001305851D2E
:103DE00097B00100E78020D93DA058410DEF97D54D
:103DF0000100938525FC17D501001305658597B053
:103E00000100E78040D717D501001305251C97B0A6
:103E10000100E78040D62244B2402945410117B352
:103E20000100670023DAA1679386D7036313D702E3
:103E300097D50100938505F817D501001305458135
:103E400097B00100E78020D317D5010013050519AD
:103E50007DBFED0797D501009385C5F517C5010016
:103E60001305057F631BF70097B00100E780A0D022
:103E700017D501001305C51759BF97B00100E7809A
:103E800080CF4C4017D501001305851891BF411113
:103E900097D50100938585ED17C501001305457B76
:103EA00006C697B00100E78000CDB2402945410128
:103EB00017B30100670003D1797122D426D24AD00A
:103EC0002E842A898145B2844800714606D697E03F
:103ED000FFFFE780C02297F7FF1F9387E74CDC477F
:103EE00083D70700231421012313F100975000000A
:103EF000E780C0E89547A305F1009307401F3EC641
:103F0000FD572305A100230AF10097500000E78028
:103F100020FB2686A285480097500000E780E0E855
:103F2000B250225492540259456182809717002062
:103F30002399077E971700202382076EB7E70400B6
:103F4000BC47411106C641468145170500201305AF
:103F5000651B829797200000E780C06497200000CF
:103F6000E780C043014597500000E78000761707BF
:103F700000200347271B9307F00A6315F7029307F6
:103F8000F0F88945170500201305C519170700200B
:103F9000230AF71897070020A386071897600000E8
:103FA000E780409D97600000E780A0C98145370504
:103FB00004009707002023A5071497070020239FDC
:103FC000071297070020238C071297070020239BD6
:103FD000070A970700202399070897070020239EC8
:103FE0000710970700202397071297300000E780FB
:103FF000202C014597600000E780C0A097D5010004
:10400000938545D917C501001305856497B0010054
:10401000E78060B617D501001305C50597B001000C
:10402000E78060B5B2402945410117B30100670040
:1040300063B9411122C406C626C293F715002E8427
:10404000638F0710814617F6FF1F13062633854539
:10405000170500200355050197C00000E780602385
:1040600015C997D501009385A5D317C50100130580
:10407000255E97B00100E78000B017C50100130569
:10408000E57497B00100E78000AF294597B00100C3
:10409000E78040B397D50100938585D017C501000F
:1040A0001305055B97B00100E780E0AC17C5010080
:1040B0001305057397B00100E780E0AB294597B081
:1040C0000100E78020B017F5FF1F1305E52D5C45C3
:1040D00005472390E70097400100E780E0D397D59C
:1040E00001009385E5CB17C501001305655697B010
:1040F0000100E78040A817C501001305A56F97B020
:104100000100E78040A7294597B00100E78080AB18
:10411000930710F8170700202306F70097070020E1
:1041200083D707F417070020A30EF7FE170500201A
:10413000130545FFA1839145170700202305F7FECE
:1041400097070020A38107FE97600000E780808228
:1041500013451400B240224492444101828093F7F7
:104160002500E1C717070020035747F945CF9706F9
:1041700000209386E6F8944297D70100938787F151
:10418000170600200346A6F78145170500201305F2
:1041900065F797700000E780202F97F7FF1F23999E
:1041A000A710AA8441C197D50100938525C617C5DC
:1041B00001001305E54997B00100E780C09BA68583
:1041C00017C501001305856497B00100E780A09A28
:1041D000294597B00100E780E09E97070020239FC4
:1041E00007F0930710F817070020230DF7F2970741
:1041F000002083D7E7E617070020A305F7F2A18385
:10420000170700202301F7F291458D47170500207D
:10421000130545F117070020A307F7F0975000009A
:10422000E78040751345240035B793F74500D1C3A7
:1042300097D50100938585BD17C50100130545413C
:1042400097B00100E780209317C501001305C55DF5
:1042500097B00100E7802092294597B00100E780E0
:104260006096930720F817070020230DF7EA9707B9
:10427000002083D727E117070020A305F7EAA183D1
:10428000170700202301F7EA854717070020A30C32
:10429000F7E897500000E780A0C21705002013053B
:1042A00065E8914597500000E780C06C13454400D5
:1042B00055B593F78500A9C797D50100938505B536
:1042C00017C501001305C53897B00100E780A08A23
:1042D00017C501001305855697B00100E780A08936
:1042E000294597B00100E780E08D970700202397CC
:1042F00007E097700000E78000291345840099BD0E
:1043000093F70501D1C3854517050020035585D7CF
:1043100097600100E78020DB97D50100938505AF0A
:1043200017C501001305C53297B00100E780A084CE
:1043300017C501001305C55197B00100E780A083A0
:10434000294597B00100E780E087930730F8170709
:1043500000202309F7DC9707002083D7A7D217078F
:104360000020A301F7DC170500201305A5DBA183BE
:104370008D45170700202308F7DA97500000E780E3
:10438000605F13450401F9B393F70502D1C797D5D0
:1043900001009385A5A717C501001305652B97A0FC
:1043A0000100E780407D17C501001305A54C97A0CB
:1043B0000100E780407C294597B00100E7808080BC
:1043C000930740F817070020230EF7D49707002023
:1043D00083D787C917070020A306F7D4A18317073F
:1043E00000202302F7D4854717070020A30DF7D23A
:1043F00097070020239A07C697500000E78040AC3B
:1044000017050020130505D2914597500000E7805D
:104410006056134504023DBB93F70504FDC397D5D1
:1044200001009385A59E17C501001305652297A07D
:104430000100E780407417C501001305254597A0CA
:104440000100E7804073294597A00100E78080774D
:104450009707002083C707CD1307700A6386E70616
:104460001307800A638CE7081307600A6393E70465
:10447000930760F8170700202306F7CA9707002064
:1044800083D7A7C717070020A30EF7C8A183170774
:104490000020230AF7C8854717070020A309F7C89B
:1044A000B145170500201305E5C797500000E780C8
:1044B000604C97500000E780A0A0134504049707C4
:1044C0000020239C07C279B1930770F817070020DA
:1044D000230AF7C49707002083D727C217070020B5
:1044E000A302F7C4A18317070020230EF7C2854754
:1044F00017070020A30AF7C2994565B7930780F80C
:10450000F1B793F705080145E38607C497D5010085
:104510009385C58F17C501001305851397A001006A
:10452000E780606517C501001305C53797A0010036
:10453000E7806064294597A00100E780A0689307A1
:10454000A0F817070020230FF7BC9707002083D798
:1045500067BC17070020A307F7BCA183170700203B
:104560002303F7BC854717070020A30EF7BA970768
:104570000020239107BA97500000E7806094170548
:104580000020130525BA914597500000E780803E32
:1045900013450408C1B6411122C497D50100938583
:1045A000A5822A8417C501001305850A06C697A0AF
:1045B0000100E780405C4C4017D501001305059DC4
:1045C00097A00100E780205B294597A00100E780C4
:1045D000605F034704009307F00F631FF70297C55E
:1045E00001009385657E17C501001305650697A038
:1045F0000100E78040584C4017D501001305059A8B
:1046000097A00100E78020572244B240294541018C
:1046100017A301006700035BB2402244410182807E
:10462000B1C1411122C417C50100130565022E84D2
:1046300097C501009385457406C697A00100E780E1
:104640008053A28517D50100130585A097A001000E
:10465000E78060522244B2402945410117A301007E
:10466000670043568280411122C426C22E84AA8448
:1046700097C501009385057117C50100130545FD18
:1046800006C697A00100E780004F17D5010013056B
:10469000E59C97A00100E780004E294597A0010006
:1046A000E780405297C501009385C56D97070020AC
:1046B000239A979A17C50100130585F98544970732
:1046C0000020239F879897070020239C979897178F
:1046D00000202398870497A00100E780C049971520
:1046E000002083D5050417D501001305A59797A0D1
:1046F0000100E7804048294597A00100E780804CF1
:1047000097170020238C97F097200000E78000C9BE
:10471000228597500000E78040FB05459750000038
:10472000E780402E97F7FF1F938707C8DC4703D722
:104730000700C167FD176312F7022244B7E70400C0
:10474000B240924403A3870517F5FF1F0345851068
:104750001306000A854541010283B2402244924477
:1047600041018280011122CC37E404005C5C06CE5A
:10477000354697C501009385E57617D501001305E9
:10478000A544829711E917C50100130525F297A0EA
:104790000100E780205601A097F7FF1F9387470C81
:1047A0003EC4B7F50700856793870780814617F6F3
:1047B000FF1F1306660AE10519453EC697E0FF1F75
:1047C000E78000017C44194697F5FF1F9385C508D3
:1047D000170500201305458B8297340017F6FF1F3D
:1047E0001306860797D50100938505C117D50100EB
:1047F000130505C297700000E780009E2A841DCD36
:1048000097C501009385855F17C50100130545E431
:1048100097A00100E7802036A28517C50100130587
:10482000656D97A00100E7800035294597A001003C
:10483000E7804039F24062440561828097E00000E1
:10484000E780600017C501001305C561976000008F
:10485000E780409297A00000E780A0549760010095
:10486000E78020B917F5FF1F130585B09760010099
:10487000E780C0A117C501001305C55F976001005F
:10488000E780A0B92A8497600000E78080F897103D
:104890000100E780009197800100E780202A97704F
:1048A0000000E780C05097600000E780806E97307E
:1048B0000100E780605297C501009385255417C514
:1048C00001001305E5D819C897A00100E780A02AC8
:1048D000A28517C5010013052564A1B797A00100A3
:1048E000E780602917C501001305456597A0010001
:1048F000E7806028294597A00100E780A02C973029
:104900000100E780402E97F00000E780004D55C978
:1049100085453705040097300000E780609997C50A
:1049200001009385A54D17C50100130565D297A019
:104930000100E780402417C501001305A56197A079
:104940000100E7804023294597A00100E7808027E8
:1049500097F7FF1F9387C79483D707001717002087
:104960002311F7DC8547171700202309F7CA972082
:104970000000E780E0BB97200000E78020A2171529
:104980000020035505DA97500000E78000D4054564
:1049900097500000E780000797C501009385054602
:1049A00017C501001305C5CA97A00100E780A01C28
:1049B00017C501001305455C97A00100E780A01B07
:1049C000ADB597C501009385654317C50100130573
:1049D00025C897A00100E780001A17C5010013053C
:1049E000656997A00100E7800019294597A001009B
:1049F000E780401D014569BF411122C437E404002E
:104A00008327041A06C6829797500000E780A0CF3C
:104A10008327040817F5FFFF1305E561829797F7D1
:104A2000FF1F2389A7E217F5FF1F1305E59797409E
:104A30000000E780807B2244B24041011703000060
:104A4000670083D2B7E70400FC471171A2DDCAD921
:104A500086DFA6DBCED72E8432892E86AA8517F56F
:104A6000FF1F1305256C829717F7FF1F1307876B2E
:104A700083470700930680029387E70793F7F70FB2
:104A8000E3ECF610BA898A0717C70100130787C538
:104A9000BA979C43BA9782878D4797C50100938543
:104AA000253817C501001305A5BA630FF40097A0B8
:104AB0000100E780400C17C50100130525F597A0FC
:104AC0000100E780400BBDA497A00100E780A00A89
:104AD00017C50100130505F597A00100E780A0099F
:104AE000294597A00100E780E00D930720F81146C3
:104AF00097F5FF1F938505634A8517F7FF1F23036B
:104B0000F76297F7FF1FA380076297F0FFFFE78028
:104B1000E03A2A841DC997C501009385653017C501
:104B200001001305E5B297A00100E780C004A2854B
:104B300017C501001305C5F297A00100E780A00387
:104B4000294597A00100E780E00797C501009385FC
:104B5000252D17C501001305A5AF97A00100E7801B
:104B6000800117C501001305E5F097A00100E7805B
:104B70008000294597A00100E780C00441659307A4
:104B800030FA054697F5FF1F9385C5597D1517F730
:104B9000FF1F2309F75897F0FFFFE78020322A8490
:104BA0001DC997C501009385A52717C501001305E9
:104BB00025AA97A00100E78000FCA28517C5010087
:104BC000130505EA97A00100E780E0FA294597A0C0
:104BD0000100E78020FFB7E70400BC4F056613061D
:104BE00006C8A14517F5FF1F0345C5C68297FE50AD
:104BF0006E54DE544E59BE59116182809147630351
:104C0000F40297C501009385A52117C5010013057E
:104C100025A497A00100E78000F617C50100130541
:104C2000A5E871BDB7E70400FC4F914517F5FF1FDC
:104C3000034545C2829797C501009385651E17C538
:104C400001001305E5A097A00100E780C0F217C599
:104C50000100130525E797A00100E780C0F1294571
:104C600097A00100E78000F697400000E78040250C
:104C7000914535A485476303F40297C501009385E8
:104C8000251A17C501001305A59C97A00100E78010
:104C900080EE17C50100130565E415B597F7FF1FF2
:104CA0002392273FB7E704000566BC4F130606C8EA
:104CB000C1450DBF8D476303F40297C5010093857D
:104CC000251617C501001305A59897A00100E780D8
:104CD00080EA17C50100130525E2D5B3930740F814
:104CE000114697F5FF1F9385E5434A8517F7FF1F88
:104CF000230AF74297F7FF1FA387074297F0FFFFAA
:104D0000E780C01B2A84E30405EE97C50100938564
:104D1000251117C501001305A59397A00100E78091
:104D200080E5A28517C50100130585D397A0010072
:104D3000E78060E4294597A00100E780A0E845BD31
:104D40009147E31CF4F6B7E70400FC4F930500021B
:104D500017F5FF1F034505B0829797C5010093859E
:104D6000250C17C501001305A58E97A00100E7804B
:104D700080E017C501001305A5D9F1BD894763E39C
:104D8000870297C501009385A50917C50100130582
:104D9000258C97A00100E78000DE17C501001305F0
:104DA00065D831BB97F4FF1F83C4E43797F7FF1F23
:104DB00083C7573797C5010093858506A20417C599
:104DC00001001305E588DD8C97A00100E780A0DADB
:104DD000A28517C50100130525D697A00100E7801D
:104DE00080D9C204294597A00100E780A0DDC184D5
:104DF0009305D4FF93960401C1824A8693F5F50F7B
:104E000017F5FF1F1305353297200000E780004E8D
:104E1000E35F90DC930750F817F7FF1F2304F73088
:104E200083C73900228697F5FF1F9385A52F850735
:104E30004A8517F7FF1FA308F72E97F0FFFFE780BB
:104E4000E0072A84E30505DA97C50100938545FD4F
:104E500017B501001305C57F97A00100E780A0D119
:104E6000A28517C501001305A51DC9B5894763E3D0
:104E7000870297C501009385A5FA17B501001305B0
:104E8000257D97A00100E78000CF17C5010013051D
:104E900065CC35B197400000E7808002A28517F508
:104EA000FF1F1305252897500000E780A0AC81B3B1
:104EB0008D476303F40297C50100938565F617B526
:104EC00001001305E57897A00100E780C0CA17C567
:104ED00001001305E5C9E5B6B76602000146B775DE
:104EE0000200054597E0FF1FE780808E930760F87A
:104EF00017F7FF1F2308F72297F7FF1FA385072245
:104F00009307000617F7FF1F2300F722894717F7BB
:104F1000FF1FA30BF72097F7FF1F2388072097F7A2
:104F2000FF1FA3840720C14717F7FF1F2300F720A7
:104F3000930720F917F7FF1FA30AF71E314697F7CB
:104F4000FF1FA386A71E97F5FF1F9385A51D4A8502
:104F500097F7FF1F238D071C97F0FFFFE78000F6F0
:104F60002A84E30605C897C50100938565EB17B54C
:104F700001001305E56D97A00100E780C0BFA28581
:104F800017C50100130545C055B3B1476303F402CB
:104F900097C501009385C5E817B501001305456B5A
:104FA00097A00100E78020BD17C50100130585BF4C
:104FB00039B6B7E70400FC4F9305000417F5FF1F4F
:104FC00003454589829797400000E78060EFB1452F
:104FD000F9B5914763E3870297C50100938545E4DE
:104FE00017B501001305C56697A00100E780A0B8BA
:104FF00017C501001305C5BCD9B497F4FF1F83C4BE
:10500000A41297F7FF1F83C71712A204DD8C8E042A
:10501000B77702006D14BE942286A68517C50100DD
:10502000130545BB97A00100E780E0B4B7E7040093
:10503000FC47228697F5FF1F9385150F280082975E
:1050400093160401C1823000A685094597D0FF1F41
:10505000E78000782A8409C917C50100130545B9FE
:1050600097A00100E78000C9930770F8194697F5EB
:10507000FF1F9385250B4A8517F7FF1F2304F70AA7
:1050800097F7FF1FA382870A97F0FFFFE78000E3EF
:105090002A84E30E05B497C50100938565D817B53A
:1050A00001001305E55A97A00100E780C0ACA28576
:1050B00017C501001305C5B495B99947630BF412E0
:1050C00097C501009385C5D517B50100130545584F
:1050D00097A00100E78020AA17C501001305C5B3FA
:1050E000F9BA914763E3870297C50100938545D3D9
:1050F00017B501001305C55597A00100E780A0A7CB
:1051000017C501001305C5B25DBA97F4FF1F83C42C
:10511000A40197F7FF1F83C71701A204DD8C8E043B
:10512000B77702006D14BE942286A68517C50100CC
:10513000130545B197A00100E780E0A3B7E704009D
:10514000FC47228697F5FF1F938515FE280082975E
:1051500093160401C1823000A6850D4597D0FF1F2C
:10516000E78000672A8409C917C50100130545AF08
:1051700097A00100E78000B8930780F8194697F5DB
:10518000FF1F938525FA4A8517F7FF1F230CF7F8B1
:1051900097F7FF1FA38A87F897F0FFFFE78000D2F9
:1051A0002A84E30605A497C50100938565C717B552
:1051B00001001305E54997A00100E780C09BA28587
:1051C00017C50100130505AB95B699476303F402B3
:1051D00097C501009385C5C417B501001305454760
:1051E00097A00100E780209917C50100130505AAC3
:1051F000F9B0B7E70400FC4F9305000417E5FF1F63
:1052000003454565829797400000E78060CB99454C
:1052100079B18D476303F40297C50100938545C0BA
:1052200017B501001305C54297A00100E780A094BF
:1052300017C50100130505A759B017C501001305CF
:1052400065A797A00100E780E0AA1305C01297D0D8
:10525000FF1FE780000F014597E0FFFFE780C0E2F6
:105260000D4597100000E78060A1294597D0FF1FEA
:10527000E780200D97D0FF1FE78080FD8DBA99470A
:105280006303F40297C50100938585B917B5010042
:105290001305053C97A00100E780E08D17C50100CC
:1052A000130505A229B817F7FF1F0347F7E797F77C
:1052B000FF1F83C767E722075D8F9166BA96C20614
:1052C0001166C1821306F6EF8D476365D60297E734
:1052D000FF1F9387670D9C4B17F6FF1F0346B6E42D
:1052E0009386C7002DC203D6070069CA8907E39CCD
:1052F000D7FE89471307A0F8114697F5FF1F93853E
:1053000065E24A8597F6FF1F238EE6E017F7FF1F39
:10531000A30BF7E097F0FFFFE78040BA2A84E30889
:10532000058C97C501009385A5AF17B5010013053E
:10533000253297A00100E7800084A28517C50100EF
:1053400013054599E5B203D60700630EE60A8907FF
:10535000E39BF6FE8D4779BF91476304F40297C53E
:1053600001009385E5AB17B501001305652E97A0E5
:105370000100E780408017C50100130525976FF0F5
:105380000FF4B7E70400FC4F9305000817E5FF1F73
:105390000345454C8297C9B897C50100938545A838
:1053A00017B501001305C52A97900100E780A07C7E
:1053B00017C50100130505956FF06FF02390E70006
:1053C00017E5FF1F130545FE97300100E78020A772
:1053D00097C501009385C5A417B50100130545279E
:1053E00097900100E780207917C501001305859289
:1053F00097900100E7802078294597900100E78089
:10540000607C8147C5BD2390070017E5FF1F13058A
:10541000A5F997300100E78080A297C50100938528
:1054200025A017B501001305A52297900100E7807C
:10543000807417C501001305658F5DBF411122C43B
:1054400006C6834705002A849DC797C5010093853A
:10545000E59817B501001305A51F97900100E78097
:1054600080714C4017C501001305C5C3979001001A
:10547000E7806070E1A05841B707CF009387777D40
:10548000631DF70697C501009385459517B5010083
:105490001305051C97900100E780E06D1C448356BE
:1054A000E4008355C40003C6070017C501001305B7
:1054B000E5C097900100E780006C294597900100B6
:1054C000E78040700357E4009707002083D76725E3
:1054D0006309F7008355C400084497E0FFFFE780A5
:1054E00020CF0356E4008355C40008442244B24050
:1054F000410117F3FFFF67002355B707CC009387DF
:10550000777D6315F70497C501009385258D17B541
:1055100001001305E51397900100E780C0651C4466
:105520008356E4008355C40003C6070017C5010075
:105530001305C5B897900100E780E0632244B240AC
:1055400029454101179301006700C367B707CE00E3
:105550009387777D6304F70297C5010093850588DB
:1055600017B501001305C50E97900100E780A060F4
:105570004C4017C501001305A5A9CDBDB24022447A
:1055800041018280B7E70400FC4741112E8606C620
:1055900022C426C24AC02E842A89AA8517F5FF1F75
:1055A000130545B8829797C501009385258917B5DE
:1055B00001001305E50997900100E780C05B97F5AE
:1055C000FF1F83C525B617B501001305252F97903A
:1055D0000100E780405A294597900100E780805EEE
:1055E00097F4FF1F938404B483C704004147938753
:1055F000070693F7F70F636AF75C17B70100130705
:10560000A7188A07BA979C43BA9782879D47630772
:10561000F40297C501009385658217B50100130553
:10562000250397900100E780005517B50100130589
:10563000652997900100E7800054ADAC97F7FF1FF4
:1056400083C757AEDDCB17F7FF1F0347D7AD97F7DB
:10565000FF1F83C747AD22075D8F97F7FF1F83C7E3
:10566000A7ACC2075D8F97F7FF1F83C7F7ABE207B1
:10567000D98F17F7FF1F2325F7A883C7640097B5B5
:1056800001009385A57B17B50100130565FC17F78D
:10569000FF1F2306F7A697900100E780C04D97F7FC
:1056A000FF1F9387E7A58C4317F6FF1F034626A528
:1056B00017B501001305C52297900100E780A04BA4
:1056C000294597900100E780E04F97F7FF1FA38BD4
:1056D00007A42244B24092440249930700F817F706
:1056E000FF1F2301F7A49D4517F5FF1F130585A391
:1056F0004101174300006700E32797600000E7803F
:1057000000F897F7FF1F2380A7A29357850017F78C
:10571000FF1FA30AF7A0935705012A8417F7FF1F5D
:105720002304F7A093578501014517F7FF1FA30D29
:10573000F79E97600000E78040F597F7FF1F2386EC
:10574000A79E97B501009385656F17B501001305F6
:1057500025F097900100E780004217F6FF1F0346EF
:10576000C69CA28517B5010013050519B1B7CD4731
:105770006303F40297B501009385456C17B50100EA
:10578000130505ED97900100E780E03E17B5010095
:105790001305051879BD37E404007C44414697F5AC
:1057A000FF1F9385359817F5FF1F1305A595829761
:1057B00017F5FF1F1305059597100000E78040D3EC
:1057C00097100000E78080BD97F7FF1F83C7A7965B
:1057D00017F7FF1F03471796A20703238405D98FE6
:1057E00017F7FF1F231CF7901306000A8945224470
:1057F000B2409244024917E5FF1F0345A505410148
:1058000002838D476303F40297B501009385056316
:1058100017B501001305C5E397900100E780A03597
:1058200017B501001305851E29B517F4FF1F0344A2
:10583000848F97F7FF1F83C7F78E97B50100938575
:10584000E55F220417B50100130585E05D8C979094
:105850000100E7804032A28517B501001305C50C91
:1058600097900100E7802031294597900100E7805B
:1058700060350D4697F5FF1F9385C58A228597E011
:10588000FFFFE780A063AA8421C197B5010093853B
:10589000E55A17B501001305A5DB97900100E780D5
:1058A000802DA68517B501001305450997900100C5
:1058B000E780602C2244B2409244024929454101CC
:1058C000179301006700033097E7FF1F239C877A37
:1058D000B7E70400116603A38705130606E89145A0
:1058E00039B78D476303F40297B5010093850555D9
:1058F00017B501001305C5D597900100E780A027D3
:1059000017B501001305451F2DB317F4FF1F0344FE
:10591000848197F7FF1F83C7F78097B501009385B0
:10592000E551220417B50100130585D25D8C9790CF
:105930000100E7804024A28517B501001305450149
:1059400097900100E7802023294597900100E78088
:1059500060270D4697E5FF1F9385C57C228597E05C
:10596000FFFFE780A055AA841DC197B5010093856C
:10597000E54C17B501001305A5CD97900100E78010
:10598000801FA68517B501001305C5FD05B797E76C
:10599000FF1F239B876CB7E70400116603A38705ED
:1059A000130606E89305000299B5894763E3870269
:1059B00097B501009385854817B50100130545C9C2
:1059C00097900100E780201B17B50100130585158E
:1059D0008DB197E4FF1F83C4047597E7FF1F83C74A
:1059E000777497B5010093856545A20417B501004A
:1059F000130505C6DD8C97900100E780C017A685CA
:105A000017B50100130585F797900100E780A016F0
:105A1000294597900100E780E01A228697E5FF1F4D
:105A200093854570268597E0FFFFE78020492A840B
:105A3000630E051A97B501009385454017B501001F
:105A4000130505C197900100E780E012A28517B504
:105A500001001305E5F399BD854763F98718834570
:105A600019002244B24092440249B335B00097E78E
:105A7000FF1F2383B76217B501001305A5F241018B
:105A8000179301006700230FA2852244B24092447D
:105A90004A850249410117030000670063249947C2
:105AA0006303F40297B501009385453917B50100EA
:105AB000130505BA97900100E780E00B17B50100C8
:105AC00013050520BDB617E4FF1F0344C46597E71F
:105AD000FF1F83C7376597B50100938525362204DC
:105AE00017B501001305C5B65D8C97900100E780DE
:105AF0008008A28517B50100130545EC97900100B9
:105B0000E7806007294597900100E780A00B1946C0
:105B100097E5FF1F93850561228597E0FFFFE780EA
:105B2000E039AA841DC197B501009385253117B5C9
:105B300001001305E5B197900100E780C003A68539
:105B400017B50100130585E895B397E7FF1F239369
:105B5000875CB7E70400116603A38705130606E810
:105B60009305000869B1854797B501009385052D18
:105B700017B501001305C5AD630BF4009790010044
:105B8000E78060FF17B50100130585E55DB49790C8
:105B90000100E78040FE17B501001305E5E5979089
:105BA0000100E78040FD294597900100E7808001D2
:105BB0002244B2409244024997E7FF1F23900754C2
:105BC0004101176300006700039C97B501009385AE
:105BD000E52617B501001305A5A797900100E780FA
:105BE00080F917B501001305E511A1B4B2402244B4
:105BF0009244024941018280411106C622C497E0C5
:105C0000FFFFE780A02B21CD97E7FF1F83D7E74851
:105C100085072A8417E7FF1F2311F74897B501006E
:105C20009385452397E7FF1F239AA74617B50100E1
:105C3000130505A297900100E780E0F3A28517B550
:105C400001001305E53F97900100E780C0F2224470
:105C5000B24029454101179301006700A3F697E779
:105C6000FF1F83D7C743B2402244850717E7FF1FB2
:105C70002317F74241018280411122C491462A84B0
:105C800017E6FF1F130606589D652D4506C697D0DB
:105C9000FF1FE780E0B3B7F7070003C70701A54779
:105CA0006313F70001A09306001001469D6525458A
:105CB00097D0FF1FE780C0B197E7FF1F2384875469
:105CC0002244B240914617E6FF1F1306A6539D6576
:105CD0002945410117D3FF1F670083AF1171CED74C
:105CE000B7E9040083A7C904CAD917E9FF1F13093C
:105CF0006943A2DD2E8686DFA6DB2E84AA854A852F
:105D0000829797E7FF1F83C7E7411307700A6385F0
:105D1000E710636DF7001307600A6385E704FE5020
:105D20006E54DE544E59BE59116182801307800AA9
:105D30006385E7161307900AE393E7FE8D47630632
:105D4000F41C97B501009385E54217B501001305D2
:105D5000259097900100E78000E217B50100130538
:105D6000A53E25A08D47630CF40297B501009385ED
:105D7000654017B501001305A58D97900100E780D8
:105D800080DF17B501001305653597900100E780A6
:105D900080DE294597900100E780C0E249B785473A
:105DA00017B501001305453517E7FF1F2306F72E2A
:105DB00097900100E78000F4B7750200B766020013
:105DC0000146054597D0FF1FE78080A0930760F844
:105DD00017E7FF1F2308F73497E7FF1FA385073452
:105DE0009307002617E7FF1F2320F734E5779387F3
:105DF000072117E7FF1F231BF732B14597E7FF1F66
:105E00002387073297E7FF1FA383A7324A859700AE
:105E10000000E780E01621B7914763E3870297B55A
:105E200001009385253517B501001305658297900C
:105E30000100E78040D417B501001305E52DB1B787
:105E400097E4FF1F83C4442E97E7FF1F83C7B72D36
:105E5000A204DD8C83A7C9046D14228697E5FF1F79
:105E60009385952C280082978E0493160401B775AC
:105E70000200C1823000A695094597D0FF1FE78038
:105E80002095930770F817E7FF1F230DF728994512
:105E900097E7FF1FA38AA72895BF914763E387026F
:105EA00097B501009385052D17A501001305457AC7
:105EB00097900100E78020CC17B501001305452716
:105EC000E9B597E4FF1F83C4242697E7FF1F83C724
:105ED0009725A204DD8C83A7C9046D14228697E55B
:105EE000FF1F93857524280082978E049316040162
:105EF000B7750200C1823000A6950D4597D0FF1FEF
:105F0000E780008D930780F8BDBF17B5010013052A
:105F1000E52497900100E780E0DD930790F82304E3
:105F2000F100834719008D452800A304F100834741
:105F300029002305F10097000000E78060041305A5
:105F4000C01297C0FF1FE780C03F014597D0FFFFF9
:105F5000E78080130D4597000000E78020D2294597
:105F600097C0FF1FE780E03D97C0FF1FE780402EEE
:105F70007DB397E7FF1F23AFA728828097E7FF1F16
:105F80009387472903A30700630303000283174392
:105F900000006700239E41114AC097F6FF1F83D679
:105FA0004678328917D6FF1F0356264222C426C2DE
:105FB00006C62A84AE8497000000E780A06635C13B
:105FC0002DC0994763FF97048347140003470400DB
:105FD000A207D98F13978700A183D98FC207316792
:105FE000C1831307C755639EE70297D7FF1F83D767
:105FF000C73DA301F400A1832302F40097F7FF1F1C
:1060000083D7277291C7A302F400A1832303F4006E
:10601000A68517B501001305E51997900100E780E3
:1060200080B597F7FF1F83C7675FB9CF97D5FF1F6D
:1060300083D5A53917B5010013058519979001007F
:10604000E78060B32686A28517D5FF1F0355E53785
:1060500097000000E78080BA6301090497E7FF1FFB
:1060600083C7871B9DCB95C897E7FF1F83C7C702D0
:106070008DE722852244B2400249A685924441011F
:10608000174300006700038F17B50100130545157E
:1060900097900100E78000C6C1B7B2402244924405
:1060A000024941018280834755008345450017B569
:1060B00001001305E50EA207DD8D179301006700AF
:1060C00083AB17B501001305A50C179301006700FA
:1060D00063C28D4763FBB70A011126CA06CE22CCE4
:1060E0000344350097E4FF1F83C4141397B50100E0
:1060F0009385C50FB337800017E7FF1FA30EF71076
:1061000009C497B501009385250F17B50100130544
:10611000250F97900100E78000A697E7FF1F83C730
:10612000B70F6386970097000000E780603097E71D
:10613000FF1F83C7770E8DC785472306F100B7E79A
:10614000040083A7471770008545130550308297D8
:1061500017B501001305C50B97900100E78080B9C2
:106160009967938757EE2316F1006800854791459C
:10617000A30781002307F10097000000E78040E0BB
:10618000F2406244D244056182808280894763F78D
:10619000B708011122CC06CE26CA834425008547C4
:1061A0002A84639DF404914763F5B70403454500D1
:1061B0008347340022055D8D97D7FF1F2397A720C3
:1061C00097000000E780E04E9967938767EE2314FD
:1061D000F1008347340023059100A305F1008347B4
:1061E0004400954528002306F10097000000E78051
:1061F00020D9F2406244D24405618280FDF899675B
:10620000938767EE2314F10097D7FF1F83D7E71B0F
:10621000A305F10023050100A183E1B782800111EC
:10622000996722CCD51717F4FF1F1304243F2314BA
:10623000F1008347040026CA97F4FF1F9384644E3D
:106240002305F10083D7040028009545A305F1003C
:10625000A18306CE2306F10097000000E78040D21C
:1062600003D604008345040017B501001305C5FBE0
:1062700097900100E7802090F2406244D24405618B
:1062800082809D677971D9172316F10097F7FF1F58
:1062900083C7C73806D62307F100A9C3B7E70400B0
:1062A000FC47414697E5FF1F9385C5E51305F100BF
:1062B00082976800CD4597000000E78060CC97F595
:1062C000FF1F83C5A53517B501001305E5F89790A5
:1062D0000100E780408AB25045618280B7E7040040
:1062E000BC47414681451305F1008297D9B745C5A2
:1062F000411106C622C4930750FA2300F500930704
:10630000A005A300F50089472301F5009147A301EB
:10631000F50093079002A302F50097F7FF1F9387FC
:10632000E72F83C70700230205002A842303F50013
:1063300097E7FF1F938757EE83C70700414697E50E
:10634000FF1F938525DCA303F50097F7FF1F83D775
:10635000473D2304F500A183A304F50097D7FF1F51
:1063600083D7A7062305F500A183A305F500B7E7AA
:106370000400FC47310582972285F1459700000013
:10638000E7804026230EA4002181A30EA400B24082
:1063900022444101828082805D710A8586C6A2C442
:1063A00097000000E780E0F437E404007C448A852D
:1063B0000810794682973C441305E103094681455C
:1063C0008297101093050002014597D0FFFFE780E8
:1063D000E031B640264461618280011122CC2A84DA
:1063E000680006CE26CA4AC8AE84328902C697D053
:1063F000FFFFE78060C9A28585660146254597C0F5
:10640000FF1FE780E03CCA862686A285294597C003
:10641000FF1FE780E03B324597D0FFFFE78080C851
:10642000F2406244D2444249056182800111B7C7FB
:10643000A55A22CC9387C73317E4FF1F1304D4DD7A
:106440003EC4834704002C002146196506CE3EC693
:1064500097000000E780A0F88345040017B501000D
:10646000130545F097800100E780E070F240624438
:10647000056182800111A146300099652D4522CC2D
:1064800006CE97C0FF1FE780A034A24737C4A55AA5
:106490001304C43363958702B24517B50100130591
:1064A000A5DFB335B00097E7FF1FA387B7D6978066
:1064B0000100E780406CF240624405618280916592
:1064C000A1463000938505F02D4597C0FF1FE7805A
:1064D0002030A247E38287FC97E7FF1FA38E07D2F5
:1064E000814517B50100130565DDD1B7B7C7A55ABA
:1064F00079719387F7353EC6B7E70400FC4706D6A7
:10650000AA854146080882976C005146116597009C
:106510000000E780C0EC17B50100130565E897801F
:106520000100E780207DB250456182807971D146BB
:10653000700091652D4522D406D697C0FF1FE780D5
:106540002029B24737C4A55A1304F435639887024B
:10655000B7E70400FC4717E5FF1F1305A5BA41463E
:106560000C08829717B50100130545DB97800100E1
:10657000E7804078B2502254456182809165D146CF
:106580007000938505E82D4597C0FF1FE7804024E4
:10659000B247E38F87FA17B50100130525DAF9B77B
:1065A0000111680006CE02C697D0FFFFE780C0AD9C
:1065B000856601469165254597C0FF1FE78040210C
:1065C000324597D0FFFFE780E0AD17B50100130516
:1065D000E5CA97800100E780E071F24005618280A2
:1065E000C16769768146FD17050613970601418349
:1065F0006364B7003E8582803307D50003470700F8
:10660000B98F214713F81700858363050800B18F00
:10661000C207C1837D171377F70F6DF78506F1B7B2
:1066200041C5A547054763F2B708834715000347EF
:1066300005003168A207D98F13978700A183D98FEE
:10664000C207C1831308C855054763900707411166
:1066500006C622C426C203442500914763F087047E
:106660009307540063ECF502A301C50021822302C5
:10667000C5009304340091C6A302D500A182230370
:10668000D5002A84A68597000000E780A0F526940F
:106690002300A4002181A300A4000147B2402244AA
:1066A00092443A854101828005473A8582800111F2
:1066B000B7C7A55A22CC9387E7342A842AC6214635
:1066C0002C00156506CE3EC497000000E78020D15F
:1066D000A28517B501001305E5CA97800100E78080
:1066E000804997000000E78060CBF240624405617A
:1066F00082800111A146300095652D4522CC06CE41
:1067000097C0FF1FE780C00CA24737C4A55A1304E7
:10671000E43463958702B24517B50100130505BC43
:1067200097D7FF1F2393B7CAC205C1819780010085
:10673000E7806044F2406244056182809165A14631
:106740003000938505EE2D4597C0FF1FE780400878
:10675000A247E38287FCD14717D7FF1F2317F7C64D
:10676000D14517B50100130565B9C9B721C141115C
:1067700026C206C622C4AE848DC52A8497000000B6
:10678000E780406497E7FF1F83C707A999CB22855D
:106790002244B240A68592444101173300006700AD
:1067A000631DB240224492444101828082800111E3
:1067B0004AC806CE22CC26CA4EC693F715002E89AB
:1067C0009DCBAD67371700409387A7AA1CC3B7E7D7
:1067D0000400BC4F13060019854517D5FF1F03455C
:1067E000A5BE829713451900F2406244D244424943
:1067F000B2490561828093F72500638A071C17F769
:10680000FF1F0357E7F1954763F9E70C014417F6BB
:10681000FF1F1306E6E09306300513055004130826
:1068200010049308B0041303900593076400637485
:10683000F7043A84FD5997F4FF1F83C464DE97F789
:10684000FF1F83C7F7DDA204DD8CAD679387B755C3
:10685000638BF41463E3970AA9679387A755638E44
:10686000F414A28517F5FF1F130585DB97000000C0
:10687000E78000F031A2B307860083C50700639A62
:10688000D50483C517006396A50483C527006392CA
:10689000050583C53700639ED50283C54700639A0B
:1068A000150383C7570063966702A2890DE897F521
:1068B000FF1F83D5E5E6B3853541C20517F5FF1FF8
:1068C000130505D6C1814E9597000000E78040EA88
:1068D000E1A005044204418089BF3A84FD598547FF
:1068E000E3EB87F45DC4854517F5FF1F130545D31A
:1068F00097000000E780C0E769A8B1679387C75594
:106900006380F404B5679387D755E39CF4F4A285BC
:1069100017F5FF1F1305C5D097300000E7808005ED
:106920008947630FF4049305E4FFC205C18117F59D
:10693000FF1F130505CF97000000E780A04889A03E
:1069400097200000E78080F597000000E780E04690
:1069500011C9A28517F5FF1F130585CC970000000C
:10696000E78040460546A28517F5FF1F130545CB76
:1069700097F0FFFFE780606297200000E78000F259
:10698000A68517B501001305A5A397800100E78030
:10699000801EFD57E39DF9F097F7FF1F239207D85C
:1069A0001345290091B5A28517F5FF1F130545C7AB
:1069B00097F0FFFFE780606FE1B7A28517F5FF1F33
:1069C000130505C697F0FFFFE780E06F55BF93F70B
:1069D00045000145E38A07E017B501001305859FCF
:1069E00097800100E780003197300000E780202782
:1069F00013454900D5BB411122C437E404005C5C57
:106A000006C6354697A501009385C54D17B501000B
:106A10001305851B829711E917B501001305459CE5
:106A200097800100E780002D01A08327041C829736
:106A30002A84054597C00000E78040E09760010088
:106A4000E780606597600100E780603A97B00000DA
:106A5000E780C0F12285B24022444101828015675F
:106A6000B71700401307575598C3D8439D66558FF5
:106A7000D8C3D843FD76758FD8C3D8431367F70FB3
:106A8000D8C335671307C7CC98C382804111054529
:106A900006C622C426C297C0FFFFE780C048130580
:106AA000A00497B0FF1FE7808060757585457D1550
:106AB00097C0FFFFE78060327D7585451305F53689
:106AC00097C0FFFFE780C03B371400408327840A4C
:106AD0008D451305002093E707202324F40A97C06F
:106AE000FFFFE780802FB7E4040097C0FFFFE78037
:106AF000A074C85897800100E780C01F17B5010037
:106B00001305850C97800100E780C01E8327840C45
:106B10008545414593E707082324F40C97C0FFFF00
:106B2000E78000368D451305000897C0FFFFE7801A
:106B3000203597C0FFFFE780006237A507001305E7
:106B4000051297C0FFFFE780A05D014597C0FFFFDA
:106B5000E780C06395450545894717F7FF1F230365
:106B6000F7BC97C0FFFFE7800064B7E700E01307BA
:106B70000006238DE7403707000423A0E71097D0D5
:106B8000FFFFE78000F597D0FFFFE780C008970080
:106B90000000E78080E697000000E780E08D970026
:106BA0000000E78040B597E0FFFFE78020E5970011
:106BB0000000E780602297000000E780600B83A759
:106BC0000408170500001305C5BE829797C7FF1F6D
:106BD000238CA77EBC4C13060064854582979700E2
:106BE0000000E78000E897C0FF1FE7806080014554
:106BF0008280B7F7070003C70701A547AE86631673
:106C0000F7009397450191C301A0AA850146254548
:106C100017C3FF1F6700C3BB4111B2862E86AA852A
:106C20002D4506C697C0FF1FE78080BAB2400145D8
:106C3000410182809307000463E8C7021D71A2CC62
:106C40002A84080886CE32C697800100E78040E794
:106C5000B2461008A285294597C0FF1FE78040B7BC
:106C6000F6406644256182803955828041110D6568
:106C70008D4506C697C0FFFFE7802016B717004076
:106C80008D6623A6D70A17F5FF1F1305E5A91387FD
:106C9000C70A9387870A1CC15CC5856689675CC97A
:106CA00058C114C518C9B7E70400B24003A3871E32
:106CB000410102838145B307B5008387070089E757
:106CC00017230000670023C48505C205C181E5B70D
:106CD00097B701009387C78A1357C5003E970347AC
:106CE0000700011106CE2304E100135785003D8BF8
:106CF0003E970347070023060100A304E100135752
:106D000045003D8B3D893E97AA970347070083C7FF
:106D1000070028002305E100A305F100970000000B
:106D2000E78080F9F24005618280411126C2E9774F
:106D300097F4FF1F9384C4AF22C49387A7552E8472
:106D40002381B4002E86AA8517F5FF1F130585AE93
:106D500006C62390F400A381040097800100E78019
:106D600020D693052400C205C18117F5FF1F130526
:106D700045AC97000000E780E086B387840023825B
:106D8000A7002181A382A700930564002244B2409A
:106D900026859244C205C181410117230000670086
:106DA00083B609C99307800263E6B70017030000A2
:106DB0006700E3F7828017F5FF1F0345659882801F
:106DC00097F7FF1F83C787A689E71723000067008F
:106DD00083B3828097F7FF1F83C767A899EF41119C
:106DE00006C697200000E780E0A9B240854717F764
:106DF000FF1F2306F7A64101828082806307054AB0
:106E00006385054A5D71CAC04EDE86C6A2C4A6C2AD
:106E100052DC56DA5AD85ED662D466D26AD0B94706
:106E20002A89AE8963F9B706394697A5010093858B
:106E3000E56297800100E78040C631ED8347E900B5
:106E4000130710036394E702854717F7FF1F230F0B
:106E5000F79C17A501001305656197F7FF1F23969F
:106E6000079C97000000E78020E571A0130700034E
:106E700017A5010013058562E395E7FE97F7FF1F4D
:106E80002386079A97F7FF1F2391079A17A50100FA
:106E90001305455FF9B797F7FF1F83C727996387E6
:106EA0000722BD6AB96B938CFA55014A17FBFF1F85
:106EB000130B4B89138CEB65938AFA6605A8B3070D
:106EC000490183C6070097F7FF1F83D70796B1E3F1
:106ED0009307A005639BF600854717F7FF1F23164E
:106EE000F79497F7FF1F238FD784050A93170A019A
:106EF000C183E3E637FDB640264496440649F2597D
:106F0000625AD25A425BB25B225C925C025D616162
:106F10008280054D639BA7039307500A639EF6008A
:106F2000894717F7FF1F2312F790930750FA17F7B7
:106F3000FF1FA309F78055BF9307A005E387F6FA63
:106F400097F7FF1F2393078E4DB71387170042074C
:106F5000DA9741832380D70017F6FF1F2317E68CAB
:106F60008D47E3F4E7F817E4FF1F0344D47D97E768
:106F7000FF1F83C7477D22045D8C9307F4FFC20780
:106F8000C1839306F00DE3EDF6FA93076400C207A0
:106F9000C183E31CF7F493052400C205C18117E502
:106FA000FF1F1305457A97F0FFFFE780A0633307C3
:106FB0008B008347570003474700A207D98F17F775
:106FC000FF1F231407866318F50E8144630CA40188
:106FD00097E4FF1F83C44477A20497E7FF1F83C78A
:106FE000B776DD8C170500001305E5DB97F0FFFF92
:106FF000E78060F863878407636D9C029387EB5595
:107000006382F40497E7FF1F83C70774054763890A
:10701000E70681CB1387A7051377F70F8D4663F239
:10702000E6081307F0072300E100A300F1008945FB
:107030009DA063829405E39754FD97F0FFFFE780DE
:10704000802411A8A28517E5FF1F1305E56F97F0AF
:10705000FFFFE7804008014597F0FFFFE780A0F1C0
:1070600069B5A28517E5FF1F1305056E97F0FFFFB1
:10707000E7800012CDB797F0FFFFE780801AE1BFED
:10708000930710F8130511002300F10097F0FFFF9C
:10709000E7802026FD450A8597000000E78020C98B
:1070A0005DBFA28517E5FF1F1305056A97F0FFFF77
:1070B000E78000C34DB79307F00789450A85231081
:1070C000F10097000000E78080C605B5BD4763F872
:1070D0003717414697A501009385853E4A859780DD
:1070E0000100E780809B631C051417A501001305B0
:1070F000653E97000000E78020BC17E5FF1F0355A1
:10710000456297000000E780E0BC97E7FF1F83C758
:10711000E75017A501001305653389E717A501009E
:107120001305453397000000E78000B917A501005B
:107130001305C53B97000000E78000B817C5FF1F87
:107140000355452697000000E780C0B817A5010049
:107150001305053A97000000E78000B617C5FF1F2A
:107160000355A52697000000E780C0B617A50100CB
:107170001305853897000000E78000B417D5FF1F7E
:107180000355E5F197000000E780C0B417A50100A2
:107190001305053797000000E78000B217D5FF1FE1
:1071A0000355A5EF97000000E780C0B217A50100C6
:1071B0001305853597000000E78000B017D5FF1F45
:1071C0000355C5ED97000000E780C0B017A501008A
:1071D0001305C53397000000E78000AE17C5FF1FF9
:1071E0000355050D97000000E780C0AE17A501000C
:1071F0001305453297000000E78000AC97D7FF1FCA
:1072000083C747F0A20717D5FF1F0345B5EF5D8D74
:1072100097000000E78000AC97D7FF1F83C7A7EE59
:10722000A20717D5FF1F034515EE5D8D97000000DF
:10723000E78040AA17A50100130545A21DB1C1476B
:1072400063FE3705414697A501009385E52C4A85E5
:1072500097800100E780608431E1834709011307CB
:107260001003639CE700854717E7FF1F230AF74CCD
:1072700017A501001305852BEDB61307000317A50D
:1072800001001305A52DE39EE7BC97E7FF1F2389A7
:10729000074A17A501001305E52AE1B6CE854A8500
:1072A00097C0FFFFE780C0F2B9B18280411126C2CA
:1072B000AE848D4522C406C62A8497C0FFFFE780AE
:1072C00020BCB717004099C803A5C70C418D23A661
:1072D000A70CB240224492444101828003A5870C4E
:1072E000418D23A4A70CF5B783470500034715007C
:1072F000A207D98FC2076177C18713072720639A36
:10730000E7008345250037050400170300006700E8
:1073100023FA828017E6FF1F1306C6548147B28600
:107320001303F00FA9483308F6000348080013F7C9
:10733000F70F6307A80C630668008507E39517FF3E
:107340002947B387E6002380A70097E7FF1F9387AD
:1073500027525DA8411113D765001347170006C6D1
:1073600093F63500058B954791CA05469947638783
:10737000C60009469D476383C600A14713F6450032
:107380003336C00093F68503050685C2A145638B9D
:10739000B604E145638AB604930580026388B604A7
:1073A000930580036393B600914697E5FF1F2386FC
:1073B000F57297E5FF1F2381C57297E5FF1FA38D27
:1073C000D570BE8517A501001305851F97700100B4
:1073D000E780607AB240854717E7FF1FA30FF76E7B
:1073E000410182808546D1B78946C1B78D4675BFB8
:1073F00017A501001305451F177301006700A37748
:1074000017E7FF1F1307C746BA972380B700E14766
:10741000E302F5F493077002E30CF5FC82802A87FF
:1074200023800500814717E5FF1F1305A5431308B7
:10743000F00F2946B306F50083C606006396E60200
:1074400097E6FF1F9386C642B69783C70700054598
:107450002380F5009947636EF7029D4763FDE700BF
:10746000E147630DF7008280638506018507E3939A
:10747000C7FC0145C5B7238005008280B7370040AF
:1074800003C7370083C7050093F70704D98F23800C
:10749000F50082805D7152DC56DA5ED6716A97EB38
:1074A000FF1F938BAB748D6AA6C24EDE62D486C674
:1074B000A2C4CAC05AD866D26AD06ECEC1495E8C08
:1074C00097E4FF1F9384843B130A0A20938A7ADC93
:1074D00017E9FF1F03498974B3872B0183C707008E
:1074E00093F7F70FC9EFB787004003C76700058B15
:1074F000E310077C03C76700118BE30D077E83C78A
:107500005700918B99E36F10200317E7FF1F034784
:10751000077185476304F7006F10400197E7FF1F6D
:10752000A38DE75A97E7FF1F238A074097E7FF1FBE
:107530002388074C97E7FF1F2386075897E7FF1F0D
:107540002383075897E7FF1FA38A073E97E7FF1F8C
:10755000A388074A97E7FF1FA386075697E7FF1FF1
:10756000A383075697E7FF1FA38A075697E7FF1FD6
:10757000A387076AB787004011476F0070779307AA
:10758000190093F7F70F3D476364F70617E7FF1FEE
:107590002306F76897E7FF1F93874767CA9783C754
:1075A00007001307100293F7F703638EE71E636665
:1075B000F70405446385871CE38C07620947638EE3
:1075C000E71013070002E384E74EB7E700E0370750
:1075D000400023A0E7180100010062992300090080
:1075E000FD1923A0E71093F9F90FE39309EEE5BD28
:1075F00097E7FF1F2384076271BF13073002638878
:10760000E70C63E8E71613074002638CE70A1307E9
:107610000003E39CE7FA97E7FF1F9387275ECA976B
:1076200003C70700A1471377F70FE31BF71483C7BE
:10763000640097E6FF1F2389F64897E7FF1F83C77B
:10764000572491C7FD5797E6FF1F238FF64697E50E
:10765000FF1F83C5B52297E7FF1FA387B74697E7AC
:10766000FF1F83C7A72113FB07089306000493F7A6
:107670000706639FD74C9307A009638DF51663EA4D
:10768000B7129307F0056386F54A930750096384A0
:10769000F52A014497E7FF1F83C717431547E39275
:1076A000E736B7E700E03707400023A0E7180100FE
:1076B0000100B786004023808602130680FC6F001D
:1076C000500EFD5717E7FF1F230FF73EFDBDFD5777
:1076D00017E7FF1F2308F73ECDBD17A501001305CF
:1076E000250297700100E780E06097E7FF1F93870E
:1076F000E750CA9703C40700014B97ECFF1F938C18
:107700006C301374F40F17AD0100130DEDFF6347D8
:107710008B04294597700100E780C04A854717E729
:10772000FF1FA30FF72C17E7FF1F230C872C17E76A
:10773000FF1F2305F73A37E700E0B7064000232094
:10774000D71801000100378600408347A60293F74F
:10775000370F2305F6022320D71085BDB3876C01B0
:1077600083C507006A85050B97700100E780A0407C
:1077700079BF854717E7FF1F2304F728B9B517E737
:10778000FF1F1307A7474A970347070097E6FF1F06
:10779000A386F61A97E6FF1F2383E61A17E7FF1F53
:1077A000230EF7321DB5854717E7FF1F2308F7188B
:1077B00029BD9307400A6389F5349307200B63843E
:1077C000F5369307100AE396F5EC8387240001440D
:1077D000E3D207EC97E7FF1F83C7770A93F63700DA
:1077E000638A061A0546638AC62209466395C61A45
:1077F0001D4755A217E5FF1F03456508C94797ECCC
:10780000FF1F83CCDC0797E5FF1F83C5650717E4DF
:10781000FF1F0344F4066315F510CD476392FC1077
:1078200093077008639CF5021307300FB7170E001B
:107830006308E4001307900DB7B704006314E4086D
:1078400017E7FF1F2328F728BE8517A5010013059A
:1078500025EC97700100E780003225BD9307800872
:10786000639DF500B307804013F4F70FB777460028
:10787000938787CDB3D78702E1B793079008639AC0
:10788000F500B307804013F4F70F91679387C7663D
:10789000D5B79307A008639BF500B307804013F4A6
:1078A000F70FB7173D0093870790E9B79307B00824
:1078B000639AF500B307804013F4F70F916793873D
:1078C00097D04DBF93F5F5078D47639BF500B30740
:1078D000804013F4F70FB7975B00938707D859BF21
:1078E0008947639BF500B307804013F4F70FB77720
:1078F0000B009387071BBDBF8547639AF500B3074D
:10790000804013F4F70FDD67938767E3A5B7D2874D
:1079100085F9B307804093F7F70FB3D7FA020DB795
:1079200097000000E780409FA285668597000000D1
:10793000E780809EB9BB9305610017E5FF1F0345F3
:1079400005F417E4FF1F034494F397000000E78059
:1079500040AD93057100228597000000E78060AC80
:107960003C0017E7FF1F2321F7288347610023040A
:10797000F10083477100A304F100894717E7FF1F57
:107980002304F7148357810017E7FF1F2318F7EE2E
:10799000094409B3154793F64700B336D00093F76F
:1079A0008703850685C32146638BC7066146638AC4
:1079B000C706130680026388C70613068003639315
:1079C000C700914717E6FF1F2308D61097E6FF1F51
:1079D000A384F61097E7FF1F2381E71017E7FF1F27
:1079E000034707EA9376070497E7FF1F83C757E922
:1079F0008DEE1377770C93067008630CD70213771C
:107A0000F7078D466312D70CB307F040B7955B00BC
:107A100093F7F70F938505D849A81947ADBF854758
:107A200055B7894745B78D4771BF930670086311F5
:107A3000D7021307300FB7150E006389E70213074B
:107A4000900DB7B504006383E7021307700845BFC4
:107A50009306800C6311D702B307F040B775460058
:107A600013F7F70F938785CDB3D5E70297E7FF1F8D
:107A700023A2B706D9BB9306900C631CD700B307AB
:107A8000F04093F5F70F91679387C766B3D5B702B8
:107A9000F1BF9306A00C631DD700B307F040B715E4
:107AA0003D0093F7F70F93850590B3D5F5027DBFA1
:107AB0009306B00CE315D7F4B307F04093F5F70F36
:107AC0009167938797D0D9B78946631BD700B307CF
:107AD000F040B7750B0093F7F70F9385051BF1B7CF
:107AE0008546631AD700B307F040DD6593F7F70FBB
:107AF000938565E35DBFD28535FBB305F04093F513
:107B0000F50FB3D5BA029DB783C72400C18B99C7BF
:107B1000854717E7FF1F230CF7FAA5BE97E7FF1F5E
:107B2000238707FABDB6854717E7FF1FA307F7FAB4
:107B30008DB63C0017E7FF1F2328F70A0947930774
:107B400000032314F10097E6FF1F238FE6F62DBDF7
:107B500063940756A94763E5B74217A701001307C7
:107B600067A38A05BA959C41BA97828717E4FF1FDD
:107B70000344F4D0894C6306940D63E68C06854774
:107B80006303F4089307F00F17E7FF1F0347C7F3DA
:107B900063F6E70017E7FF1F2308F7F297ECFF1FD4
:107BA00083CC8CF29307000413F4FC0F63F4970169
:107BB0001304000497E7FF1F9387070303AD070033
:107BC00022862685EA85B38C8C40229D9770010021
:107BD000E78000EF97E7FF1F238897EF97E7FF1FE6
:107BE00023A4A70145BC8D47630CF40A9947E31B06
:107BF000F4F897A70100938767A017E7FF1F2325D5
:107C0000F7FEA94751B717E7FF1F0347470197E75B
:107C1000FF1F938767ED494697A50100938505A748
:107C20006306870097A50100938545A23E8597705E
:107C30000100E780E0E817E7FF1F2327A7FAC947FD
:107C4000A1B797E6FF1F83C686FD054797E7FF1F8D
:107C5000938787E96394E6023E851306700297A531
:107C60000100938525A097700100E78060E517E784
:107C7000FF1F232BA7F69307700239B73E85130623
:107C8000300497A501009385259897700100E7803F
:107C900020E317E7FF1F2329A7F493073004EDB56E
:107CA00097E5FF1F83C5A5BD17A50100130585A78F
:107CB00097700100E78020EC054D97EDFF1F83CD05
:107CC0000DF697E5FF1F83C585BB17A501001305BA
:107CD00065A56398AD0B97700100E780C0E997E751
:107CE000FF1F83C7C7B9B5CBE36EF4E817A4010043
:107CF0001304049E638CB70117A401001304C49DF0
:107D00006386970117A401001304849E228597704F
:107D10000100E780E0061375F50F9307150086074D
:107D200017E7FF1F2302F7DC8D4717E7FF1FA30D9F
:107D3000F7DA97E7FF1F938727DB0147BE861376A5
:107D4000F70F89076365A60297E7FF1F23AED7E801
:107D500097E7FF1F83C747D905BD97A70100938702
:107D6000279017E7FF1F2321F7E8914731BD33061E
:107D7000E40003460600A380070005072380C70030
:107D80007DBF97700100E78000DF97E7FF1F83C783
:107D900007AFE1D7E368F4DE17A4010013044490B1
:107DA000638CA70117A40100130404906386970154
:107DB00017A401001304C490228597700100E78086
:107DC00020FC1375F50F93071500860717E7FF1FB3
:107DD000230CF7D08D4717E7FF1FA307F7D097E7CE
:107DE000FF1F938767D00147BE861376F70F890779
:107DF000E37CA6F43306E40003460600A3800700F4
:107E000005072380C700D5B797E5FF1F83C525A7C2
:107E100017A501001305C59197700100E780A0D553
:107E200097E7FF1F83C717CC93E7470017E7FF1FAC
:107E3000A30AF7CA83C7240017E7FF1FA302F7CAE4
:107E400089B817A501001305E58F97700100E78039
:107E500060EA97E7FF1F9387A7C883C7070017E764
:107E6000FF1F230DF7A017E4FF1F0344E4C53334BD
:107E700080000DB017A501001305058E9770010055
:107E8000E78040E797E7FF1F83C7D7C593E7070160
:107E900017E7FF1FA308F7C483C7240017E7FF1FD6
:107EA0002300F7C46FF0EFFE17A501001305058C42
:107EB00097700100E78000E403C704007D8B51EF59
:107EC000B787004003C767021377C70B1367270004
:107ED0002383E70203C7A7021377C70B13672700A3
:107EE0002385E70203C7E7021377C70B1367270051
:107EF0002387E70203C727031377C70B13672700FE
:107F00002389E702854717E7FF1F2309F7A217E731
:107F1000FF1F2307F7AE17E7FF1F2305F7BA17E781
:107F2000FF1F2302F7BA97E7FF1FA38907A097E770
:107F3000FF1FA38707AC97E7FF1FA38507B897E745
:107F4000FF1FA38207B897E7FF1FA38907B897E72A
:107F5000FF1FA38607CC6FF0CFF389476312F702A8
:107F600097E7FF1F83C7C7919146638CD70863E0EB
:107F7000F604638EE70C6369F70A05476380E70E32
:107F8000FD5717E7FF1FA301F7B437074000B7E716
:107F900000E023A0E71801000100B78600401306A7
:107FA000F0FC2381C60223A0E7106FF00FE2130755
:107FB00020086382E7086362F70213071008E39161
:107FC000E7FC378700408347670293F7C70B93E7C7
:107FD00027002303F7026FF0CFEB13073008638904
:107FE000E70213074008E39DE7F83787004083471F
:107FF000270393F7C70B93E727002309F7026FF0D6
:108000004FE9378700408347270393F73707F5B7D2
:10801000378700408347E70293F7C70B93E72700B2
:108020002307F7026FF0EFE6378700408347E70248
:1080300093F73707F5B7378700408347A70293F7D1
:10804000C70B93E727002305F7026FF08FE437870C
:1080500000408347A70293F73707F5B737870040FB
:108060008347670293F73707ADB7179501001305EC
:10807000E57097700100E780E0C797D7FF1F238F57
:10808000077ED5B317950100130545709770010061
:10809000E78040C697D7FF1F2392077E97E7FF1F11
:1080A000938787A203C40700894763F387000944C5
:1080B0001374F40F6FF00FDE13070002E392E7EC86
:1080C000631B0B0A638FF500930720026383F50897
:1080D000179501001305056F97700100E780A0A9AF
:1080E00045B5179501001305256B97700100E780D2
:1080F00060C00144179D0100130D4D6BA14CB38767
:10810000840083C507006A85050497700100E78035
:1081100080A6E31694FF17950100130525BA977002
:108120000100E78020BD17D4FF1F0344647501E8F8
:1081300097D7FF1F23860772014B6FF0AFD5894792
:10814000E310F4E4854717D7FF1F230BF7706FF098
:108150004FD417D6FF1F0346967297D5FF1F83C5CE
:108160000572179501001305E56497700100E7801B
:1081700080A06FF00FD26380F50693071002E39999
:10818000F5F497D5FF1F83C5A56F1795010013055B
:10819000656497700100E780009E97E7FF1F23A5A5
:1081A00097A497E7FF1F9387E792944383D74700ED
:1081B00017E7FF1F0347679217D6FF1F2320D66CD0
:1081C0001D4497D6FF1F239DF66A97D7FF1F238A6A
:1081D000E76A6FF02FCC97D5FF1F83C5656A1795A7
:1081E00001001305A56097700100E780C09897D73C
:1081F000FF1F2387076697D7FF1F239107686FF03C
:108200002FF92547638FE7C8994637870040639465
:10821000D70223008702B7E700E0B706400023A09B
:10822000D71801000100130600FC2301C70223A098
:10823000D7106FF08FB99306100A639FD700230001
:108240008702B7E700E0B706400023A0D718010077
:108250000100130680FCD1BF9306A009E381D7FE7D
:108260009306400AE38DD7FC93062002639DD70056
:10827000B7E700E0B706400023A0D71801000100CF
:1082800023008702F9B78546E384D7FE93070008E9
:10829000E300FBFEB7E700E0B706400023A0D718D5
:1082A00001000100130620FC23008702BDBF17E771
:1082B000FF1F034777816302F71E63E7E7029547D5
:1082C0006300F7109947630AF704B78600402380DC
:1082D0000602B7E700E03707400023A0E7180100D7
:1082E00001001306A0FC75B99307F005630AF700B7
:1082F000930750096306F70093071002E317F7FC92
:10830000B7E700E03707400023A0E71801000100AD
:10831000B7860040130620FC69B117DBFF1F034B33
:10832000AB7A930700045A8D63F46701130D0004C0
:1083300097E7FF1F9387478B83AC07001374FD0FEC
:108340002286E685268597600100E7806077B3077F
:108350008B40669417D7FF1F2308F77697E7FF1F18
:1083600023A48788B7870040630C0B022380A703F0
:10837000B7E600E03706400023A0C6180100010060
:1083800003C72702134707042381E70203C7270215
:108390001377C70F2381E70223A0C6106FF0EFA267
:1083A0002380070237E700E0B70640002320D718F4
:1083B00001000100130620FC2381C7026FF0AFB952
:1083C000378700408347370097D6FF1F83C6567113
:1083D00093F70708D58FA301F700B7064000B7E76A
:1083E00000E023A0D718010001001306A0FC35BD52
:1083F00097E7FF1F93878780CA9783C7070093F784
:10840000F70FC1CF97E7FF1F83C76781D9E717D75A
:10841000FF1F0347776B930700026310F70883ADD4
:10842000040017DDFF1F034DAD4597DCFF1F83CC14
:108430003C4517DBFF1F034BCB44E6876A87DA8690
:108440006E8697D5FF1F83C5A541179501001305BB
:10845000653B97600100E780007297D7FF1F23AB51
:10846000B76797D7FF1F2389A76797D7FF1FA385F4
:10847000976797D7FF1F2382676797D7FF1FA38050
:10848000873EB7E700E03707400023A0E718010068
:108490000100B78600406FF04FA2B7E700E0370752
:1084A000400023A0E71801000100B786004015BD79
:1084B00097D6FF1F83C6A6760547639CE604294727
:1084C0002381E70209472383E7022385E70297D741
:1084D000FF1FA385076097D7FF1FA3820774B78785
:1084E0000040A381070017D7FF1FA30B075E0547B6
:1084F0002383E700B640264496440649F259625A5F
:10850000D25A425BB25B225C925C025DF24D6161C9
:10851000828029472381E70209472383E7022385D5
:10852000E7022387E7022389E70255B717D7FF1F22
:10853000A307F7326FE01FFF854717D7FF1F230FF1
:10854000F73E17D7FF1F230DF74A17D7FF1F230B3F
:10855000F75617D7FF1F2308F7566FE0BFFE854772
:1085600017D7FF1F230CF73C17D7FF1F230AF74825
:1085700017D7FF1F2308F75417D7FF1F2305F754FA
:1085800017D7FF1FA30C073A17D7FF1FA30A0746E9
:1085900017D7FF1FA308075297D7FF1FA3850752BE
:1085A0008280411106C697000000E78080FBB787F4
:1085B000004023800700130740FC2386E7001307D1
:1085C000C004A386E70017D7FF1F1307272B2398A4
:1085D000E70017D7FF1F1307672E239AE70017D767
:1085E000FF1F1307E739239CE70017D7FF1F130767
:1085F0006745239EE70029472381E7020947238334
:10860000E7022385E7022387E7022389E702A381A4
:108610000700930600F8A380D700930690022380FA
:10862000D700FD562383D7002381E700930600057A
:1086300037E700E0230BD740B70640002320D710D0
:1086400003C7170013671700A380E700B24097D74E
:10865000FF1F2397074841018280411106C69700FA
:108660000000E78000F0B787004023800700130771
:1086700000FC2386E7003147A386E70017D7FF1FDA
:108680001307C71F2398E70017D7FF1F13070723F8
:10869000239AE70017D7FF1F1307872E239CE700B5
:1086A00029472381E70209472383E7022385E7025D
:1086B000A3810700930600F8A380D70093069002D9
:1086C0002380D700FD562383D7002381E70093063C
:1086D000000537E700E0230BD740B7064000232012
:1086E000D71003C7170013671700A380E700B24035
:1086F00097D7FF1F2396073E41018280F16793873A
:10870000072017D7FF1F2327F73C854717D7FF1FE1
:108710002314F73CA14717D7FF1F2300F73C97D737
:10872000FF1FA38C073A97D7FF1F2389073A97D7D4
:10873000FF1F2387071297D7FF1FA38207128147C6
:1087400017D5FF1F13050512FD5517D6FF1F13067A
:1087500026122947B306F5002380B600B306F600BB
:10876000238006008507E397E7FE97D7FF1FA38EB8
:10877000073497D7FF1FA38C073497D7FF1F238792
:10878000073497D7FF1F2382073497D7FF1F238112
:10879000073497D7FF1FA38B073297D7FF1F238874
:1087A0000732814717D6FF1F130646444147B306D9
:1087B000F600238006008507E39BE7FE828017D73B
:1087C000FF1F0347C74585476316F70017030000DF
:1087D0006700E3E8170300006700E3DC411122C4EF
:1087E00006C617D7FF1F0347874385472E8613F416
:1087F000F50FAA856317F70417D5FF1F1305451C4E
:1088000097600100E780C02B97D7FF1F238A071EC0
:10881000B787004023848702B7E600E037064000B0
:1088200023A0C6180100010003C7A7021377C70FD2
:108830002385E702B240224423A0C610014541012E
:10884000828017D5FF1F1305650B97600100E78035
:10885000202797D7FF1F2383070EB7870040238267
:108860008702B7E600E03706400023A0C6180100E3
:10887000010003C767021377C70F2383E7025DBFB9
:10888000411106C697000000E78080E7B240410131
:10889000170300006700E3F2411106C697F0FFFFDF
:1088A000E78080BF97D7FF1F83C75709A1CB97D514
:1088B000FF1F83C5C50889C917D5FF1F13054508C4
:1088C00097E0FFFFE780C05397D7FF1FA3880706F5
:1088D00097D7FF1F2384072037E700E0B706400043
:1088E0002320D71801000100378600408347660225
:1088F00093F7370F2303F6022320D710B24041012C
:10890000828041C9D9C597D7FF1F83C7671DD1C3CF
:10891000011122CC4AC84EC656C25AC006CE26CA3B
:1089200052C42E89AA890144930A0004371B03000C
:1089300063772403B3078940C207C183BE8463F40D
:10894000FA0093040004C204C180130A1BD497D711
:10895000FF1F83C7A7FE9DE37D1A631C0A00F24038
:108960006244D2444249B249224A924A024B0561CA
:10897000828097F0FFFFE78020B2D1BF3385890066
:108980002694A685420497000000E78060E54180B8
:1089900045B7828097D7FF1F9387072C18429C43C7
:1089A00083D645000345070083C5C700035646002C
:1089B0006396A50083D5E700638DD502011106CE2D
:1089C0002386A7002397D700B705CF00DC4B9385FC
:1089D000757D05077D162EC2230001003AC42316BB
:1089E000C1002317D10099C30A858297F24005611F
:1089F00082808280DC4DDC4B81CFB7E7040090455C
:108A000003A38705914517D5FF1F0345252502833D
:108A100082806D713C083EC6B707E50023229110A5
:108A20003EC8AA843C083285232611103ECA23245E
:108A30008110232021112E8997300000E780005EED
:108A40002A8497950100938565DF1785010013053A
:108A500025C097600100E7800012A28517950100EC
:108A6000130545EE97600100E780E0102945976007
:108A70000100E7802015B705CB009385757D680060
:108A800097100000E7802067A285680097300000FB
:108A9000E780204B014781467000CA8526859720D4
:108AA0000000E780A08A05CD2A8497950100938570
:108AB000E5D8178501001305A5B997600100E78087
:108AC000800BA28517950100130585E897600100CA
:108AD000E780600A294597600100E780A00E8320A7
:108AE000C110032481108324411003290110516116
:108AF000828097D7FF1F9387271618429C4379716E
:108B000022D406D60348070083C807012A8483D6E7
:108B10004500035546006396080183D82701638DFD
:108B2000D8022388070105072399D7003708CC000E
:108B3000DC4B1308787D3ACC1307F5FF42CA2308B3
:108B40000100231EE100231FD10099C7080832C687
:108B50002EC482973246A245228597000000E78006
:108B600080EBB2502254456182806D713C083EC05A
:108B7000B707E5003EC23C083EC42326111023245B
:108B800081102322911023170100231801002319BB
:108B90000100231A0100231B010097B7FF1F83D791
:108BA000278599E3C167FD172316F10097B7FF1FCB
:108BB00083D7278491EB97D7FF1F9387E7099C43BF
:108BC0009C43DC4783D7070017B4FF1F130444827C
:108BD000584C2317F10083574400484B2318F100E9
:108BE00031E197950100938565CC17850100130548
:108BF00025A697600100E78000F81795010013058E
:108C000025CC97600100E78000F7294597600100B7
:108C1000E78040FB8320C11003248110832441108E
:108C20005161828097A7FF1F83C7F77C89EBB7E765
:108C30000400BC5782975C4C23AA0700E1BFFD17D4
:108C400097A6FF1FA389F67A0356070183470401FD
:108C50004C470A85230BF10097300000E780802BFA
:108C600097D7FF1F938747FF9C430147814688435F
:108C70000A866C0097100000E780406DAA8429C125
:108C800097950100938585C2178501001305459CC2
:108C900097600100E78020EEA68517950100130577
:108CA000E5C297600100E78000ED2945976001006B
:108CB000E78040F1584CB7E70400BC57484B9DBFD4
:108CC00097A7FF1F83C73773F5D7B7E70400BC4FDB
:108CD0001044854517D5FF1F034545F882971DBFF2
:108CE0005C4EDC4BB9CFB1CD411122C417850100D8
:108CF000130505962E8497950100938565B906C6E0
:108D000097600100E78020E7A28517950100130511
:108D1000A5BE97600100E78000E629459760010045
:108D2000E78040EAB7E704002244B24003A3870586
:108D300017D5FF1F034585F21306400691454101F3
:108D400002838280411122C417A4FF1F1304046808
:108D50001C4C06C689C7DC4399C34C488297584CC3
:108D6000B7E70400BC57484B82975C4CB2402244A2
:108D700023AA07004101828017A7FF1F1307076777
:108D8000834707009306F00B850793F7F70F63E916
:108D9000F60097A6FF1F238BF66403450700828029
:108DA000930700F8FDB7835745006386071001114C
:108DB0004AC817A9FF1F1309A96352C4032AC9018E
:108DC00006CE22CC03274A0126CA4EC656C2F15708
:108DD00035E31307D00DFD57636EC704B7E90400F0
:108DE00083A709072A841305860042054181B284BE
:108DF000AE8A8297232AAA000325C9015C49A9E704
:108E0000979501009385C5A6178501001305458434
:108E100097600100E78020D617950100130505B67D
:108E200097600100E78020D5294597600100E78021
:108E300060D9DD57F2406244D2444249B249224AE5
:108E4000924A3E850561828093874400B705CF0032
:108E50002319F5009385757D310597100000E78093
:108E600080290325C901834564003105973000003E
:108E7000E780200D0325C9012686D6853105973068
:108E80000000E78020097146A2854A8597600100AD
:108E9000E78000C3504419CA83A78905854517D5C3
:108EA000FF1F0345A5DB8297814769B79700000044
:108EB000E780E0CBD5BFFD573E858280411126C2B9
:108EC00097A4FF1F9384C452D84C22C437E40400F3
:108ED0003C54484B06C68297DC4C0323C40522440D
:108EE000B240924423AA070017D5FF1F034505D7B8
:108EF000854541010283411126C297D4FF1F938407
:108F0000A4D59C4006C622C44AC0D5C3DC43C5C311
:108F10005CC12300B5002A84979501009385859054
:108F2000177501001305C57297600100E780A0C4A2
:108F3000294597600100E780E0C89C4023A4070012
:108F400023A2070097A7FF1F93874748DC4FDC4BFE
:108F500091C7295597000000E78000DF97A7FF1F02
:108F600093870749DC4FDC4B89C797000000E780F7
:108F700020F537E904008327C905894517D5FF1F68
:108F80000345C5CD82978327C905914517D5FF1F96
:108F90000345C5CC82979C4003A3470163090300A6
:108FA00022852244B2409244024941010283B240E8
:108FB000224492440249410182800111328506CE49
:108FC00022CC26CA2E8497300000E7802005AA8490
:108FD000979501009385458817750100130545672E
:108FE00097600100E78020B90307840003566400FE
:108FF00083554400A686179501001305E5919760F7
:109000000100E78040B7294597600100E78080BBF9
:1090100097A7FF1F83C7E73B639D97000145970014
:109020000000E78060D281450A8597000000E78054
:10903000C0ECF2406244D244056182806D71232409
:109040008110232611102322911093F745002E84BE
:10905000638707143C083EC0B707E5003EC23C08E2
:109060003EC4231701002318010023190100231A0D
:109070000100231B010097A7FF1F83D7273599E322
:10908000C167FD172316F10097A7FF1F83D7273469
:1090900091EB97D7FF1F938727BC9C439C43DC47EA
:1090A00083D7070017A7FF1F130747322317F100C5
:1090B000544F835747002318F100DC4AA1E79785F6
:1090C00001009385A57D177501001305655897600C
:1090D0000100E78040AA178501001305657E9760AF
:1090E0000100E78040A9294597600100E78080AD35
:1090F000134544008320C1100324811083244110B0
:109100005161828097A7FF1F83C7B72C2555D9C30C
:10911000FD1717A6FF1FA30EF62A03D606018347E5
:109120000701CC460A85230BF10097300000E78049
:1091300060DE97D7FF1F938727B29C4317A7FF1FB7
:109140001307C728978601009386867A88430A8684
:109150006C0097100000E780601FAA8451D99785A2
:1091600001009385A573177501001305654E97607F
:109170000100E78040A0A68517850100130505754D
:1091800097600100E780209F294597600100E780F4
:1091900060A3268597000000E78000BB91BF93F78E
:1091A00025009DC7B7E70400BC4741468145280814
:1091B0008297255597000000E78000B9280893059D
:1091C000F00F97000000E78040D3134524001DB73F
:1091D00093F71500014599DF97000000E78020997B
:1091E0001345140001BF5C4D411106C688C317D753
:1091F000FF1F2323F7A6B7E7040083A70708170577
:1092000000001305E5E38297B24097D7FF1F23873D
:10921000A7A401454101828001113335A000A307B5
:10922000A100B7E7040083A7471706CE1306F10095
:109230008545130550308297F24005618280828017
:10924000411122C406C697D7FF1F83C7A7A20144B6
:1092500089EF97B7FF1F83C737FC054499E717C409
:10926000FF1F0344A43B1344140022859700000011
:10927000E780C0FA178501001305057C09E417850E
:1092800001001305657C2244B240410117630100CF
:109290006700638E797122D4A30F010037E40400C4
:1092A0008327841726D24AD006D6AA842E8913058E
:1092B00050309305F10132C6829732468347F1015F
:1092C00093150601C18185CB01452EC6970000008C
:1092D000E780C0F483274417B2454A8626858297E3
:1092E000054597000000E78060F3B2502254925485
:1092F000025945618280832744174A8626858297D2
:10930000EDB741119397050122C406C626C2C18755
:109310002E8463D40702B7E40400FC5417A5FF1F92
:1093200003450510829719C1BC5482972165218D90
:10933000B240224492444101828093F715008DC7C8
:10934000B7E7040083A7471A17A6FF1F1306460CAA
:1093500097D5FF1F9385459117A5FF1F0345450C22
:10936000829713451400E9B793F7250099CFB7E723
:109370000400BC4F13060064894517A5FF1F034571
:10938000250A82971345240065B793F7850085CF9A
:1093900097D7FF1F83C7C78E85E7B7E7040003A8E9
:1093A000871A1307401F97A7FF1F83C767078146C8
:1093B00013064006994517D5FF1F0355E58B029804
:1093C00013458400B5B793F745000145B5D3B7E41D
:1093D000040083A7041817D5FF1F0355E58982975A
:1093E000BC4C13060064914517A5FF1F03454503B8
:1093F0008297134544002DBF97D7FF1F83D7C78798
:109400006398A70217D7FF1F2319B78617D7FF1F27
:109410002316C78617D7FF1F2313D7862E861785D7
:1094200001001305A567BE85175301006700A374EB
:109430001785010013050568176301006700838B1A
:109440000357450097D7FF1F83D70783631EF70491
:10945000C1674111F91722C417D7FF1F232EF780C8
:1094600037E4040097D7FF1F23AA078097D7FF1F71
:10947000A382078097D7FF1F238407807C4C06C6F2
:10948000894517A5FF1F0345A5F982977C4C914597
:1094900017A5FF1F0345C5F882972244B24041013A
:1094A00017030000670003DA1785010013058560C4
:1094B00017630100670003847D15954763E2A71CCD
:1094C00017870100130707550A053A951C4101113A
:1094D00022CC06CEBA972E84828717850100130509
:1094E000E55D97600100E780E080A1A203C7250049
:1094F00099476311F7022E8597000000E78080F4FA
:1095000083456400178501001305455C97500100F1
:10951000E780606697B7FF1F238007D0178501009B
:109520001305855C7DBF03C7250095476319F702C6
:10953000C16717C7FF1F03572774F91703D5A50085
:109540006309F702B7E7040083A7C7178297178557
:1095500001001305655A97500100E780A0798547FF
:1095600017B7FF1F230AF7CA178501001305455BCC
:109570008DBF97C7FF1F2391A77083D7E50097C6BC
:10958000FF1F239CF66E83D7050197C6FF1F239705
:10959000F66E83D7250197C6FF1F2392F66E97C7F5
:1095A000FF1FA389076C631BE502B7E70400BC4FEC
:1095B000096613060690A14517A5FF1F034545E65A
:1095C00082970356E4008355A40017850100130514
:1095D000E55397500100E780005A51B79307700F89
:1095E0002316F100B7E7040083A7870D17A6FF1F16
:1095F000034606E36C0082974DF9854717C7FF1FA6
:10960000A30AF7665DB71785010013052552D1BD82
:1096100083C5250091476392F50217850100130564
:10962000655297500100E780E06C97000000E780EA
:1096300060C1F24062440561828099476392F502FD
:10964000228597000000E780E0DF834564001785EE
:1096500001001305A54797500100E780C051D1BF15
:109660009547639AF50083471400E1F317850100DD
:109670001305854FBDB5178501001305654FE1BF83
:109680008280411122C417A4FF1F1304A4DAAA8602
:1096900017860100130686392285C14506C69750F4
:1096A0000100E78060660357440097A7FF1F938778
:1096B00067D92393E700035764002394E700B2407F
:1096C000224441018280411106C697000000E780D4
:1096D00080FBB7E7040083A7871417A6FF1F1306B4
:1096E00066D5D54501458297B2404D4697A5FF1FE7
:1096F000938545D5130570304101170300006700BD
:10970000A3B961712324811A37E404008327040874
:109710002326111A2322911A2320211B232E3119CB
:1097200017050000130525BE829717A9FF1F13090F
:1097300029CF994785442300A900231CF100978570
:1097400001009385A53293074006177501001305A4
:1097500025F0231CF1082308910097C9FF1F938966
:1097600049FC97500100E780004183D50900178527
:1097700001001305A52E97500100E780C03F294541
:1097800097500100E780004403D5090089699700DC
:109790000000E78040EF8327441710088545130534
:1097A000503082978327441717A6FF1F130686C9D8
:1097B000CD451305703082978327441717A6FF1FE6
:1097C000130646C6B54513056030829783274417B4
:1097D00030088945130510318297832744173009D3
:1097E0008945130520318297832744159385099075
:1097F0000D458297832744159385099011458297DB
:10980000A3059100230691002308910002CD230CAB
:109810000100832784163009914513057040829713
:10982000832784161306B1008545130500408297EF
:10983000832784167000854513051040829783277F
:1098400084163008854513052040829783278416A7
:1098500010088545130550408297832704157D55D0
:109860008297832744137D5582977D5597A0FFFFEC
:10987000E780A0E08327440C829797A0FFFFE78052
:1098800000BC8327841417A6FF1F1306A6BAD5456C
:109890000145829789471306700F814528092306E1
:1098A000F1009790FFFFE78080858D471306000841
:1098B00081452808230CF1089790FFFFE78020845A
:1098C0009147230CF100977701009387E7C99843EC
:1098D00083C747003AC8230AF10097D0FFFFE7800B
:1098E000E0AB70008545054597A0FFFFE78000E0ED
:1098F00030099305700F094597A0FFFFE78000DF4F
:109900003008930500080D4597A0FFFFE78000DEB3
:1099100010089545114597A0FFFFE78020DDC1673E
:1099200017C7FF1F13074735F9171CC3232207006A
:1099300017A5FF1F130585AE97A0FFFFE780E0D9AD
:109940008327C41D17C5FF1F1305853182973C4827
:1099500003450900854582978320C11A0324811A93
:109960008324411A0329011A8329C1195D61828068
:10997000C16717C8FF1F03582830F9176301F8089B
:109980003DCDB5CD011126CAB7E4040083A78412EA
:1099900022CC2E862315B10006CE2A8401478146AB
:1099A000ED45428582972AC611ED17850100130502
:1099B000E50C97500100E780E033F2406244D24466
:1099C00005618280FC440356A100A28582972C0089
:1099D00017C5FF1F0355452A97A0FFFFE780A0DCAE
:1099E00069DD178501001305A50A97500100E7807E
:1099F000603083A7C412ED45280082977DBF828026
:109A0000411106C61DC9854717A7FF1FA301F7A26D
:109A1000354697A5FF1F9385E5A01305603097A7EE
:109A2000FF1F238707A097000000E780E086B24071
:109A30004101170300006700E38097A7FF1FA38879
:109A4000079EF9B797C7FF1F83C78723A9EFC16791
:109A500017C7FF1F03574722F9176306F704411181
:109A6000854722C417C7FF1F230CF72037E40400E3
:109A70007C4C06C6A14517A5FF1F0345659A829732
:109A80000323841A2244B24097A7FF1F83C7479934
:109A900017C5FF1F0355451E1307401F814631465A
:109AA00099454101028382806D7123248110232610
:109AB000111023229110328401CD8947630AF502E7
:109AC0008320C110032481108324411051618280BE
:109AD000178501001305850AAE8497500100E780C1
:109AE0006021A285268597C0FFFFE780E0A9C9BF56
:109AF000B7E70400FC47280082971785010013058B
:109B0000A50897500100E780E01E8347810039C413
:109B10001307000B6380E7021387A7051377F70F7E
:109B20008D4663EDE602A285280097C0FFFFE7801F
:109B3000201B79B78547E3F587F8834591001775B2
:109B40000100130525E6B335B00097A7FF1F238555
:109B5000B75497500100E78000029DB7034791007A
:109B6000A207D98F35671307D7556385E708636860
:109B7000F7022D671307B7556387E70631671307A9
:109B8000C755638AE70429671307A7556394E7025B
:109B9000A285280097C0FFFFE780E05215B739671C
:109BA0009306E7656381D70863E9F6001307E75575
:109BB0006384E706A28528003DB73D679306F75505
:109BC000638AD7061307F766E396E7FE97C0FFFFA1
:109BD000E780606BF5B50146A285280097C0FFFFBE
:109BE000E780A03BF1BDA285280097C0FFFFE7807A
:109BF000C04BF9B58947E3F587EC97000000E78093
:109C0000A0E49305E4FFC205C1811305A10097906C
:109C1000FFFFE780E05B6DB5A285280097C0FFFFDE
:109C2000E780604B71BDA285280097C0FFFFE780E9
:109C3000205679B597C0FFFFE780A05E51B5C16798
:109C400017C5FF1F03554503F9176307F500B7E76D
:109C5000040003A3C71702838280854717C7FF1F2D
:109C6000230AF700014517F3FFFF6700235B178303
:109C7000FFFFE70223442A8408452E89B28919C9C7
:109C800000C1971500009385A586610597300100F6
:109C9000E780800181447D5A97100000E780E03919
:109CA00063C7A404814497100000E780003A63C8AA
:109CB000A40497C7FF1F9387E7FC9C43DC47B307C7
:109CC000F94091872302F400638309048327C900C4
:109CD000B307F4409587A302F4001C4C89C79C4746
:109CE00099C3228582971783FFFF6700E33F5C4497
:109CF000139714008504BA972390470171BF1C483D
:109D0000139714008504BA972390070069BF83272F
:109D100089000547B307F4409587A302F4008357F1
:109D20000400638EE7028DC309476384E7040D478F
:109D3000E395E7FA978701009387C7371CCC97878D
:109D400001009387273811A897870100938707FEA2
:109D50001CCC97870100938767FE5CC8BDBF9787BF
:109D600001009387A7E91CCC97870100938707EA36
:109D7000EDB7978701009387A7381CCC9787010020
:109D800093870739D9BF95E51783FFFFE70223348F
:109D9000004618448347940075839D8B6317F70032
:109DA00097100000E78060B448C41783FFFF670086
:109DB000433482801783FFFFE702C32F13893500E6
:109DC000C16442094111AA890144F11413590901DE
:109DD000054A2EC697100000E7802026B24563484A
:109DE000A400014541011783FFFF6700E32F83A70C
:109DF000090013171400BA9783D707006388B700C8
:109E00006394970063742A010504E1B70545D9BF3F
:109E10001783FFFFE7022329AA892E89328BB68494
:109E20003A8ABE8A97A00000E78020FB71C9268588
:109E300097200000E78020098D4763E7A7007D5544
:109E40001783FFFF6700A32983DB440097100000FE
:109E5000E780A0242A8497100000E780402593071C
:109E6000740031443305850263CDA70297100000CA
:109E7000E780A02297100000E78020222A84971014
:109E80000000E780C0229307740031443305850247
:109E900063C3A70497100000E780202093074500C4
:109EA00029A897100000E78080203305850213075A
:109EB000F0179307C017E35FA7FA2D55E3C277F9B0
:109EC00063040B02D6865286A6854A859720010038
:109ED000E78020BAB5B797100000E780401D330532
:109EE00085029307C5FFD1BF832749001385C900A9
:109EF00083D5270097000000E78000EC61F581B76B
:109F000069553DBF97C7FF1F2390A7D897C7FF1F6D
:109F1000938747D7904381470C463307F5004207A4
:109F200041836393B70082805446139847008507A6
:109F3000C2962390E600D5B797C7FF1F938787D4B3
:109F40009C4303C58700828017C5FF1F0355C5D3F7
:109F500082801783FFFFE7028317C1671387D7FF4C
:109F6000630BE502636AA700F1176300F502014580
:109F70001783FFFF6700E3171387E7FF6302E5021C
:109F8000FD171D8D13351500E5B797500000E780CC
:109F9000C0267D15C5BF97500000E78040FBD5BFA8
:109FA00097500000E78060F9EDB71783FFFFE702E5
:109FB00003124111AA8401442EC697100000E780C5
:109FC000C008B2456348A400014541011783FFFF63
:109FD000670023129C48131514003E958357050013
:109FE000E385B7FE0504C9BF03485500814693F7D2
:109FF000F60F63E5070181473E85828058459397B8
:10A000005600BA9703D727006316B70003D7070097
:10A01000E304C7FE8506E1BF834645000147937709
:10A02000F70F63E4D700814711A81C4513165700AA
:10A030000507B29703D60700E313B6FE3E8582807C
:10A040001783FFFFE702030793170501C18797CA2C
:10A05000FF1F938A2AC3635BF00883A70A00C047E7
:10A060009C4703570400198D420541816368F50040
:10A07000014422851783FFFF6700030712052A9416
:10A08000CDBFDC4713944900014A3E948347440006
:10A090006341FA02014A834754006349FA02850981
:10A0A000C20993D9090183A70A009847E3EBE9FCA9
:10A0B000C1B71C4413195A00A6853E994A859700DA
:10A0C0000000E780C0EE05E1050AC9B75C4413193A
:10A0D0005A00A6853E994A8597000000E78020ED4A
:10A0E00019E1050A4DBFE30C09FA61B7AA84814959
:10A0F0005DBF1783FFFFE70283FD1C452A8481E7CC
:10A100009307C5001CC51C44231204001CC0930700
:10A11000F00F63EDB70093F5F50F2285972000004F
:10A12000E78020E21783FFFF6700A3FC93940501FB
:10A13000C167C18063F9F500A685228597200000DC
:10A14000E78040E5C5B7C18193F5F50F22859720DB
:10A150000000E78000DFA685228597200000E780C9
:10A1600040E0C9B797C7FF1F9387C7B18843828074
:10A170001C4599C797C7FF1F23A6A7B0014582803A
:10A180007D55828097C7FF1F9387C7AF984383474A
:10A190004500484792073E9582801783FFFFE702FC
:10A1A00003F3617100451C183EC6B70780013EC825
:10A1B0001C183ECA8357440002CE02D002CC231E94
:10A1C000F100834784002A8902D22301F1023C086E
:10A1D0003ED402D697000000E78000FB83570500BD
:10A1E0002316F10297500000E78060C42307A10204
:10A1F0005C4003556400F18313F717008347F102B5
:10A2000052055181F99BD98FA307F10297100100E4
:10A21000E780807539CDAA840355050097A000001A
:10A22000E78080BC83D704002AD26800231CF10099
:10A2300083D72400231DF1001C4803D647008C431C
:10A2400097200000E78000CD8347B400CA861786B8
:10A250000100130626948117A305F4006C00481032
:10A2600097200100E780E0805D611783FFFF6700B2
:10A2700043E82155D5BF1C45B1CF03C5A70089468A
:10A2800013576500630BD7028D46630ED7028546D0
:10A290006300D702130740063305E50203C7B70082
:10A2A000418B15CB83C7B700BD8B3355F5408280FA
:10A2B0001375F5031307803EC5B709671375F503DA
:10A2C00013070771D1BF372709001375F50313076B
:10A2D000077CD9B7014582801783FFFFE70223DFA0
:10A2E00003A98500630C09048347B900AE8493F782
:10A2F000070E85C303459900930520030D810505CD
:10A30000B305B5028844610597300100E780E0A9F4
:10A3100035A02E8597000000E78020F62A8419CD0D
:10A3200097000000E780605C8325C900B307B54053
:10A3300063FA87002E94B305A440E9F51783FFFF65
:10A34000670023DB85457DBF1783FFFFE70223D826
:10A350002A8403D50500011132C636C43AC22EC084
:10A3600002CA02CC02CE97A00000E780E0A7824597
:10A370002ACA22852ECC97000000E780E0E0035730
:10A380000500231EE10097500000E78040AAA24686
:10A3900032469247230FA10036874C08B2862285A9
:10A3A000014697000000E780E0A605611783FFFFE4
:10A3B000670023D41783FFFFE70263D161711C1884
:10A3C0003EC6B70780013EC81C183ECA3C0800457F
:10A3D0003ED4AA8402CC02CE02D002D202D697008A
:10A3E0000000E78060DA8357050035592316F10233
:10A3F00097500000E780A0A32307A10209C4835758
:10A40000440081EB21594A855D611783FFFF670096
:10A4100043CE035564005205518197100100E78037
:10A42000A0542A8965D18347B40093F7070E99C7D2
:10A430001305840197300100E78060998357440039
:10A44000231EF100834784002301F1025C40035581
:10A450000900D98313F7070883471102231CA100C1
:10A4600093F7F707D98FA300F10283572900231D23
:10A47000F1005C40F18313F717008347F102F99B69
:10A48000D98FA307F10297A00000E780E0952AD2B8
:10A4900035D9834794006800139757008347B40069
:10A4A000FD8BD98FA305F4001C4803D647008C43CD
:10A4B00097200000E78000A6A68717770100130702
:10A4C000676D740005464C10268597000000E780F4
:10A4D00060942A890DD98347B400A685FD8BA30516
:10A4E000F40097000000E78060DF31BF1783FFFFB3
:10A4F000E702E3BD832485FE2A8441112685970067
:10A500000000E78080D7834734FF93F7070E8DCB99
:10A510002AC6268597000000E78060C809CD8347DA
:10A5200034FFB245FD8BA309F4FE91C52285973017
:10A530000100E780808741011783FFFF670063BB4D
:10A540007DD98327C4FF2685829775F5834734FF1D
:10A5500093F7070E91C7228597300100E780208787
:10A56000032584FE97000000E78000E5E9B7178324
:10A57000FFFFE702C3B29C4141112A8903C70700CC
:10A5800089472E84935667006380F6040D466388DE
:10A59000C6049307F0076304F7022E859720000096
:10A5A000E780C0A7AA848149C16B130C490097B703
:10A5B000FF1F9387276D9C43984763E4E90441019B
:10A5C0001783FFFF670063B103D745008547E3F8B2
:10A5D000E7FE2E8597200000E780A0A9E1B703D70A
:10A5E0004500E3FEE7FC2E8597200000E78000A3EE
:10A5F000AA84228597200000E78060A4C204C98C49
:10A600005DB7DC470355A900139A49003E9A93179A
:10A610000501C187635DF00083570A006397A702B5
:10A6200063E774038327CA00034D5A002DA0A16776
:10A630002167A98F1307F7EFE374F7FE639709000B
:10A6400097000000E780209161FD85098DB7832781
:10A650008A00034D4A00835DA90003576900216AFF
:10A66000138BC7003AC6814A33CA4D01631E5D0190
:10A6700097B7FF1F938787619C43E1DBA2866286C1
:10A68000814526858297D1B7A1679387F7EF930C11
:10A690004BFF63F24703B2455A8597F0FFFFE7800F
:10A6A000A0710DC103278B00104709CE10436382B0
:10A6B000C4023107D5BFEE85668597000000E780AC
:10A6C000008F71F993861A0093FAF60F130B0B02A1
:10A6D00071BF835644005C43E3E9F6F622853AC62F
:10A6E00097100000E780807DA1679387D7042A8AAE
:10A6F000035D4400324763E897008347D90093E73E
:10A7000007F8A306F9001C4766852286E285829732
:10A71000C1670844FD17337AFA00529508C0231226
:10A72000A40125B797B7FF1F9387C7559843814763
:10A7300015C31447814763FFD500939745004C47E5
:10A74000BE9519C903C7550081476375E600DC450E
:10A750001606B2973E85828003C745008147E37B9A
:10A76000E6FE16069C45F5B71783FFFFE7028394C4
:10A77000AA892E8A814497BAFF1F938AAA5083A779
:10A780000A00984763E6E4001783FFFF6700C3955C
:10A79000DC471394440001493E9413BB14008347E3
:10A7A0004400634BF900014913BB14008347540074
:10A7B000634FF9008504E1B70844931759005287A5
:10A7C000DA860146A2853E9582990509C9BF4844AB
:10A7D000931759005287DA860546A2853E958299DD
:10A7E0000509E9B71783FFFFE702638E814517F577
:10A7F000FFFF1305054897B7FF1F239707489700EA
:10A800000000E780A0F61783FFFF6700838E97B7ED
:10A81000FF1F938727479C4395C31783FFFFE702DA
:10A82000038B814517F5FFFF1305A5449700000032
:10A83000E780C0F31783FFFF6700A38B8280178335
:10A84000FFFFE702238737E40400832784124111C6
:10A850002315E100AE893289368A3A86814601475E
:10A86000ED45AA8482972AC621C90356A100D28544
:10A8700097400100E780C0248327C413CE85268536
:10A880008297058905C98327440D231421010146B8
:10A890002C00268582972A8401C9B7E7040083A784
:10A8A000C712ED4528008297228541011783FFFFDB
:10A8B000670083834944D5B76554FDB75C41FD17F4
:10A8C0005CC182801783FFFFE7026380B7E7040063
:10A8D000FC5F829795473305F50281450D8117830B
:10A8E000FFFF670003811773FFFFE702437EB7E7AF
:10A8F0000400FC5F829795473305F5020D811773BD
:10A90000FFFF6700037F1773FFFFE702437CB7E792
:10A91000040083A7870B0355050082971773FFFF79
:10A920006700237D1773FFFFE702637A0355050075
:10A930003287AE861796FF1F0356E6B697B5FF1F00
:10A940009385053597000000E780A0EF1773FFFFA0
:10A950006700237A1773FFFFE7026377B7E7040006
:10A9600083A7C71782971773FFFF67008378177352
:10A97000FFFFE702C375B7E7040083A7871397B506
:10A98000FF1F9385E530829701451773FFFF67002E
:10A9900043761773FFFFE7028373B7E7040083A7CB
:10A9A000C71F81451795FF1F0355E5AB82971773A6
:10A9B000FFFF670003741773FFFFE7024371B7E7F8
:10A9C000040083A7871397B5FF1F9385652D829792
:10A9D00001451773FFFF6700C3711773FFFFE7029D
:10A9E000036FB7E7040083A7C71F81451795FF1FB3
:10A9F000035565AD82971773FFFF6700836F177369
:10AA0000FFFFE702C36C2E8597800000E780E0AF70
:10AA100097800000E780E0EC1773FFFF6700636D2D
:10AA20001773FFFFE702A36A97800000E780E0F654
:10AA30001773FFFF6700E36B5C49E1175CC95CC5F6
:10AA400083572501A1072319F50083570501A107A5
:10AA50002318F5008280F1473305F50297B7FF1FF1
:10AA6000938707269C433E9582808D476315F608A1
:10AA700003D74600854763F0E7081773FFFFE70237
:10AA80000365368536842E8997100000E7800059CB
:10AA900029C98357440093140501C18063E39704D7
:10AAA000228597100000E7806057FD142312940060
:10AAB0009307A0026300F5029307B0026307F50253
:10AAC00093079002631FF500228597000100E7803D
:10AAD000C08501A80146CA85228597A00000E780AD
:10AAE00060B01773FFFF6700C360228597100000F6
:10AAF000E780C003FDB7828097B6FF1F9386861C50
:10AB00009C42014599CF9843D44217B6FF1F232B8F
:10AB1000E61A6396D70097B6FF1F23A7E61A138598
:10AB2000C7FE82801773FFFFE702635A9700000099
:10AB3000E780A04B71443305850291459790000052
:10AB4000E78020E911E565551773FFFF6700635A39
:10AB500097B7FF1F23A4A71697000000E780E048DF
:10AB600033058502914597900000E78080E661DD1E
:10AB700097B7FF1F23A6A71497000000E780E046C1
:10AB800097B7FF1F2396A71297000000E780E045C4
:10AB900097B7FF1F239FA710977701009387C704DC
:10ABA00017B7FF1F232AF71097070000938707E9BD
:10ABB00017B7FF1F2320F710014579B71773FFFF61
:10ABC000E702E350AA8517B5FF1F1305650E97101E
:10ABD0000000E780C05B1773FFFF670083511773A6
:10ABE000FFFFE702C34E97000000E78060FD97106B
:10ABF0000000E780405B97B7FF1F9387A70C9C433B
:10AC000091CF1387C7FE19CB83D5C7FF17B5FF1F99
:10AC10001305C50B97200100E78020191773FFFF6C
:10AC20006700234D1773FFFFE702634A9700000098
:10AC3000E780C0EC09CD834785002A8493F7070499
:10AC400099EB0355E50097000000E78080F9177342
:10AC5000FFFF6700034A8347C5009304450117B906
:10AC6000FF1F1309290685E3832709005CC997B7ED
:10AC7000FF1F23A9970483274900F1FB97B7FF1F04
:10AC800023A49704E9B7FD172306F5006105978013
:10AC90000000E780C0D68307840063CB07048347A6
:10ACA000840093E707F82304F400B7E704009C5FEF
:10ACB00082974205A94741813375F5028347840095
:10ACC00093F707FCC98F2304F4008347D4003E9513
:10ACD0001C402318A40089CF984319CB8347C40094
:10ACE0005040814585073305F502420541810297B1
:10ACF000832709005CC897B7FF1F23A597FC83270C
:10AD0000490089E797B7FF1F23A097FC8347C4003A
:10AD10009DDF8355040117B5FF1F130525FB972001
:10AD20000100E780800825B71773FFFFE702233A89
:10AD300097B7FF1F9387C71E9C4701448583858B68
:10AD400085E3AE84B2853A8697100000E780804B99
:10AD50002A8419C597100000E780C041829408CC6E
:10AD600022851773FFFF6700C3381773FFFFE702E1
:10AD7000633441112E8932C6AA8997000000E7800A
:10AD8000C031324713060502CA8697050000938535
:10AD9000C5CC17B5FF1F1305A5F197000000E7808C
:10ADA000E0F82A8425C99304C50097000000E780D5
:10ADB000E0411946AA85268597100000E780801596
:10ADC0008545268597100000E78060111775010002
:10ADD000130545DF4E958345050026859710000035
:10ADE000E78020165C4831468145A1075CC85CC4F9
:10ADF00083572401E1172319F40083570401E11755
:10AE00002318F4001C4C3E859770FFFFE780202F2D
:10AE1000A3042501228541011773FFFF6700C32C9E
:10AE20001773FFFFE702A32A4111AA842EC632C47A
:10AE300097100000E7806036004DB24522468347F8
:10AE400084000CC050C093F7F70393E70704230472
:10AE5000F40023180400268597100000E780803155
:10AE600083479400A9462317A40013D7370005078A
:10AE70003307D7029D8B85072306F400A306E40061
:10AE800083C70401D8488507230FF7FE17B7FF1FB4
:10AE9000130747E35843232A04009307440129E397
:10AEA00017B7FF1F2322F7E217B7FF1F232CF7E086
:10AEB00017B4FF1F130484E1228597200100E78067
:10AEC00000E11C44858B5D8D19E581452285972025
:10AED0000100E78080ED41011773FFFF67006321E8
:10AEE0001CC317B7FF1F2321F7DED9B71773FFFF66
:10AEF000E702E31D97050000938565B701459700BC
:10AF00000000E78000B001451773FFFF6700631E74
:10AF10001773FFFFE702A31B97000000E78080B0D4
:10AF20001773FFFF6700E31C8347C500A5E3177392
:10AF3000FFFFE702C3192A840355E50097000000CC
:10AF4000E78000C821C18347840093F7F7FB2304FF
:10AF5000F4001C4091C7DC4381C74C4001458297F7
:10AF600097000000E78080B917B5FF1F130505D6CD
:10AF700097200100E780A0E50355E400970000005A
:10AF8000E78020C61773FFFF6700A3168280177340
:10AF9000FFFFE702C31397B7FF1F9387A7D2970559
:10AFA0000000938565C817B5FF1F130525D223A0A0
:10AFB000070023A2070097200100E780E0CE177367
:10AFC000FFFF670003131C4D91CFDC4381CF177344
:10AFD000FFFFE702C30F8345070082971773FFFF48
:10AFE00067002311828097B7FF1F938767D09C4328
:10AFF00003C50700828097B7FF1F938767CF9C43E5
:10B0000003C51700828097B7FF1F938767CE9C43C5
:10B0100003C52700828097B7FF1F938767CD9C43A6
:10B0200003C54700828097B7FF1F938767CC9C4377
:10B0300003C53700828097B7FF1F938767CB9C4378
:10B0400003C55700828097B7FF1F938767CA9C4349
:10B0500003C56700828097B7FF1F938767C99C432A
:10B0600003C57700828097B7FF1F938767C89C430B
:10B0700003C58700828097B7FF1F938767C79C43EC
:10B0800003C59700828097B7FF1F938767C69C43CD
:10B0900003C5A700828097B7FF1F938767C59C43AE
:10B0A00003C5B70011E11D45828097B7FF1F938745
:10B0B00027C49C4303C5C700828097B7FF1F9387AF
:10B0C00027C39C4303C5D700828097B7FF1F938790
:10B0D00027C29C4303C5E700828097B7FF1F938771
:10B0E00027C19C4303D50701828097B7FF1F938731
:10B0F00027C09C4303C52701828097B7FF1F938712
:10B1000027BF9C4303D54701828097B7FF1F9387D2
:10B1100027BE9C4303D56701828097B7FF1F9387A3
:10B1200027BD9C4303D58701828097B7FF1F938774
:10B1300027BC9C4303C5A701828097B7FF1F938755
:10B1400027BB9C4303C5B701828097B7FF1F938736
:10B1500027BA9C4303C5C701828097B7FF1F938717
:10B1600027B99C4303C5D701828097B7FF1F9387F8
:10B1700027B89C438857828097B7FF1F938747B7AC
:10B180009C4303D5C702828097B7FF1F938747B6BA
:10B190009C4303D5E70219E11305800C828097B721
:10B1A000FF1F9387E7B49C4303C50703828097B7CB
:10B1B000FF1F9387E7B39C43C85B828097B7FF1F4D
:10B1C000938787B28843828097B7FF1F938707B220
:10B1D0008843828019E17D558280F5DE984265DFE3
:10B1E000FDD917B7FF1F1307A7D31847AA877155B3
:10B1F000058B631D072403C507001547E37DA7FCE6
:10B2000003C737001305F0057D171377F70FE364C5
:10B21000E5FC03C35700E30003FC83C86700E38C2D
:10B2200008FA03C77700494579171377F70FE364E6
:10B23000E5FA03C7A70011481305F7FF1375F50FCB
:10B24000E36BA8F803CE97000D481305FEFF1375B6
:10B25000F50FE362A8F803C8B70063090800651892
:10B260001378F80F1305600DE36705F703C5C700F2
:10B27000794879151375F50FE36FA8F403C8D70063
:10B280000D457D181378F80FE36705F503D807011E
:10B29000930E40175118420813580801E3ED0EF3BE
:10B2A00003C8E7007D181378F80FE36605F303C8B9
:10B2B00027017D181378F80FE36F05F103C88700A5
:10B2C000C54E75181378F80FE3E70EF103D8670140
:10B2D000856E938EBEE06D18420813580801E3ECAA
:10B2E0000EEF03D847016D18420813580801E3E434
:10B2F0000EEF03D887017918420813580801E36C50
:10B3000005ED03C8A7017D181378F80FE36505ED77
:10B3100003C5B7011D487D151375F50FE36DA8EA48
:10B3200003C5D701714879151375F50FE365A8EAD0
:10B3300003D5E7011308E00F7D1542054181E36C59
:10B34000A8E803C50702494879151375F50FE364AA
:10B35000A8E8C85301C937C834005915130858BFA5
:10B36000E36BA8E603A8870237C53400130555BF71
:10B370005918E36205E717B5FF1F2329C59603C6D1
:10B38000050117B5FF1F2325F5960545E375C5E4AF
:10B3900003D82501D04933760603E31E06E203C62F
:10B3A0001501E30A06E217B6FF1F232FB69283C5E5
:10B3B000270001466387A50003C61700F145330641
:10B3C000B60283C707039305C00272971A071307D3
:10B3D000C70516031A9796084697B387B7024155D3
:10B3E0003E973297420741836362E8061773FFFF77
:10B3F000E702E3CD368597800000E780A0689700DC
:10B400000100E78020482A8497A00000E780805A46
:10B410002A9497F00000E78060262A949790000015
:10B42000E780A0812A9497F0FFFFE780E06F2A94DD
:10B4300097400000E78060932A9497700000E780AF
:10B44000A09C22951773FFFF6700A3CA8280177321
:10B45000FFFFE702C3C74111A307A10097A00000A7
:10B46000E780A0C59305F100170500001305E5B5B9
:10B4700097F0FFFFE780802F014541011773FFFF21
:10B48000670023C71773FFFFE702E3C117B4FF1F6D
:10B49000130404A90328840079599368180097B409
:10B4A000FF1F23A314A91378180063100802BA849D
:10B4B000BE89368B328A2E89AA8A97F0FFFFE780F1
:10B4C000E0A77D15269519E531594A851773FFFFC9
:10B4D0006700E3C097F0FFFFE78040A67D15269543
:10B4E000A167E353F5FE97B7FF1F938727DA9843C9
:10B4F0003E8C814B01CB014597F00000E780204452
:10B50000933B15004A85DA865686D28597900000CF
:10B51000E780C04D2A8911CD1C44F99B17B7FF1F46
:10B520002324F7A083270C00CDD3E3800BFA829766
:10B5300069BF268597B7FF1F23A6079E97F0FFFFD9
:10B54000E780809C4146CE8517B5FF1F1305C5A631
:10B5500097300100E780C05697D00000E7804099FF
:10B560000325040B97D00000E780009D054597D088
:10B570000000E78000A4054597000000E78060ED2B
:10B58000A9B797B7FF1F9387A7999C47858BEDC7EE
:10B590001773FFFFE702A3B317B5FF1F130505A03D
:10B5A00097B7FF1F23AE079697B7FF1F23AC0796E9
:10B5B00097B7FF1F23AA079697200100E7802081F5
:10B5C00097500000E780E0F597100100E780A04C5D
:10B5D00097100100E780A05297B7FF1F9387C7928B
:10B5E0009C4391C7054597800000E780402097A7BE
:10B5F000FF1F9387277B9C4399C741657D159770F3
:10B600000000E78040A297F00000E780E03D97D07F
:10B610000000E780808F97B7FF1F938727A59C4383
:10B62000139717016356070097F00000E78000ADFD
:10B6300097B7FF1F23A2079897B7FF1F23A007986C
:10B6400097B7FF1F23AE079697B7FF1F23AC079648
:10B6500097000000E780008C97000000E7800072F0
:10B6600097F0FFFFE780401897F00000E78040D692
:10B670001773FFFF6700E3A7828097B7FF1F9387C9
:10B68000278A884382801773FFFFE70243A49780CD
:10B690000000E780607597800000E780C07717732F
:10B6A000FFFF670003A51773FFFFE702A3A02A842B
:10B6B0009304140201112E85B289A685214636C64F
:10B6C0003A8997300100E780403D0DE9B2463808DD
:10B6D0002686CE851305940497500000E7806041CC
:10B6E00021462C084A8597300100E780003B13353E
:10B6F000150005611773FFFF6700039F0145D5BF64
:10B700001773FFFFE702A39C9305450617A5FF1FCC
:10B710001305455E97100100E78020691773FFFF4E
:10B720006700239D1773FFFFE702639A41112EC63E
:10B7300097F0FFFFE780601BB24588C14101177396
:10B74000FFFF6700039B1773FFFFE702A396AA841E
:10B750002E8497800000E780006CAA8985452285A9
:10B7600097000000E780E07D83C7E4011389940817
:10B7700099E313890403CE85228597000000E780B2
:10B78000407C214693051902228597000000E7803E
:10B79000607897A7FF1F9387A7788C43228597101F
:10B7A0000000E780C08221469385840222859700AD
:10B7B0000000E78020761773FFFF6700E39217739E
:10B7C000FFFFE702438E397197F00000E780E0B495
:10B7D0009305400661E997800000E78000606302FE
:10B7E000051497A7FF1F83C7A75213B7170097A683
:10B7F000FF1F238FE650014499CFC16417A9FF1F93
:10B80000130909729309400EFD1497000000E780A8
:10B81000C0866342A40A97F0FFFFE780000D4169EC
:10B82000B7290900096AFD7A2A8B81447D19938919
:10B83000F97B130A0A71938A8AC797000000E78090
:10B84000C08363D7A4041304400EB387840217A7F0
:10B85000FF1F1307E76C0324070B3E948357C401B3
:10B860006382270B18403307EB4063EAE900834704
:10B8700044008507B3874703D6976365F7080146F9
:10B880008145094597F0FFFFE780604EAA8B29E5C7
:10B8900097400000E780808385476317F506896538
:10B8A0009385057117A5FF1F1305C5449710010067
:10B8B000E780A04F95A0B30734030327090BBA977D
:10B8C00003D7C7016308970003C75700A382070087
:10B8D0002382E700050415BF9305C5002285970064
:10B8E0000000E78080E65E852286976501009385EB
:10B8F000A52E97F0FFFFE780E0525E8597100000CD
:10B90000E780608A850415BF97A7FF1F938747616B
:10B910009C478D83858BC1F721611763FFFF67000B
:10B92000037C01468545094502D002D202D402D6E5
:10B9300097F0FFFFE780A043AA8479DD97F000002D
:10B94000E780E09C1389C4002A8481454A859700DA
:10B950000000E780005F0C4041464A8597000000E8
:10B96000E780405B832944006385090C4E8502D83B
:10B9700002DA02DC02DE97300100E78060402ACE66
:10B98000141005462C0808184ECC97500000E7808C
:10B99000E00A1375F50F51ED8355840093E52500FA
:10B9A0004A8597000000E780E05E11460C104A854A
:10B9B00097000000E78000560146976501009385D7
:10B9C0002522268597F0FFFFE780C0452685970052
:10B9D0000000E780407D5C40A1D3014685450D45D0
:10B9E00097F0FFFFE780A038AA841DD5484013894F
:10B9F000C40097300100E780A0382AC64A85970026
:10BA00000000E780404C3246636FC5004C404A85D9
:10BA100097000000E780005001468145268597F099
:10BA2000FFFFE7802040268597000000E780A07791
:10BA3000E5B583558400ADB71763FFFFE7022369BF
:10BA400097A7FF1F9387C74D9C471DC193E78700AA
:10BA500017A5FF1F1305052A17A7FF1F2326F74C5D
:10BA600097100100E78040321763FFFF67006368AB
:10BA7000DD9B17A7FF1F2329F74A97300000E780B7
:10BA8000E0647DF117A5FF1F1305C526971001007F
:10BA9000E780E033D1BF1763FFFFE702C36041696E
:10BAA000AA892E8AB28A368BBA8B814417ACFF1FC3
:10BAB000130C0C47930C400E7D1997F0FFFFE780A5
:10BAC000C05B63C4A40001443DA033849403832776
:10BAD0000C0B3E948357C401638627055A87D6868C
:10BAE0005286CE851305040397000000E780E0BB73
:10BAF00001C923800B0022851763FFFF6700235EC7
:10BB00008347F40185C35A87D6865286CE851305AE
:10BB1000940897000000E78040B909C58547238055
:10BB2000FB00D1BF850451BF835745006380071ECA
:10BB30001763FFFFE702035801112A8497000000F2
:10BB4000E780C04D09C985476309F506056117639C
:10BB5000FFFF6700635997E00000E780007C7DF5F8
:10BB6000835744004947ED9BE392E7FEC145228598
:10BB700097000000E7804033AA84228597000000E8
:10BB8000E780204F0357440002CE91472A89631A69
:10BB9000F700228597000000E780A0513C082ACCDE
:10BBA0003ECE97E00000E78080765C55C5D37408F0
:10BBB0004A86A6850545829751BF03574400D14761
:10BBC000E3F6E7F8032A0400C169014997AAFF1FB9
:10BBD000938A0A35130B400EFD1997F0FFFFE7809B
:10BBE000C049634FA90E2285032A04009700000074
:10BBF000E780C042A1452A89228597000000E7809E
:10BC0000A02AAA84228597000000E780804A144079
:10BC10002A86AA8978082685CA8597000000E780C9
:10BC2000C0E7AA8405D503C7F40189476315F70067
:10BC30008347C10181DF5546D28513856400973063
:10BC40000100E780E0E7014597800000E780C01928
:10BC500001C583D7C401A5E797A7FF1F9387472C8A
:10BC60009C4793551900858913D73700058B01CF61
:10BC70008983858B6399B70001452EC69700000024
:10BC8000E780C0DBB2454E8597800000E780601FEB
:10BC90000346C1012A8493751900268597900000F8
:10BCA000E780E03935C1268597800000E780E018FD
:10BCB000268511C0014597800000E780004C973031
:10BCC0000000E780A0408547E312F5E883C75400F1
:10BCD0001307F00FE38CE7E68507A382F400BDB5F8
:10BCE000B304690383A70A0BBE9483D7C401638B93
:10BCF00037015546D2851385640097300100E780EF
:10BD0000C0D955DD0509D1BD5DD86DB782801763F7
:10BD1000FFFFE702233A97800000E780000C05C18F
:10BD2000C164014417A9FF1F1309891F9309400E1D
:10BD3000FD1497F0FFFFE7804034634EA40017A581
:10BD4000FF1F130525FB97100100E780E003176331
:10BD5000FFFF67006339330534038327090B3E95E2
:10BD60008357C50163889700231205009780000060
:10BD7000E780A00C050475BF97A7FF1F9387471A9C
:10BD80009C478D83858B8DE31763FFFFE702233488
:10BD900017A5FF1F130505F697100100E780200384
:10BDA0001763FFFF6700E33482801763FFFFE7023A
:10BDB0000332970500009385C5A017A5FF1F130543
:10BDC00065F397100100E78020EE1763FFFF67001F
:10BDD00043321763FFFFE702832F8841B7E7040070
:10BDE000BC5B050542054181829709C58547230053
:10BDF000F50005051763FFFF6700A32F83C7F5FF55
:10BE00002E858507A38FF5FE828083C7F5FFFD177A
:10BE100093F7F70FA38FF5FE99EF1763FFFFE70284
:10BE2000032BB7E70400BC571385F5FF8297176310
:10BE3000FFFF6700032C82801C41035745008D8F54
:10BE4000BA951CC12312B5003E85828093D7850028
:10BE5000A2051441DD8D835745001387E6FF18C105
:10BE600089072312F50013D685004111238FB6FEF2
:10BE7000A38FC6FE4101828018419307F7FF1CC1C2
:10BE80008357450085072312F500A30FB7FE828074
:10BE9000835745008D8F2312F5001C41BE950CC1C0
:10BEA0002E858280AA8703D7470008410D8FAA9567
:10BEB0002392E7008CC38280184108453305A740D0
:10BEC000828083574500035765001D8F1C4108453C
:10BED0003385A7403305A74082801763FFFFE70241
:10BEE000031F41112EC62A8497000000E780A0FDA1
:10BEF000B2456373B50001A0835744000840BE9566
:10BF00002312B4003E9541011763FFFF6700631ED3
:10BF10001763FFFFE702A31B41112E84B28532C6CF
:10BF200097000000E780A0FB3246A2859730010011
:10BF3000E78000B941011763FFFF6700831B1763A8
:10BF4000FFFFE702C3182E84854597000000E780B5
:10BF500000F9230085001763FFFF6700831917634B
:10BF6000FFFFE702C31641112317B100894597006F
:10BF70000000E780C0F68347E1002300F500834717
:10BF8000F100A300F50041011763FFFF670063168E
:10BF90001763FFFFE702A31393D78500A2054111A2
:10BFA000DD8D2317B100894597000000E78020F35D
:10BFB0008347E1002300F5008347F100A300F5006B
:10BFC00041011763FFFF6700C3121763FFFFE7021A
:10BFD00003101397850193D78501C166938606F0F8
:10BFE000D98F13D78500758FD98FA2053707FF002A
:10BFF000F98D4111DD8D2EC6914597000000E78037
:10C0000000EE6C00114697300100E78060AB410103
:10C010001763FFFF6700E30D1763FFFFE702230BC2
:10C020001C41854503C4070097000000E78080E6B7
:10C0300022851763FFFF6700C30B1763FFFFE7024B
:10C0400003091C414111894503C7070083C7170035
:10C050002307E100A307F10097000000E78080E3D9
:10C060000355E10041011763FFFF67008308176371
:10C07000FFFFE702C3051C414111894503C70700C3
:10C0800083C717002307E100A307F1009700000012
:10C09000E78040E08357E100410113D58700A20704
:10C0A0005D8D420541811763FFFF670083041763BD
:10C0B000FFFFE702C3010C4141112A8411466800C9
:10C0C00097300100E780C09F9145228597000000CE
:10C0D000E78040DCB247C166938606F0139787017C
:10C0E00013D58701598D13D78700758F598DA207F6
:10C0F0003707FF00F98F5D8D41011763FFFF670070
:10C1000043FF1C45BE950CC18280AE87944391E6E7
:10C11000584101EF0CC15CC1828003C7570013670F
:10C120001700A382E700B687D5B70CC3EDB7AA877F
:10C13000084119CD1841D44398C36313D500D8C31F
:10C140002A87034657009376160081E623200700CE
:10C150008280944381CA8C4203A847008CC36393B6
:10C160000601CCC3799A14C3A302C7003687D1BF96
:10C170001C45DC471D8DB777DBB6938777DB0985D8
:10C180003305F502420541818280F147B385F5020E
:10C1900048452E9582808347450085072302F50098
:10C1A00082801763FFFFE70283F22A8409E41763A2
:10C1B000FFFF670003F483474400F5DBFD1793F7A7
:10C1C000F70F2302F400E5F71C4403D72700050707
:10C1D0002391E700DC4399C3228582974C4889CD9F
:10C1E00083475400898B99E71C4422859C479C43D4
:10C1F0009C478297232A04000040232004007DB737
:10C200001763FFFFE702A3EC8357250041112EC6F9
:10C2100081EB0144228541011763FFFF670063ED55
:10C22000035705008147F146E305F7FEB385D702C2
:10C23000404585072E948345440008C4F5F5B24770
:10C24000AA8481E7232A040009A81C456C002285E2
:10C250009C439C43829748C84DDD85472312F400D8
:10C26000B24723200400231804002319F4005C487B
:10C270005CC483D72400FD172391F40061BF1763CA
:10C28000FFFFE702C3E497A7FF1F9387A7A8884390
:10C290002326050023240500410597100100E780AF
:10C2A00000B31763FFFF6700C3E41763FFFFE702F4
:10C2B00003E217A4FF1F1304E4A51C40411199CF0A
:10C2C0009C472300B5002AC65CC197000000E780A8
:10C2D00040FB1C40DC4399C3324582974101176300
:10C2E000FFFF670003E10347450029E3584DAA8794
:10C2F0007D551DCF1763FFFFE70263DD1CC3DC47DD
:10C3000097A6FF1F23A8E6A0F15613050701239067
:10C31000D700970500009385050297100100E7807C
:10C32000A09801451763FFFF6700A3DC7D5582805D
:10C3300082801763FFFFE70283D9011161468145BF
:10C3400028009760FFFFE78080DB97A7FF1F938798
:10C35000679C9C4328009305F00FDC473EC697007E
:10C360000000E780C0F405611763FFFF670063D832
:10C3700097A7FF1F9387079A9C43D847A167938786
:10C38000C702631EF70A397106DE22DC26DA800056
:10C390004AD84ED652D456D23285B2849700000085
:10C3A000E780C0C7AA89268597000000E78020C9DA
:10C3B0002318A4FC268597000000E78040C82319B5
:10C3C000A4FC268597000000E78060C783D744005F
:10C3D0000A8A231AA4FC858393F7F70F230EF4FC33
:10C3E0008607BD0793F7073F3301F1408A8A014969
:10C3F0008347C4FD6367F902CE85130584FC232CB3
:10C4000054FD97000000E78080EA5281130104FC8C
:10C41000F2506254D2544259B259225A925A21616E
:10C420008280268597000000E78060C1931719007D
:10C43000D69705092390A7001379F90F55BF82807D
:10C4400097A7FF1F9387078D9C43D847A1679387C2
:10C45000A702631AF70A397106DE22DC26DA8000A9
:10C460004AD84ED652D456D23285B28497000000B4
:10C47000E780C0BAAA89268597000000E78020BC23
:10C48000FD572318A4FC26852319F4FC970000000F
:10C49000E780E0BA83D744000A8A231AA4FC858384
:10C4A00093F7F70F230EF4FC8607BD0793F7073FBA
:10C4B0003301F1408A8A01498347C4FD6367F90269
:10C4C000CE85130584FC232C54FD97000000E780E3
:10C4D00000DE5281130104FCF2506254D2544259DE
:10C4E000B259225A925A2161828026859700000013
:10C4F000E780E0B493171900D69705092390A700A9
:10C500001379F90F55BF828097A7FF1F9387878004
:10C510009C43D847A16789076310F70A397106DE83
:10C5200022DC26DA80004AD84ED652D456D2328542
:10C53000328997000000E78060AEAA894A8597009B
:10C540000000E780C0AF835749000A8A2318A4FC83
:10C55000858393F7F70F230CF4FC8607BD0793F749
:10C56000073F3301F1408A8A8144834784FD63E7B2
:10C57000F402CE85130584FC232A54FD97000000A5
:10C58000E780E0D25281130104FCF2506254D2548D
:10C590004259B259225A925A216182804A859700A3
:10C5A0000000E780C0A993971400D69785042390D4
:10C5B000A70093F4F40F55BF82809797FF1F9387CE
:10C5C00067759C43D847A1679387E704631EF70A02
:10C5D000397106DE22DC26DA80004AD84ED652D4E3
:10C5E00056D23285B28497000000E78020A3AA8942
:10C5F000268597000000E78080A42318A4FC2685E8
:10C6000097000000E780A0A3231AA4FC26859700CA
:10C610000000E780C0A283D744000A8A2319A4FC43
:10C62000858393F7F70F230EF4FC8607BD0793F776
:10C63000073F3301F1408A8A01498347C4FD63679C
:10C64000F902CE85130584FC232C54FD97000000CD
:10C65000E780E0C55281130104FCF2506254D254C9
:10C660004259B259225A925A2161828026859700F6
:10C670000000E780C09C93171900D6970509239006
:10C68000A7001379F90F55BF82809797FF1F9387F3
:10C6900067689C43D847A1679387C704631AF70A62
:10C6A000397106DE22DC26DA80004AD84ED652D412
:10C6B00056D23285B28497000000E7802096AA897E
:10C6C000268597000000E7808097FD572318A4FC7B
:10C6D0002685231AF4FC97000000E780409683D754
:10C6E00044000A8A2319A4FC858393F7F70F230ECD
:10C6F000F4FC8607BD0793F7073F3301F1408A8AB0
:10C7000001498347C4FD6367F902CE85130584FCA4
:10C71000232C54FD97000000E78060B9528113017B
:10C7200004FCF2506254D2544259B259225A925ADD
:10C7300021618280268597000000E7804090931752
:10C740001900D69705092390A7001379F90F55BF53
:10C7500082809797FF1F9387E75B9C43D847A16729
:10C76000DD076317F7041763FFFFE702439679714C
:10C770003285328497000000E780408A2AC62285ED
:10C7800097000000E780A08B2311A102228597006B
:10C790000000E780A088B2452300A1022808970086
:10C7A0000000E780C0B045611763FFFF6700639436
:10C7B00082809797FF1F9387E7559C43D847A167CF
:10C7C000938787046317F7041763FFFFE70223903B
:10C7D00079713285328497000000E78020842AC670
:10C7E000228597000000E78080852311A102228521
:10C7F00097000000E7808082B2452300A10228084C
:10C8000097000000E780A0AA45611763FFFF67005B
:10C81000438E82809797FF1F9387C74F9C43D847CB
:10C82000A1679387A7046312F7021763FFFFE7026C
:10C83000038A01112800814597000000E78020A7A6
:10C8400005611763FFFF6700C38A82809797FF1F08
:10C850009387474C9C43D847A16793875702631936
:10C86000F7021763FFFFE70283860111328597F015
:10C87000FFFFE780A07A2308A100814528009700E8
:10C880000000E780C0A205611763FFFF67006386B1
:10C8900082809797FF1F9387E7479C43D847A167FC
:10C8A0009387E702631BF7041763FFFFE702238206
:10C8B00001113285328497F0FFFFE7804078AA8427
:10C8C000228597F0FFFFE7808077854709E9228579
:10C8D00097F0FFFFE78080744205B337A00028007F
:10C8E0008145231891003ECA97000000E780209CF4
:10C8F00005611753FFFF6700C37F82809797FF1F73
:10C90000938747419C43D84799476313F7081753C8
:10C91000FFFFE702C37B79713285328497F0FFFF16
:10C92000E780C06F2AC6228597F0FFFFE78020715D
:10C930002310A102228597F0FFFFE780206E2301DC
:10C94000A102228597F0FFFFE780406DA301A102BD
:10C95000228597F0FFFFE780606C2302A102228509
:10C9600097F0FFFFE780806B2313A102228597F0E9
:10C97000FFFFE780A06AB2452314A10228089700B0
:10C980000000E780C09245611753FFFF67006376A0
:10C9900082809797FF1F9387E7379C43D847A1670B
:10C9A0009387C7036313F7081753FFFFE702237248
:10C9B00079713285328497F0FFFFE78020662AC6BE
:10C9C000228597F0FFFFE78080672310A102228570
:10C9D00097F0FFFFE780A0662311A102228597F060
:10C9E000FFFFE780A0632302A102228597F0FFFFEB
:10C9F000E780C062A302A102228597F0FFFFE780D3
:10CA0000E0612303A102228597F0FFFFE780006128
:10CA1000B245A303A102280897000000E7802089FF
:10CA200045611753FFFF6700C36C82801753FFFFF8
:10CA3000E702E36901112A8497F0FFFFE780005EB7
:10CA4000AA84228597F0FFFFE780605F228597F038
:10CA5000FFFFE780C05E035744008D4763F7E700A0
:10CA6000228597F0FFFFE780805D228597F0FFFF2A
:10CA7000E780E05C2800A68597000000E78020831F
:10CA800005611753FFFF6700C3669797FF1F9387E2
:10CA900067289C43D847A167FD07631FF70017531A
:10CAA000FFFFE702C362328597000000E78040F88D
:10CAB0001753FFFF6700E36382809797FF1F9387F9
:10CAC00067259C43D847A167E5076315F708175307
:10CAD000FFFFE702C35F79713285328497F0FFFF71
:10CAE000E780C0532AC6228597F0FFFFE7802055D4
:10CAF000228597F0FFFFE78080542310A102228552
:10CB000097F0FFFFE780A053520551812311A10246
:10CB100022852302010297F0FFFFE7802050A30245
:10CB2000A102228597F0FFFFE780404F2303A10277
:10CB3000228597F0FFFFE780604EB245A303A10274
:10CB4000280897F0FFFFE780807645611753FFFFC5
:10CB50006700235A82809797FF1F9387A71B9C43E8
:10CB6000D847A1679387E703631FF7001753FFFFB9
:10CB7000E702E355328597000000E78060EB17532A
:10CB8000FFFF6700035782809797FF1F93878718DF
:10CB90009C43D847A16793874704631EF702175346
:10CBA000FFFFE702C35279713285328497F0FFFFAD
:10CBB000E780C0462AC6228597F0FFFFE78020481D
:10CBC000B245280897F0FFFFE780606E4561175374
:10CBD000FFFF6700035282809797FF1F9387871399
:10CBE0009C43D847A167938787026310F7041753C4
:10CBF000FFFFE702C34D79713285328497F0FFFF62
:10CC0000E780C0412AC6228597F0FFFFE7800041F8
:10CC1000B2452300A102280897F0FFFFE7802069B2
:10CC200045611753FFFF6700C34C82801753FFFF16
:10CC3000E702E349011197F0FFFFE780203EAA8554
:10CC4000280097F0FFFFE780806605611753FFFF1C
:10CC50006700234A9797FF1F9387C70B9C43D847CA
:10CC6000A167D107631FF7001753FFFFE7022346B1
:10CC7000328597000000E780A0FB1753FFFF670095
:10CC8000434782809797FF1F9387C7089C43D847E5
:10CC9000A167C507631FF7001753FFFFE702234390
:10CCA000328597000000E780A0F81753FFFF670068
:10CCB000434482809797FF1F9387C7059C43D847BB
:10CCC000A167B907631FF7001753FFFFE70223406F
:10CCD000328597000000E780A0F51753FFFF67003B
:10CCE000434182809797FF1F9387C7029C43D84791
:10CCF000A167AD07631FF7001753FFFFE702233D4E
:10CD0000328597000000E780A0F21753FFFF67000D
:10CD1000433E82809797FF1F9387C7FF9C43D84766
:10CD200089476318F7021753FFFFE702433A0111DF
:10CD3000328532C897F0FFFFE780402EAA85280091
:10CD400097F0FFFFE780A05605611753FFFF6700CC
:10CD5000433A82809797FF1F9387C7FB9C43D8472E
:10CD6000A1678D076311F7041753FFFFE70223360E
:10CD700001113285328497F0FFFFE780202A1306E5
:10CD80006100AA844C00228597300000E780C02310
:10CD90002800A68597F0FFFFE780605105611753D3
:10CDA000FFFF6700033582809797FF1F9387C7F6C1
:10CDB0009C4381CFDC4391CB1753FFFFE702233124
:10CDC00082971753FFFF6700C33282801753FFFF1C
:10CDD000E702E32F79713C08AE843ED2A165B70724
:10CDE0000A002A843ED448103C08DD053ED636C4ED
:10CDF00032C63AC297D0FFFFE780E02F12474810B3
:10CE0000BA8597F0FFFFE780C01332464810B2851D
:10CE100097F0FFFFE780E014A2464810B68597F030
:10CE2000FFFFE7800012501001478146A68522854A
:10CE300097D0FFFFE780805145611753FFFF6700E0
:10CE4000432B1753FFFFE702832801117C000329BE
:10CE5000C501AE843ECAA165B70707002A843ECC4F
:10CE600048087C00C5053ECE97D0FFFFE780A0288C
:10CE70008345D900480897F0FFFFE780800C5008F1
:10CE800001478146A685228597D0FFFFE780004CA9
:10CE900005611753FFFF6700C3251753FFFFE70224
:10CEA000032383C7950093F7F707A384F500970042
:10CEB0000000E78040F91753FFFF670083231753F3
:10CEC000FFFFE702C32079713C08AE843ED2A16522
:10CED000B70709002A843ED448103C0893854504CE
:10CEE0003ED632C636C497D0FFFFE780C020A246A8
:10CEF0004810B68597F0FFFFE780A004324648103F
:10CF0000B28597F0FFFFE780C005501001478146CA
:10CF1000A685228597D0FFFFE780404345611753E0
:10CF2000FFFF6700031D1753FFFFE702431A83C784
:10CF3000950041112A8493F7F707A384F500328501
:10CF40002EC697F0FFFFE780800F85672AC46370C5
:10CF5000F50297700000E78020E92246B24509ED0E
:10CF600011478146228597000000E78060E6410175
:10CF70001753FFFF6700E31701478346F501DDB74D
:10CF80001753FFFFE702031301113C003ECAB70726
:10CF90000A003ECC3C003ECE83C79500AA8932856C
:10CFA00093F7F707A384F5002E8497F0FFFFE7803F
:10CFB00000098567637DF504A165AA8493858504CE
:10CFC000480897D0FFFFE780001326859770000080
:10CFD000E78080E12A8929E19145480897F0FFFF21
:10CFE000E78020F6A685480897F0FFFFE78060F706
:10CFF000CA85480897F0FFFFE780A0F40147814603
:10D000005008A2854E8597D0FFFFE7802034056148
:10D010001753FFFF6700430D8145480897F0FFFF56
:10D02000E78020F20349090275BF1753FFFFE702AB
:10D03000630879711C103ECAB7070F003ECC404D03
:10D040001C10AA84AE894808994532C636893ECE5E
:10D0500097D0FFFFE780200A32464808B28597F054
:10D06000FFFFE78000EE630C0902A545480897F032
:10D07000FFFFE780C0E62546CA8597200100E780CC
:10D0800020A4500801478146CE85268597D0FFFF12
:10D09000E780C02B45611753FFFF6700E30483550A
:10D0A000C402480897F0FFFFE780A0EB0355E402B5
:10D0B000814505C5854785456301F502C167FD17B3
:10D0C0009305F00F630BF5007D1597700000E78066
:10D0D000208E9305150093F5F50F480897F0FFFF94
:10D0E000E78020E683450403480897F0FFFFE780C8
:10D0F00040E583451403480897F0FFFFE78060E4AC
:10D1000083552403480897F0FFFFE78080E58355A7
:10D110004403480897F0FFFFE780A0E49DB717534A
:10D12000FFFFE702C3FA83C795008146014693F7E4
:10D13000F707A384F50097000000E78040EF17533E
:10D14000FFFF670003FB1753FFFFE70243F8797106
:10D150003E841C103ECA2E89B7070F00A1653ECC45
:10D16000FD051C10AA84480842C03AC23ECE36C40F
:10D1700032C697D0FFFFE78000F832464808B285F4
:10D1800097F0FFFFE780E0DBA2464808B68597F0FE
:10D19000FFFFE78000DD12474808BA8597F0FFFFE0
:10D1A000E78020DC0248630C08029145480897F0AC
:10D1B000FFFFE780C0D21146A28597200100E780DB
:10D1C0002090500801478146CA85268597D0FFFFE9
:10D1D000E780C01745611753FFFF670083F189455A
:10D1E000480897F0FFFFE78080CF834704002300C3
:10D1F000F50083471400A300F500E1B71753FFFFC4
:10D20000E70243EB83C7950001112A8A93F7F707DA
:10D21000A384F5003285AE8432C697F0FFFFE78025
:10D2200000E232462A89328597F0FFFFE78000DF6F
:10D2300085676373F902AA894A8597700000E780C1
:10D24000A0BA2A8419ED114781464A86A6855285DF
:10D2500097000000E780C0B705611753FFFF670024
:10D26000A3E89387E9FF93F7F70F0547E366F7FE17
:10D270008347F50195EB8947E380F9FE8346F40186
:10D28000528501474A86A68597000000E78040B492
:10D29000A167D90748083ECC230A010002CE9700B7
:10D2A0000000E780A0B04DBF639EE7008947639E02
:10D2B000F90093071020231FF50097700000E78006
:10D2C000C0B76DBF0947E39BE7FA8D47E398F9FACA
:10D2D000228597700000E78080DF9797FF1F938774
:10D2E000A7C29C4399E79797FF1F9387A7AB9C43DF
:10D2F00099C703D5040097800000E780A0CE231FC4
:10D30000040022855DBF1753FFFFE70243DC0111D4
:10D310003C003ECAB7070B003ECC3C003ECE83C764
:10D3200095002A89328593F7F707A384F500AE8428
:10D3300097F0FFFFE780A0D093170501C187635ADC
:10D34000F006A1652A849385E502480897D0FFFF7F
:10D35000E78060DAA285480897F0FFFFE78060C0A9
:10D360009797FF1F938707A49C43A9EB01449375EC
:10D37000F40F480897F0FFFFE780A0BC9355844066
:10D3800093F5F50F480897F0FFFFE78080BB9355B2
:10D39000044193F5F50F480897F0FFFFE78060BA66
:10D3A000014781465008A6854A8597D0FFFFE78050
:10D3B000E0F905611753FFFF6700A3D34165854678
:10D3C0000546A2857D1597500000E78060BD59DDB8
:10D3D000510597000100E780808F13044006334415
:10D3E000850271B71753FFFFE70263CE0111B7073C
:10D3F00006003EC683C7950021642A8993F7F70784
:10D40000A384F500AE8428009305A4040AC40AC8C6
:10D4100097D0FFFFE78020CE300001478146A685E8
:10D420004A8597D0FFFFE78060F297E0FFFFE78033
:10D43000801513049404480822CC230A010002CE6C
:10D4400097000000E780809605611753FFFF670093
:10D4500043CA1753FFFFE702E3C5C1642A890144A9
:10D460009799FF1F9389C9AB130A8002FD1497E0B7
:10D47000FFFFE78080C16347A40001451753FFFF0A
:10D48000670083C6B307440303A7C90ABA9703D743
:10D4900007006306970083D72700638427010504EC
:10D4A000F9B70545E1BF1753FFFFE702A3C02A8A7A
:10D4B0002E8999C123A0050081498144979AFF1FB5
:10D4C000938ACA85614B97E0FFFFE78040C263C73C
:10D4D000A4004E851753FFFF670003C13384640324
:10D4E00083A70A003E948357040099E76304090068
:10D4F000232089008504C1BF4146D285130544001D
:10D5000097100100E780605975F5A289E5B71753B8
:10D51000FFFFE70223BA39717C083ED4B7070A003F
:10D520003ED67C083ED883C795002A8A328593F779
:10D53000F707A384F5002E8932C697F0FFFFE78036
:10D5400000B085676373F5083246AA84328597F088
:10D55000FFFFE780A0AC8547AA8963E8A706A1651D
:10D5600093858504281097D0FFFFE780C0B82685F3
:10D5700097700000E78040872A8429ED91452810A4
:10D5800097F0FFFFE780E09BA685281097F0FFFF4C
:10D59000E780209DCE85281097F0FFFFE780609AF6
:10D5A000014781463010CA85528597D0FFFFE7803A
:10D5B000E0D9A1679387770448183EDC230A01026B
:10D5C00002DE97F0FFFFE780607E21611753FFFFC7
:10D5D000670083B18145281097F0FFFFE7806096D0
:10D5E000A685281097F0FFFFE780A0979797FF1F69
:10D5F000938787C99C4381CB22856389090097D093
:10D600000000E78040248345040271B797D00000F2
:10D61000E780C022CDBF1753FFFFE702A3A983C74E
:10D6200095004111AA8993F7F707A384F500328585
:10D63000AE84328A97F0FFFFE78060A08567637F42
:10D64000F5022A8997600000E780007A2A849146D3
:10D6500031C58347F50105476387E70291C70D4749
:10D660006366F704AD461DA89305050303250A006C
:10D67000414697100100E78040420DE941011753F0
:10D68000FFFF670063A69305950803250A0041463E
:10D6900097100100E7806040814669F54A86A685BB
:10D6A0004E8597000000E780C081C9BF83250A002E
:10D6B0001305940897700000E780A02919C1C1469E
:10D6C000F1BF9797FF1F938727849C4399E797871C
:10D6D000FF1F9387276D9C4399C722859780000081
:10D6E000E780208A69FD8547A30FF400228597B063
:10D6F0000000E7806084228597600000E780E07387
:10D700004E8581464A86A68597F0FFFFE780607BBD
:10D71000A1679387570448003EC42302010002C654
:10D7200097F0FFFFE780806891BF1753FFFFE70284
:10D73000839783C795004111AA8993F7F707A384BC
:10D74000F50032852E89B28A97F0FFFFE780208F9F
:10D7500085676374F50EAA8497600000E780C0684F
:10D760002A840DED416B014A978BFF1F938B4B7BF6
:10D77000130C400E7D1B19A833048A0383A70B0BDF
:10D780003E948357C40163836705050A97E0FFFF52
:10D79000E780A08EE342AAFE95460DA08357C501FF
:10D7A000639697029305050303A50A004146971067
:10D7B0000100E780802E994611E181462686CA85C0
:10D7C0004E8597F0FFFFE780C06F85A883A50A000C
:10D7D0001305040397700000E780A017C14679FD88
:10D7E0002285231E940097A00000E780E074228524
:10D7F00097600000E78060649797FF1F9387C7A832
:10D800009C43A9C323000402228597D00000E7802F
:10D8100040F04E8581462686CA8597F0FFFFE78057
:10D82000406AA1679387070448003EC423020100B1
:10D8300002C697F0FFFFE780605741011753FFFFD3
:10D840006700E38989472300F402E1B7397106DEF6
:10D8500022DC4AD8800052D456D25AD026DA4ED68C
:10D860005ECE2E8A32892A8B97D0FFFFE780E07D3B
:10D870000605710541998A8A3301A140232224FCBF
:10D88000231404FC97D0FFFFE780207C83479A0095
:10D890000605350593F7F7072315A4FCA304FA0042
:10D8A0004A85232624FC97E0FFFFE7804079931701
:10D8B0000501C1876340F0025681130104FCF25058
:10D8C0006254D2544259B259225A925A025BF24BD4
:10D8D00021618280AA844A8597E0FFFFE780207655
:10D8E000AA894A8597E0FFFFE7806075A165938567
:10D8F000C5022A89130544FC97C0FFFFE780A07F7B
:10D90000268597C0FFFFE780E073854511C94A86E9
:10D91000CE8597C0FFFFE780606DAA8B21E989451E
:10D92000130544FC97E0FFFFE780A061A68513057F
:10D9300044FC97E0FFFFE780C062CE85130544FCFE
:10D9400097E0FFFFE780E061CA85130544FC97E09C
:10D95000FFFFE780006101478146130644FCD28542
:10D960005A8597D0FFFFE780609EB9B781451305C0
:10D9700044FC97E0FFFFE780C05CA685130544FCEC
:10D9800097E0FFFFE780E05DCE85130544FC97E05C
:10D99000FFFFE780005DCA85130544FC97E0FFFFA9
:10D9A000E780205C814497D0FFFFE780006AE3D4E2
:10D9B000A4FA83A70B0113971400BA9783D5070025
:10D9C00099C5130544FC97E0FFFFE7808059850463
:10D9D000D9BF797106D622D44AD000184ECE52CC87
:10D9E00056CA26D25AC8AE893289AA8A97D0FFFF72
:10D9F000E780A0650605690541990A8A3301A140BF
:10DA0000232A24FC231C04FC97D0FFFFE780E0635B
:10DA100083C7990006052D0593F7F707231DA4FC7E
:10DA2000A384F9004A85232E24FC97E0FFFFE780BA
:10DA3000006193170501C187634FF0005281130104
:10DA400004FDB250225492540259F249624AD24A19
:10DA5000424B45618280AA844A8597E0FFFFE780B8
:10DA6000005EA1659385A5022A89130544FD97C030
:10DA7000FFFFE7804068268597C0FFFFE780805C56
:10DA8000854509C9CA8597C0FFFFE78020592A8BC1
:10DA900029E18945130544FD97E0FFFFE780604ACF
:10DAA000A685130544FD97E0FFFFE780804BCA85FC
:10DAB000130544FD97E0FFFFE780A04A0147814638
:10DAC000130644FDCE85568597D0FFFFE78000887A
:10DAD000B5B78145130544FD97E0FFFFE780604639
:10DAE000A685130544FD97E0FFFFE7808047CA85C0
:10DAF000130544FD97E0FFFFE780A046814497D0DF
:10DB0000FFFFE7808054E3DBA4FA83270B01139720
:10DB10001400BA9783D5070099C5130544FD97E013
:10DB2000FFFFE78000448504D9BF1743FFFFE702EA
:10DB3000035A83474500404DD5EFFD575DC48346EA
:10DB4000940009476363D70A0346B400854663EE31
:10DB5000C6088306E40063CA06085C45F9562390AC
:10DB6000D7009787FF1F83C7A71B99E3A304E4008F
:10DB70009787FF1F938707239C4381E78947A30665
:10DB8000F4009787FF1F938727709C4381E789479D
:10DB90002306F4009705000093854506AA84130523
:10DBA000040197F00000E7802010FD57231AF402CB
:10DBB00081471CDC01489787FF1F23AF8714978795
:10DBC000FF1F9387A715232E040304C0804397D01B
:10DBD000FFFFE780C05161463306C50281452285BB
:10DBE0009740FFFFE780A05181473E851743FFFF25
:10DBF00067002350FD57D5BF1743FFFFE702234DB2
:10DC00002A840355450297600000E780E01D19E56E
:10DC1000231E04001743FFFF6700A34D8357E40151
:10DC2000F5DB930504FF174501001305253597E043
:10DC30000000E780E014F9BF1743FFFFE702234924
:10DC40002E89A16541119385E5032A8436C432C625
:10DC5000BE843AC297C0FFFFE780E04912472285A1
:10DC6000BA8597E0FFFFE780C02D32462285B28556
:10DC700097E0FFFFE780E02EA2462285B68597E079
:10DC8000FFFFE780002E630309029145228597E09C
:10DC9000FFFFE780C0241146A68597100100E780AA
:10DCA00020E241011743FFFF6700A3448945228515
:10DCB00097E0FFFFE780A02283C704002300F50060
:10DCC00083C71400A300F500E9BF1743FFFFE70275
:10DCD000034083C79500444D054793F7F707A38496
:10DCE000F5001C42411183C707006367F7062E84C5
:10DCF0002A89B1C003C7D400630FF7021787FF1F3B
:10DD00001307470A184305C3A386F40097A0000031
:10DD1000E780404A83C7D40099E741657D15974065
:10DD20000000E780403083D72403918B89C797E0B8
:10DD30000000E780C0134A85A28597F0FFFFE780C7
:10DD40008010A167C10748003EC42302010002C63B
:10DD500097F0FFFFE780800541011743FFFF670051
:10DD600043391743FFFFE702833603D745008D474A
:10DD7000AA8441112E8432892E8563E3E70297E05D
:10DD8000FFFFE780C02BAA8523000900268597C0E6
:10DD9000FFFFE780A02841011743FFFF67006335BD
:10DDA00097E0FFFFE780A0292AC6228597E0FFFFC2
:10DDB000E780E028B24585472A862300F9002685BA
:10DDC00097C0FFFFE7808022F9B7397106DE22DCB9
:10DDD00026DA80004ED652D456D24AD85AD05ECED9
:10DDE000AE89B284AA8A97D0FFFFE7800025060596
:10DDF0001305250241990A8A3301A140232224FCFC
:10DE0000231404FC97D0FFFFE780202383C79900E9
:10DE100006054D0593F7F7072315A4FCA384F90025
:10DE20002685232624FC97E0FFFFE78040219317F7
:10DE30000501C1876340F0025281130104FCF250D6
:10DE40006254D2544259B259225A925A025BF24B4E
:10DE500021618280AA8B03AB040097C0FFFFE7809B
:10DE6000601E51E583D7440001498544F11793B7FB
:10DE70001700A301F4FC834734FCA165C9C793854F
:10DE8000E504130544FC97C0FFFFE780C026A68584
:10DE9000130544FC97E0FFFFE780A00ADE85130529
:10DEA00044FC97E0FFFFE780C00B834734FC11463A
:10DEB00091E30946DA85130544FC97E0FFFFE7800C
:10DEC00060058144630A0900416B7D1B97D0FFFF09
:10DED000E780A01663CCA40201478146130644FCE8
:10DEE000CE85568597C0FFFFE7804046B1B7A6852F
:10DEF000130634FC97000000E780E0E69334150039
:10DF00002A8986048DBF9385C504A5BF8327C900D0
:10DF100013971400BA9783D507006388650113052A
:10DF200044FC97E0FFFFE780C003850445B7174333
:10DF3000FFFFE702431779711C103EC4B7070F00BB
:10DF40003EC61C103EC883C79500AA8A328593F747
:10DF5000F707A384F500AE89328497E0FFFFE780DE
:10DF6000000E93170501C187635AF0062A8A22859D
:10DF700097E0FFFFE780A00C2A895285032B04005D
:10DF800097C0FFFFE780000C39ED835744008144C0
:10DF90000544F11793B71700A303F10083457100FF
:10DFA000DA872287CA865286280097000000E78019
:10DFB000E0C8014781463000CE85568597C0FFFFF7
:10DFC000E780C038A1679387D70348083ECC230A6F
:10DFD000810026CE97F0FFFFE78040DD45611743C3
:10DFE000FFFF6700C30FA2851306710097000000B2
:10DFF000E78060D7AA84094455D13544E30055FB36
:10E000004A8597F0FFFFE78000450D4441D9014460
:10E0100097D0FFFFE7806002634DA400C16B01440D
:10E02000FD1B97D0FFFFE7804001634EA40015441D
:10E03000B5B7DC4413171400BA9783D7070063837E
:10E0400027030504F1B7D84493171400BA9703D7F0
:10E050000700631B770123902701268597A0000006
:10E06000E78080DB01441DBF050465BF1743FFFF48
:10E07000E702430483C7950041112A8A93F7F70703
:10E08000A384F50032852E89328497E0FFFFE78074
:10E0900000FB93170501C1876353F006AA89228507
:10E0A00097E0FFFFE780A0F92311A1004E85832AA6
:10E0B000040097C0FFFFE780E0F839E5835744008C
:10E0C00085440144F11793B71700A300F1000348FA
:10E0D000110003572100D6875285CE862686CA8531
:10E0E00097F0FFFFE7806006A167F10748003EC494
:10E0F0002302910022C697F0FFFFE78020CB410169
:10E100001743FFFF670043FEA28513061100970027
:10E110000000E78040C52A84894455D983572100EF
:10E1200011678544BA97C2071167C1831307F7EFD8
:10E13000E36FF7F89787FF1F938707DD9C4381CB39
:10E1400085451305210097500000E7802075835511
:10E1500021002285814497C0FFFFE78040E525D953
:10E1600023100500228597A00000E78040CD85B7E9
:10E170001743FFFFE70223F383C7950041112A8B62
:10E1800093F7F707A384F50032852E8A328497E04F
:10E19000FFFFE780C0EA93170501C1876351F006CE
:10E1A000AA8A228597E0FFFFE78060E92A895685E1
:10E1B000832B040097C0FFFFE780C0E831E5835759
:10E1C000440081440544F11793B71700A301F100FF
:10E1D00003483100DE875A854A87D6862286D28553
:10E1E00097F0FFFFE78060F6A167ED0748003EC4A7
:10E1F0002302810026C697F0FFFFE78020BB410184
:10E200001743FFFF6700A3EDA285130631009700B7
:10E210000000E78040B5AA8409445DD99167CA9798
:10E22000C2071167C1831307F7EF0544E362F7FAEA
:10E23000CA8597C0FFFFE78080D7014451F9814923
:10E2400097D0FFFFE78060E063DBA90098489397D1
:10E250001900BA9703D7070005EF2390270197D03D
:10E26000FFFFE78080DE1544E384A9F6268597A0AA
:10E270000000E780C0BC9787FF1F9387E7C89C43D7
:10E280000144B9D74A8597500000E780C05889B744
:10E2900085097DB71743FFFFE702C3E179713E842B
:10E2A0007C083EC82E8AB7071400A1653ECAE50562
:10E2B0007C08AA89080836C4428932C6BA8AC6844C
:10E2C0003ECC97C0FFFFE78000E3CA85080897E0CF
:10E2D000FFFFE78000C732460808B28597E0FFFFDE
:10E2E000E78020C8A246630A09049D45080897E014
:10E2F000FFFFE780C0BE1D4681459740FFFFE780D6
:10E3000000E063890A089145080897E0FFFFE7806D
:10E3100000BD1146A68597000100E780607A1008CD
:10E3200001478146D2854E8597C0FFFFE7800002F6
:10E3300045611743FFFF670023DBB685080897E0B8
:10E34000FFFFE78000C21C400808D8439355C7016F
:10E35000858912075183B205D98D97E0FFFFE780C9
:10E3600040C01C40080883C5870097E0FFFFE78096
:10E3700040BD1C40080883C5A70097E0FFFFE78069
:10E3800040BC1C40080883C5970097E0FFFFE7806A
:10E3900040BB85BF8945080897E0FFFFE78020B4B0
:10E3A00083C704002300F50083C71400A300F50011
:10E3B000BDB71743FFFFE702E3CF83C795004111C5
:10E3C000AA8993F7F707A384F5003285AE843284D7
:10E3D00097E0FFFFE780A0C693170501C187635D43
:10E3E000F0042A89032A040097C0FFFFE78080C554
:10E3F00019E9835744000548F11793B71700A3079D
:10E40000F100814631A81306F100A28597000000B3
:10E41000E78060951DC51C459DC783D64700014810
:10E420000347F10093078500D2884A86A6854E856A
:10E4300097000000E78040E641011743FFFF6700B7
:10E44000A3CA09487DBF1D486DBF1743FFFFE70200
:10E4500063C665715C083EC4B7077B013EC65C08B5
:10E460003EC883C795002A8A328593F7F707A384AD
:10E47000F500AE8997E0FFFFE78040BA8357E100DF
:10E48000E1C78945280097C0FFFFE780C0C68145E6
:10E49000280097E0FFFFE780C0AA97C0FFFFE78052
:10E4A000A0CC9787FF1F938727DE9C431784FF1F0D
:10E4B00003440487AA843334800099C3136424007E
:10E4C0009787FF1F9387078E9C4399C3136444006B
:10E4D0009787FF1F938747A39C4399C313648400C6
:10E4E00083D504002800014997E0FFFFE78060A77B
:10E4F00083D52400280097E0FFFFE78080A683D51E
:10E500004400280097E0FFFFE780A0A597D0FFFF19
:10E51000E780A0AE93150501C181280097E0FFFFB9
:10E52000E78020A4A285280097E0FFFFE78060A392
:10E530009C446360F902014781463000CE855285D4
:10E5400097C0FFFFE78080E059611743FFFF670036
:10E55000A3B9DC441314490028003E9497E0FFFF60
:10E56000E780609683474400034754008907060705
:10E57000BA978607E36AF5FC835524002800814A90
:10E5800097E0FFFFE780E09D83454400280097E087
:10E59000FFFFE780009B83455400280097E0FFFFC2
:10E5A000E780209A8347440063C9FA00814A834781
:10E5B000540063C1FA020509A5BF1C4413975A0011
:10E5C0002800BA9783D50700850A97E0FFFFE78008
:10E5D0004099C9BF032BC40093975A0028003E9B63
:10E5E00083552B00850A97E0FFFFE78080978355CE
:10E5F0000B00280097E0FFFFE780A0964DBF174370
:10E60000FFFFE702C3AC5C4993E717005CC997A022
:10E610000000E78020B61743FFFF670083AD174374
:10E62000FFFFE702C3AA2E84814597F0FFFFE78032
:10E63000C0E705C583570500FD172310F50009C481
:10E64000835725002310F40097000000E78060FB4B
:10E6500001451743FFFF6700C3A931457DD823104B
:10E660000400C5BF1743FFFFE702C3A483C795009B
:10E6700041112A8A93F7F707A384F50032852E8982
:10E68000328497E0FFFFE780809B93170501C187E5
:10E690006356F006AA89C145228597E0FFFFE7800F
:10E6A000A0802A8B4E85832A040097C0FFFFE78055
:10E6B000609931E983574400231101000544F117A3
:10E6C00093B71700A300F1008144034811000357DA
:10E6D0002100D6875285CE862286CA8597F0FFFF15
:10E6E000E780A0A6A1679387170248003EC42302D3
:10E6F000810026C697E0FFFFE780406B410117438A
:10E70000FFFF6700639E13061100A28597F0FFFFCD
:10E71000E7806065AA8409E523110100094475B703
:10E72000930521005A8597000000E78080EF83570A
:10E7300021002A84D9DB9777FF1F9387E77C9C43CE
:10E7400081CB85451305210097500000E780001517
:10E75000835521002685314497C0FFFFE78020853F
:10E760002DD523100500268597900000E780206DA9
:10E770000144A1BF1743FFFFE702639541112E89B2
:10E780006C00AA8402C697F0FFFFE78000D20DC19B
:10E790000357050005072310E50097000000E780F8
:10E7A00040E681473E8541011743FFFF67006394C0
:10E7B0003247954765DBCA85268597300000E7809C
:10E7C000400DC147E34005FE3244854741462310D2
:10E7D000F40083570900A685130544002311F400B3
:10E7E00097000100E780C02D228545BF1743FFFF3A
:10E7F000E702438C83C795004111AA8A93F7F70774
:10E80000A384F5003285AE89328497E0FFFFE7806C
:10E81000008393170501C1876356F0062A8AC14514
:10E82000228597D0FFFFE7802068AA845285032BBA
:10E83000040097C0FFFFE780E08031E98357440080
:10E84000231101008544F11793B71700A300F100CD
:10E8500001440348110003572100DA875685D28608
:10E860002686CE8597F0FFFFE780208EA1679387ED
:10E87000070248003EC42302910022C697E0FFFF32
:10E88000E780C05241011743FFFF6700E385A2857F
:10E890001306110097F0FFFFE780E04C2A8409E59A
:10E8A00023110100894475B726859305210097003F
:10E8B0000000E78060ECAA8449FD83552100228591
:10E8C00097B0FFFFE780A06E49F5014997C0FFFFB1
:10E8D000E780A077635DA900184893171900BA97DD
:10E8E00003D707000DEF035721002390E70097C0DF
:10E8F000FFFFE7808075630625039777FF1F9387E7
:10E90000A7609C4399C70355210097500000E780FA
:10E9100080F0228597900000E78060521DBF0509B6
:10E9200075B795443DB705C19307F00F630FF50028
:10E93000C547630CF5009307F5FF05453315F50052
:10E940004205418182800145828041657D1582803A
:10E95000B9E91733FFFFE7028377034506033284E3
:10E9600097000000E78060FC9305803EB305B50288
:10E97000C205C18181CD0357E402854763F8E700F2
:10E980001305040197E00000E78020428357E4026A
:10E9900041677D176385E700FD172317F4021733DE
:10E9A000FFFF6700037582801733FFFFE702A36F45
:10E9B000004283C79500444D0349140093F7F707BD
:10E9C000A384F50083470400220911673369F90025
:10E9D000A167B347F90041112A8BAE8A63ECE70EB9
:10E9E000834724001307C00EB91793F7F70F63731B
:10E9F000F71003473400C14763EEE70E8347440036
:10EA00001307E00793C707086371F70C8349840075
:10EA100083477400A209B3E9F900856763F7F90A2F
:10EA2000034A6400834754004E85220A336AFA0081
:10EA300097500000E780403B61C123962403834B3D
:10EA40003400137AFA00239A340323887403239939
:10EA5000440393890401631C090023A6040223983C
:10EA600004024E8597E00000E78060363DA0034930
:10EA700024004A8597000000E78020EB2397A4023A
:10EA8000834744004E85A388F402E38D0BFCE30B1F
:10EA900009FC97E00000E780202F97900000E780B6
:10EAA000007381460146D6855A8597E0FFFFE780CF
:10EAB0000058A167938797033EC4230201004800D2
:10EAC00002C697E0FFFFE780602E41011733FFFF8A
:10EAD0006700E3608544A2862686D6855A8597E03E
:10EAE000FFFFE780C054A167938797033EC42302CA
:10EAF0009100F1B7BD44C5B79144F1BF1733FFFF93
:10EB0000E702435B01111C08404D3EC2B7070F00EE
:10EB10003EC41C083EC62A89AE8997C0FFFFE78025
:10EB2000A0DA585C1C5C6346B70E6394E50063E2B0
:10EB3000A70E3385A740B3B7A700B305B7401306A8
:10EB4000803E81469D8D97000100E78080B7931439
:10EB50000501C180A1659385C503480097B0FFFFFB
:10EB6000E78060598145480097D0FFFFE780603D0E
:10EB700083550404480097D0FFFFE780803E83550B
:10EB80002404480097D0FFFFE780A03D814589CC51
:10EB9000C167FD179305F00F6388F4002685975031
:10EBA0000000E780E0E0AA85480097D0FFFFE780FB
:10EBB000403903554404814501CDC167FD179305D4
:10EBC000F00F6307F50097500000E78060DEAA852C
:10EBD000480097D0FFFFE780C036834564044800B3
:10EBE00097D0FFFFE780E03583457404480097D055
:10EBF000FFFFE7800035500001478146CE854A85FA
:10EC000097B0FFFFE780807405611733FFFF67004F
:10EC1000A34D814481B71733FFFFE702434B83C7FE
:10EC2000950093F7F707A384F50097000000E780AD
:10EC300020ED1733FFFF6700C34B1733FFFFE702D9
:10EC4000634783C795004111404D93F7F707A384AD
:10EC5000F5002A8A3285B284AE8997D0FFFFE7801B
:10EC6000003E2A8B268597D0FFFFE780403D2A890A
:10EC7000268597D0FFFFE780603A93170B0163CAA0
:10EC80000702E177CA97C207C183116763E3E7020E
:10EC900093070910C207C1831307B00F637BF70006
:10ECA00093170901C187AA8A634AF000C54763FE2A
:10ECB000570141011733FFFF6700034397B0FFFF80
:10ECC000E780C028E31725FFD5B763080B0263066A
:10ECD0000902814463890A02B7077F002310640593
:10ECE000231124057CC0568597000000E780E0C30F
:10ECF0009304803EB304950239A0B7077F00232018
:10ED000004047CC081440355240497E00000E7809C
:10ED1000A0A3A1C497C0FFFFE78000BB269593D7AF
:10ED2000F44133379500AE97BA9708DC5CDCCE85AA
:10ED3000528597000000E780A0DC99E023220404BC
:10ED4000A1679387B70348003EC42302010002C6AF
:10ED500097E0FFFFE7808005A9BF814701481CDCE1
:10ED6000232E0403E9B71733FFFFE702433697C0AA
:10ED7000FFFFE780C037E1473305F5029145975023
:10ED80000000E78000C5E55711C59777FF1F23A74F
:10ED9000A7F881473E851733FFFF67008335854716
:10EDA0001777FF1F230EF7F682801733FFFFE70266
:10EDB00003329777FF1F938727F680433DC0835721
:10EDC00004046390A70683572404639CB704368920
:10EDD000B28497C0FFFFE78020AF5C5C63C3B704D9
:10EDE0006395B7001C5C63EEA7028347640463F37A
:10EDF000F400A6872303F4048347740463F39700A5
:10EE0000A687A303F4048357440441677D176385F1
:10EE1000E70085072312F4043C4481C7CA85268590
:10EE200082971733FFFF6700C32C9777FF1F9387E5
:10EE3000A7EE9C43014599C303C587008280173321
:10EE4000FFFFE702C3280111B70707003EC683C7CB
:10EE50009500584D0AC493F7F7070AC8A384F50034
:10EE60002A89AE8411CB1C4283C707002304F70014
:10EE700097900000E7800034216493055402280035
:10EE800097B0FFFFE780202797000000E78020FA77
:10EE9000AA85280097D0FFFFE780A00A300001472D
:10EEA0008146A6854A8597B0FFFFE780204A130474
:10EEB0004402480822CC230A010002CE97E0FFFF5B
:10EEC000E780C0EE05611733FFFF67008322173329
:10EED000FFFFE702C31F01117C003ECAB70707000E
:10EEE0003ECC7C003ECE83C795002E84AA8493F747
:10EEF000F707A384F500A16593855502480897B0EC
:10EF0000FFFFE780401F97000000E78040F2AA85DE
:10EF1000480897D0FFFFE780C002500801478146AC
:10EF2000A285268597B0FFFFE78040420561173331
:10EF3000FFFF6700031C9777FF1F9387E7DD9C4364
:10EF4000094599C303C5970082809777FF1F938770
:10EF5000A7DC9C43094599C303C5D70082809777F6
:10EF6000FF1F938767DB9C43014599C303C5A70037
:10EF700082801733FFFFE702E3130111B707080090
:10EF80003EC683C79500404D0AC493F7F7070AC8E9
:10EF9000A384F5002A89AE8429C41442854703C797
:10EFA000060063E0E70A83479400094681496380CD
:10EFB000C702B307F740A304E400B339F00083C7E6
:10EFC00016002305F40097900000E780A01E035769
:10EFD0002403058B19C76386090097D00000E780DA
:10EFE00000E9216493058402280097B0FFFFE780C1
:10EFF000801097000000E78040F4AA85280097D091
:10F00000FFFFE78000F497000000E78080F5AA8505
:10F01000280097D0FFFFE780C0F20147814630000B
:10F02000A6854A8597B0FFFFE7804032130474023B
:10F03000480822CC230A010002CE97E0FFFFE780B8
:10F04000E0D605611733FFFF6700030A1733FFFFA0
:10F05000E702E30701117C003ECAB70708003ECC77
:10F060007C003ECE83C795002E84AA8493F7F707D1
:10F07000A384F500A16593858502480897B0FFFF3A
:10F08000E780600797000000E78020EBAA8548082A
:10F0900097D0FFFFE780E0EA97000000E78060EC90
:10F0A000AA85480897D0FFFFE780A0E950080147EC
:10F0B0008146A285268597B0FFFFE780202905615C
:10F0C0001733FFFF6700E3029777FF1F9387C7C4DB
:10F0D0009C43014599C303C5B70082801733FFFFE6
:10F0E000E702E3FE0111B70707003EC683C795009C
:10F0F000404D0AC493F7F7070AC8A384F5002A898C
:10F10000AE8405C81C42054783C707006368F7063D
:10F110000347B400630FF700A305F40097900000C5
:10F12000E78040098347B400B9CF97D0FFFFE7805D
:10F1300040BE21649305B400280097B0FFFFE7802C
:10F1400080FB97000000E78060F8AA85280097D030
:10F15000FFFFE78000DF014781463000A6854A8532
:10F1600097B0FFFFE780801E2904480822CC230ABD
:10F17000010002CE97E0FFFFE78040C3056117332F
:10F18000FFFF670003F797D0FFFFE78020BF55B769
:10F190001733FFFFE702A3F301117C003ECAB70754
:10F1A00007003ECC7C003ECE83C795002E84AA8407
:10F1B00093F7F707A384F500A165AD05480897B05C
:10F1C000FFFFE78040F397000000E78020F0AA856A
:10F1D000480897D0FFFFE780C0D650080147814616
:10F1E000A285268597B0FFFFE7804016056117339B
:10F1F000FFFF670003F09777FF1F9387E7B19C43FA
:10F20000094599C303C5C70082801733FFFFE70292
:10F2100003EC01117C00AE843ECAA165B70707006C
:10F220002A843ECCD1057C0048083ECE97B0FFFF33
:10F23000E78060EC97000000E78020FCAA85480882
:10F2400097D0FFFFE780E0CF500801478146A685B1
:10F25000228597B0FFFFE780600F05611733FFFF3E
:10F26000670023E91733FFFFE70263E683C79500D2
:10F2700093F7F707A384F50097000000E78020F9D3
:10F280001733FFFF6700E3E61733FFFFE70283E270
:10F2900083C795000329C501411193F7F707A3849C
:10F2A000F5001C4283C90700854763E63707977757
:10F2B000FF1F938767FD9C432E84AA8485CF970008
:10F2C0000000E78080F389476306F50263040902C2
:10F2D0008347C900638037032306390197900000F4
:10F2E000E78040ED83572903898B89C797D00000B9
:10F2F000E780E0B72685A28597000000E78020F12F
:10F30000A167CD0748003EC42302010002C697E072
:10F31000FFFFE780A0A941011733FFFF6700C3DCAF
:10F320009777FF1F9387479F9C431D4599C303C54C
:10F33000E70082801733FFFFE70263D90111B707A7
:10F3400007003EC683C79500584D0AC493F7F707D8
:10F350000AC8A384F5002A89AE8415C71C4283C756
:10F36000070093968701E18663C40606854663819C
:10F37000D7068346E7006388F6002307F7009790D7
:10F380000000E78020E321649305E400280097B0A3
:10F39000FFFFE78040D697000000E780A0F8AA852D
:10F3A000280097D0FFFFE780C0B9014781463000B1
:10F3B000A6854A8597B0FFFFE78040F935044808E5
:10F3C00022CC230A010002CE97E0FFFFE780009ED7
:10F3D00005611733FFFF6700C3D11733FFFFE70253
:10F3E00003CF01117C003ECAB70707003ECC7C006A
:10F3F0003ECE83C795002E84AA8493F7F707A38493
:10F40000F500A165B905480897B0FFFFE780A0CED9
:10F4100097000000E78000F1AA85480897D0FFFF19
:10F42000E78020B2500801478146A285268597B023
:10F43000FFFFE780A0F105611733FFFF670063CB93
:10F440001733FFFFE70203C7AA8401441779FF1FA0
:10F450001309C98CE14997C0FFFFE78040C96344A5
:10F46000A400014519A833053403832709003E95FC
:10F47000835725006397970011051733FFFF670037
:10F48000A3C60504C9BF032E8500630A0E121773B5
:10F49000FF1F130363A7032303006315030029431E
:10F4A0006390061203234E01631503001D43639905
:10F4B00007101733FFFFE70203BFC689428A3E8960
:10F4C000BA8AB684328BAE8B2A84B5E103554E00DE
:10F4D00019E501431A851733FFFF670043C0A16791
:10F4E000A98F116763FBE70097000000E78080F5B4
:10F4F000814597F0FFFFE780C0120844B70700E09E
:10F500005841F98F18455CC1B707001FF98F1CC51A
:10F510005C4991C7610597E00000E780408BE38A72
:10F5200009FA228597900000E78060C65DB73285B2
:10F5300097C00000E78040430D4349DD1C4411673C
:10F5400003D54700A167A98F63FBE7009700000080
:10F55000E78040EF814597F0FFFFE780800C0323B1
:10F56000840093164B01D1828347B3000356630096
:10F570008588FD8BA305F300FD777D8E558EFD7686
:10F58000FD16B204F18E83274301C58E2312730149
:10F590002313D3002304530123052301A3044301B0
:10F5A000BDDF228597B0FFFFE78020CDAA85084404
:10F5B000B5D1610597D00000E780207F8DB71D434E
:10F5C0001A8582801733FFFFE702C3AE0569AA845C
:10F5D000AE89328A0144FD5A7D1997C0FFFFE7804A
:10F5E000C0A56347A40001451733FFFF6700C3AF01
:10F5F000D84493171400BA9703D70700631F370343
:10F600002390570163070A00268597900000E78042
:10F61000A0809C449DC383D76700B3F72701639EF6
:10F620003701D2880148814701478146014681451B
:10F63000268597000000E78040E5050479BF173371
:10F64000FFFFE70223A779711C103EC4B7070F0024
:10F650003EC61C103EC883C79500AA8A328593F720
:10F66000F707A384F5002E89328497D0FFFFE78047
:10F67000009D93170501C187635AF006AA89228568
:10F6800097D0FFFFE780A09B2A8A4E85032B0400BA
:10F6900097B0FFFFE780009B39ED8357440081441A
:10F6A0000544F11793B71700A303F10083457100D8
:10F6B000DA872287D2864E86280097E0FFFFE78010
:10F6C000E057014781463000CA85568597B0FFFF55
:10F6D000E780C0C7A1679387F70348083ECC230A99
:10F6E000810026CE97D0FFFFE780406C456117333D
:10F6F000FFFF6700639FA2851306710097E0FFFF7D
:10F70000E7806066AA84094455D1528597E0FFFFDF
:10F71000E78060D40D4459D90546D28526859700E7
:10F720000000E78060EA2A8451B71733FFFFE70241
:10F73000039A835507000346270041112A842E852A
:10F7400032C62EC497E0FFFFE780E0D001C9324601
:10F75000A245228597000000E78000E741011733AA
:10F76000FFFF670003991733FFFFE702C39383C7C7
:10F7700095004111AA8A93F7F707A384F500328513
:10F78000AE89328497D0FFFFE780608B9317050125
:10F79000C1876357F00AC1452A8A228597C0FFFFB7
:10F7A000E78080702A8D228597D0FFFFE78020892F
:10F7B0002A89228597D0FFFFE7804086930705F8C6
:10F7C00093F7F70F1307E007AA8B637BF7062285F1
:10F7D00097D0FFFFE78080842A8C228597D0FFFF97
:10F7E000E780C083AA8C5285032B040097B0FFFFEB
:10F7F000E780408539E983574400231101008144A3
:10F80000F11793B71700A300F10005440347110057
:10F8100083562100938784005685DA882288528691
:10F82000CE8597F0FFFFE78020A7A167E907480092
:10F830003EC42302810026C697D0FFFFE780005711
:10F8400041011733FFFF6700838913061100A2856A
:10F8500097E0FFFFE7802051AA8409E5231101000A
:10F8600009446DB7930521006A8597F0FFFFE78093
:10F87000A0F02A8441FD835521009356C900131638
:10F88000490185486688E2875E87858A5182268598
:10F8900097000000E78060BF2A848DBF1733FFFF09
:10F8A000E702638083C7950041112A8B93F7F7071E
:10F8B000A384F5003285AE89328497C0FFFFE780CC
:10F8C000007893170501C1876352F00A2A8A2285BE
:10F8D00097C0FFFFE780A076AA8A228597C0FFFF26
:10F8E000E780E0752A89228597C0FFFFE7800073D3
:10F8F000930705F893F7F70F1307E0072A8C637750
:10F90000F706228597C0FFFFE7804071AA8C228509
:10F9100097C0FFFFE78080702A8D5285832B0400FB
:10F9200097A0FFFFE780007239E5835744008544C4
:10F930000144F11793B71700A301F1000347310009
:10F94000930784005A85DE882688D6865286CE851F
:10F9500097F0FFFFE78040948D4748003EC42302A4
:10F96000910022C697D0FFFFE78040444101172352
:10F97000FFFF6700C376A2851306310097E0FFFF03
:10F98000E780603E2A84894455D99356C9001316EE
:10F99000490185486A88E6876287858A5182D685CB
:10F9A00097000000E78060AEAA8449BF1723FFFFDD
:10F9B000E70243702A8981440144617A916A176B96
:10F9C000FF1F130B6B5497B0FFFFE780006863C7FE
:10F9D000A40022851723FFFF670003718327090016
:10F9E00093991400CE9703D50700330745014207CA
:10F9F00041836364570305C103270B0019C785457D
:10FA00003E8597400000E78060E9832709000504F0
:10FA1000CE972390070085047DB797000000E7800C
:10FA200060A2832709000504CE972390070065D5BF
:10FA3000814597F0FFFFE780C0BEF1BF1723FFFFAE
:10FA4000E702436783C7950041112A8A93F7F707B6
:10FA5000A384F50032852E89328497C0FFFFE780AA
:10FA6000005E93170501C187635AF004AA89832AAF
:10FA7000040097A0FFFFE780E05C31E58357440076
:10FA800085440144F11793B71700A301F10003481F
:10FA90003100D68752850147CE862686CA8597D003
:10FAA000FFFFE780806AA167F50748003EC4230294
:10FAB000910022C697D0FFFFE780402F4101172316
:10FAC000FFFF67006362A2851306310097E0FFFF26
:10FAD000E78060292A8489445DD99767FF1F93874F
:10FAE000A7429C4381CF044997B0FFFFE780E055D0
:10FAF000AA85268597400000E78040DA13050401B7
:10FB000097000000E780C0EA228597800000E78028
:10FB100000338144ADBF1723FFFFE702C35883C7FB
:10FB200095004111AA8A93F7F707A384F50032855F
:10FB3000AE8932842311010097C0FFFFE780205077
:10FB400093170501C1876354F0062A8AC1452285AF
:10FB500097C0FFFFE7804035AA8B5285032B040036
:10FB600097A0FFFFE780004E21E9835744008544BA
:10FB70000144F11793B71700A300F10003481100E7
:10FB800003572100DA875685D2862686CE8597D000
:10FB9000FFFFE780805BA1679387270248003EC490
:10FBA0002302910022C697D0FFFFE7802020410169
:10FBB0001723FFFF6700A352A2851306110097E0E9
:10FBC000FFFFE780401A2A8489444DD99767FF1FB9
:10FBD0009387873398433E8901CF044997B0FFFF4D
:10FBE000E780A046AA85268597400000E78000CBE5
:10FBF0001305040197000000E78080DB97B0FFFF4A
:10FC0000E780A04495443DD9930521005E8597F097
:10FC1000FFFFE78060B6AA8435F11C480357210036
:10FC200022852390E70097800000E780402183270A
:10FC30000900A9D70355210097400000E780A0BD27
:10FC400035BF1723FFFFE702034683C79500411125
:10FC5000AA8A93F7F707A384F5003285AE89328428
:10FC600097C0FFFFE780A03D93170501C18763514F
:10FC7000F0062A8A228597C0FFFFE780403C2A8948
:10FC80005285032B040097A0FFFFE780A03B31E5DE
:10FC90008357440085440144F11793B71700A3012B
:10FCA000F10003483100DA8756854A87D2862686D6
:10FCB000CE8597D0FFFFE7804049A167F90748004C
:10FCC0003EC42302910022C697D0FFFFE780000EBA
:10FCD00041011723FFFF67008340A285130631000F
:10FCE00097E0FFFFE78020082A8489445DD9916767
:10FCF000CA97C2071167C1831307F7EF8544E36210
:10FD0000F7FA9767FF1F938727209843BE8B01CF91
:10FD1000044997B0FFFFE7804033AA8526859740C6
:10FD20000000E780A0B71305040197000000E780FA
:10FD300020C897B0FFFFE780403195443DD11C4873
:10FD4000228581442390270197800000E780200FBF
:10FD500083A70B00B9D74A8597400000E780A0AB86
:10FD600089B71723FFFFE70283362A844105B2844F
:10FD700097000000E780C0C311C52285978000006E
:10FD8000E780E00B81460146A6852285978000002A
:10FD9000E780C04E1C4C89C7DC4799C322858297F7
:10FDA0001723FFFF6700E3349767FF1F9387C7F6AA
:10FDB0009C43014599C31385070182809767FF1F04
:10FDC000938787F5884382801723FFFFE70223305C
:10FDD0009317C600DD8DC2054111C1812A8432C648
:10FDE00097C0FFFFE780E0173246228511829375A6
:10FDF000F60F97C0FFFFE780C01441011723FFFFF4
:10FE00006700232F1723FFFFE702C32A79713C08FD
:10FE10003ED2B7070C003ED43C083ED683C79500BF
:10FE2000AE842A8993F7F707A384F500A16593852B
:10FE30003504481097A0FFFFE780E02BC165FD1552
:10FE40000144176AFF1F130AAA0D930A400EAE89D8
:10FE50002E8B2EC697B0FFFFE78020224205931716
:10FE600004014181C183B24563E9A702C167FD175F
:10FE70006387F500481097C0FFFFE780800E5010A1
:10FE800001478146A6854A8597A0FFFFE780004C81
:10FE900045611723FFFF670023253307540383279A
:10FEA0000A0BBA9703D6C701630A3601638A350184
:10FEB000481097000000E78060F1DA85050451BF23
:10FEC000B285EDBF1723FFFFE702E31D79717C08C0
:10FED0003EC8B70711003ECA7C083ECC83C79500D8
:10FEE000AA89328593F7F707A384F5002E8997C076
:10FEF000FFFFE780C01485676378F504A165AA84D5
:10FF00008905080897A0FFFFE780E01E2685974037
:10FF10000000E78060ED133415000A04A28508088C
:10FF200097C0FFFFE780E001A685080897C0FFFFA4
:10FF3000E780200325CC014781461008CA854E85FD
:10FF400097A0FFFFE780804045611723FFFF670010
:10FF50000319B30754030327CA0ABA9703D7070044
:10FF6000631C970003D62700638065050808970087
:10FF70000000E780A0E5DE8505042EC697B0FFFFF0
:10FF8000E780A0104205931704014181C183B24567
:10FF9000E3E1A7FCC167FD17E38FF5F8080897C0F8
:10FFA000FFFFE78000FC41BFB285F9B7C165FD15D1
:10FFB0000144176AFF1F130AAAF6930A80022E8BC8
:10FFC000AE8B65BF1723FFFFE7026310184183471D
:10FFD000170083460700A207D58FD207D18323904D
:10FFE000F50083472700034717008D45A207D98FE7
:10FFF00091832310F60097C0FFFFE780A0E9172345
:020000040001F9
:10000000FFFF6700030F1723FFFFE702A30AC16486
:1000100001441769FF1F1309A9F093098002FD1419
:1000200097B0FFFFE78060066347A40001451723F0
:10003000FFFF6700630B330534038327C90A3E952E
:1000400083570500E38597FE0504D9BF1723FFFFFB
:10005000E70243062A8AAE89B284B68A9740000036
:10006000E78080D819E591473E851723FFFF670099
:10007000A3072A894E8597C00000E780E08E2A8476
:10008000638E0A048D476DD103570500C547E31DF4
:1000900047FD0347F9018546AD47E317D7FC834782
:1000A000450081CF4146A6855D0597F00000E780B9
:1000B000C09E814755D9AD4745BF1309650123024D
:1000C000E500CA85268597100000E780606231C18F
:1000D000A547E38B0AF82302040079B705C18357CB
:1000E0000500E39247F94146A685190597F00000FF
:1000F000E780A09A81472DD99947BDB74E859700D3
:100100000000E78080F02A84954739DD1309550007
:100110004DBF4146A6852310440123113401130528
:10012000190097F00000E780A099228597800000D1
:10013000E780A0EA81470DBF1723FFFFE70223F9FD
:1001400079717C003ECCB7070A003ECE7C003ED0E1
:1001500083C79500B2842E8493F7F707A384F50034
:100160001306A1002A892C00268597000000E7804D
:10017000A0E5A16528088D0597A0FFFFE780A0F7FF
:1001800090408355A10003558100854697000000EB
:10019000E78000ECAA84AA85280897C0FFFFE780C3
:1001A00040DA0356A100835581002808970000001B
:1001B000E780C0C1300801478146A2854A8597A0E3
:1001C000FFFFE780A018854748103ED42302910224
:1001D00002D697D0FFFFE78060BD45611723FFFF80
:1001E000670023F11723FFFFE70263EE79717C00BC
:1001F0003ECCB7070A003ECE7C003ED083C79500B8
:10020000B2842E8493F7F707A384F5001306A100A8
:100210002A892C00268597000000E780E0DAA16596
:1002200028088D0597A0FFFFE780E0EC90408355FC
:10023000A10003558100814697000000E78040E15E
:10024000AA84AA85280897C0FFFFE78080CF0356BD
:10025000A10083558100280897000000E78000B7BF
:10026000300801478146A2854A8597A0FFFFE780B5
:10027000E00D48102302910202D402D697D0FFFF6E
:10028000E780C0B245611723FFFF670083E61723AD
:10029000FFFFE702C3E397000000E78060DB17235E
:1002A000FFFF670003E59767FF1F938727A7884332
:1002B00082801723FFFFE70283E183572500411166
:1002C000AE842A842307B10017F5FFFF13052546E6
:1002D0006C002316F10097A0FFFFE780204991C42E
:1002E000228597800000E780E0D6FD572310F400B8
:1002F000130620028145130554009720FFFFE78075
:1003000000E041011723FFFF6700A3DE1723FFFF73
:10031000E70243DA79717C003ECCB7070A003ECE93
:100320007C003ED083C79500AA89AE8493F7F70777
:100330003285A384F5001306A1002C00970000006D
:10034000E78080C803558100114497400000E78092
:10035000A0A915C50355A100014497B00000E7808E
:10036000A06011CD035705008357810045446318F1
:10037000F700854597000000E780E0F3014421691C
:1003800093053900280897A0FFFFE780C0D6A28513
:10039000280897C0FFFFE780C0BA0356A100835525
:1003A0008100280897000000E78040A2300801473C
:1003B0008146A6854E8597A0FFFFE78020F948106B
:1003C0004AD42302810202D697D0FFFFE780009E25
:1003D00045611723FFFF670023D11723FFFFE702C3
:1003E00063CD9767FF1F938727932A8488432E89BD
:1003F00015C5035745038357C4016311F70223262C
:10040000050223180502410597D00000E780209CD3
:100410006306090097800000E78060DB81449769EC
:10042000FF1F9389E9AF130A800297B0FFFFE780AF
:10043000C0C563C4A4049767FF1F9387A7969C4316
:1004400099C70355C40197200000E780C0BD63072A
:100450000900228597800000E780C0A01306400EA7
:10046000814522859720FFFFE78060C9FD57231E45
:10047000F4001723FFFF670023C73385440383A7D6
:10048000C90A3E95035705008357C4016317F70057
:10049000CA8597000000E78000E2850479B717233A
:1004A000FFFFE70223C183C795004111AA8993F793
:1004B000F707A384F5003285AE8497C0FFFFE7807D
:1004C00000B885676378F5042A8997400000E780C3
:1004D000A091014401CD83D70400314463882701F2
:1004E000854597000000E78080EF01444E85A28695
:1004F0004A86A68597D0FFFFE780A09CA1679387D7
:10050000170448003EC42302810002C697D0FFFFB3
:10051000E780C08941011723FFFF6700E3BC172371
:10052000FFFFE70223B99757FF1F9387E77E8043BA
:1005300029C4014597C00000E78000218147014898
:10054000C1641CDC232E0403232004041769FF1F4D
:100550001309099D01449309400EFD1497B0FFFF54
:10056000E780A0B1634FA400814517F5FFFF130595
:10057000857F97A0FFFFE780601F1723FFFF6700BD
:10058000A3B6330534038327090B3E958357C50172
:1005900063879700854597000000E78040E40504E5
:1005A00075BF9357050113D78700A380F5009317F4
:1005B0000501C183A1832380E5002381F500A38188
:1005C000A50082801723FFFFE70263B02300050028
:1005D00083C71500A300F50083C725002301F5009C
:1005E00083C73500A301F50083C745002302F5004A
:1005F00083C75500A302F50083C7650093059500E6
:10060000A30305002303F5002304050032859700AA
:100610000000E78040F91723FFFF670083AD172331
:10062000FFFFE70223A94111E9540DCD85CD93F9D0
:10063000C5FF2E842A89AA84338AA900B7EA040058
:1006400063189A020D88854411CCB7E704009C5FBB
:1006500082972AC622866C003305390197E0000094
:10066000E7800046268541011723FFFF6700C3A7E7
:1006700083A78A039104829793170501C183A183FD
:10068000A38EF4FE93570501238FF4FEA183238EDE
:10069000A4FEA38FF4FE6DB763E6D5021723FFFF18
:1006A000E702E3A2B28741113686BE8536C697E0DF
:1006B0000000E780E040B246410136851723FFFF86
:1006C000670023A3814636858280838705001387D0
:1006D000F5003D05FD8793F77708834607007D15F4
:1006E0008606B58FA300F5006307B7007D17834723
:1006F00017009D83DDB782801723FFFFE702239D4C
:10070000B7E7040083A7070932872A863A858297CC
:10071000133515001723FFFF6700A39D15C18147FF
:100720008DC11723FFFFE702839A414697E000003F
:10073000E780003985473E851723FFFF6700639BED
:1007400081473E8582801DCD1723FFFFE702239856
:10075000414681452A849720FFFFE780409A414621
:100760008145130504039720FFFFE7804099014767
:10077000C1672322040438C87CC805451723FFFF3E
:10078000670023970145828081473DCDB5CD172372
:10079000FFFFE702C393B2842E89130680058145CB
:1007A0002A849720FFFFE7808095CA8524C4268588
:1007B00097000000E780C0F64146814522859720DA
:1007C000FFFFE780C0933044A28522859700000098
:1007D000E780C0F293040401A285268597000000FB
:1007E000E780E0EEA6851305040297000000E7808D
:1007F00000EE228597000000E78020F585473E85C2
:100800001723FFFF6700E38E3E8582801723FFFFDB
:10081000E702438A4111E9540DCD85CD93F9C5FF17
:100820002E842A89AA84338AA900B7EA040063982F
:1008300044030D88814411CCB7E704009C5F829784
:100840002AC622866C003305390197E00000E78054
:100850002027268541011723FFFF6700E38883A730
:100860008A039104829793170501C183A183A38E04
:10087000F4FE93570501238FF4FEA183238EA4FE7B
:10088000A38FF4FE6DB765CD1723FFFFE7028382C8
:10089000B28411E605451723FFFF6700E3842A842D
:1008A0002E890145EDD93C487848B3E6E700E5D606
:1008B0009386F7FFB3B7F6007D17032A4404BA976F
:1008C00034C87CC863050A06C14913050A03B38905
:1008D00049412295637D3601B2862E86A685970012
:1008E0000000E780A0DB7C40BE9464C065B7CE8684
:1008F0002E86CE8597000000E78040DAC114D2949E
:100900004E9923220404A2879306040103C707001B
:1009100003C607038507318FA38FE7FEE398F6FE32
:100920003044A285228597000000E78020DD2699CB
:10093000C1493306994063EC9900A9DCA686A685D7
:100940001305040397000000E78040D579BF814775
:10095000B306F4003307F6000347070083C506001B
:1009600085072D8F2380E600E39437FF3044A2856E
:10097000228597000000E78060D8C1145DBF014563
:1009800082800DC11713FFFFE70263741306800511
:1009900081459710FFFFE780807605451713FFFF1D
:1009A0006700237501458280814749C5C1C517137A
:1009B000FFFFE702C371FC4141462E84AA8463997C
:1009C000C70413860501A2878146C14503C70700F6
:1009D00003C507038507298F3305D60003450500A6
:1009E0008506298FA38FE7FEE392B6FE3044A285E9
:1009F000268597000000E78060D0228597000000E0
:100A0000E78060F885473E851713FFFF6700636E38
:100A1000138507031D8E814522959710FFFFE78000
:100A2000006E7C40130700F813060402A297238887
:100A3000E70251BF3E8582801713FFFFE70223695B
:100A40006D712E84B284AA85901028003689970093
:100A50000000E780A0D309EDD55725A050400C40F9
:100A6000280097000000E78040E27DD5FD142104B6
:100A7000F5F42C004A8597000000E78020F38147B9
:100A800061DD3E8551611713FFFF67008366171311
:100A9000FFFFE702C36341112EC432C62C00054696
:100AA00097000000E78080F941011713FFFF6700FE
:100AB00043641713FFFFE702836101112A842EC6E6
:100AC00002C802CA02CC02CE97E00000E780402BA9
:100AD000B2462A86A285080897000000E78060FBDE
:100AE0001375F50F05611713FFFF67008360171378
:100AF000FFFFE702C35D7971B2872A84214623088C
:100B0000B10013051101BE853AC436C697E0000056
:100B1000E78000FBB24693059101368597000000FF
:100B2000E78060A82285141035460C089700000065
:100B3000E78020F62A84224701E921460C103A85F5
:100B400097E00000E780C0F7228545611713FFFF9B
:100B50006700235A1713FFFFE70263577171AE84D2
:100B6000AA850A85328497000000E78060BB11C91E
:100B70000A86A685228597000000E78020B8814775
:100B800011E1C5473E854D611713FFFF67006356AE
:100B90001713FFFFE702A3501D712A8AB289BE8492
:100BA00035468547130511012E8CB68A3A8BC28CC7
:100BB000468D2308F10097E00000E78060F01010F8
:100BC0000C085285231F010097000000E780C0F841
:100BD0002A843DEDA1476313FD089307900591E03A
:100BE000E5473546E2851305110113990A012308EB
:100BF000F1001359090197E00000E78060EC1357FA
:100C0000890093978A00D98F90080C085285231F7A
:100C1000F10097000000E78020F42A8415E9A1E4A0
:100C20009387FA0091831379F9003EC66313090094
:100C30004149668B8144C14B854DB247639F970CF8
:100C40006A868C0033855C0197E00000E78040E70E
:100C5000228525611713FFFF67002348930790043F
:100C6000C9F0A547BDBF834701050947C14B23080C
:100C7000F10083471105A58FA308F1009387240095
:100C8000814463E1FB04014714083386E6008C08C5
:100C9000B386E400BA95DA9683C6060083C50500DC
:100CA0000507AD8E2300D600E390E7FE4147639C25
:100CB000E70490080C08528597000000E780C0E91F
:100CC00025D181A0B3069B00BA871008B305F600B2
:100CD00090083E9603C50600034606008507850674
:100CE000298E2380C500E39277FF998F90080C0826
:100CF0005285BE9497000000E78000E689470147CF
:100D000049D12A84B1B790083E96034606001408DC
:100D1000BE962380C600850759BFB2478504638706
:100D2000971481471808B306F70098083E97338652
:100D3000F90003470700034606008507318F23802B
:100D4000E600E39177FF90080C08528597000000B9
:100D5000E78080E05DF53546E28513051101230843
:100D6000B10197E00000E780A0D51397040141830B
:100D7000939784002183D98F10180C085285231F64
:100D8000F10097000000E78020DD25FD8147101865
:100D90003387F9003E960347070003460600B30673
:100DA000FB008507318F2380E600E39277FF65A87B
:100DB0001808B306F70098083E973386F9000347F2
:100DC0000700034606008507318F2380E600E3E134
:100DD00027FFCA87639E770990080C085285970001
:100DE0000000E78060D711FD81479800B306F70047
:100DF000900818103E973E960347070003460600EA
:100E00008507318F2380E600E39177FF3546E28541
:100E1000130511012308B10197E00000E78040CAE3
:100E2000139704014183939784002183D98F10186D
:100E30000C085285231FF10097000000E780C0D105
:100E4000E31105EC814710183387F9003E960347FC
:100E5000070003460600B306FB008507318F238099
:100E6000E600E3E227FFC109410BC1BB814785B71B
:100E70009408BE9683C6060018083E972300D70044
:100E8000850789BF638006321713FFFFE70223211E
:100E900059712A84BE89B28B8547354613051102E4
:100EA0002E8B468C4289BA8A368A2300F10297E05B
:100EB0000000E780E0C010180C1022852317010203
:100EC00097000000E78040C963180512A147631F1F
:100ED000FC069307900563930900E5473546DA85DC
:100EE0001305110293140A012300F102C18097E057
:100EF0000000E780E0BC93178A0013D78400D98FE5
:100F000090080C1022852317F10297000000E7805B
:100F1000A0C47DE1639209049307FA00BD88918320
:100F200091E0C144C207C183DE8C814A3EC6414D77
:100F3000B24763E2FA0E6286B3854B01881097E0F0
:100F40000000E78080B54DC93D557DA09307900412
:100F5000E39609F8A54759B7834701050947C14CEE
:100F60002300F10283471105B3C7F900A300F10282
:100F700093872900814963E1FC04814618103306F8
:100F8000D7008C083387D900B695569703470700DA
:100F900083C5050085062D8F2300E600E390D7FE6C
:100FA00041476390E70690080C10228597000000E7
:100FB000E78080BA35D189A0B3863A01BA8710108C
:100FC000B305F60090083E9603C5060003460600EA
:100FD00085078506298E2380C500E39297FF338716
:100FE000EC4090080C102285BA9997000000E78029
:100FF000A0B68947014741D165611713FFFF67001C
:10100000C30D90083E96034606001410BE9623803A
:10101000C600850779B7B247850A93990A01939D5F
:101020008A0093D909016391570F85473546DA85C0
:10103000130511022300F10293D9890097E0000003
:10104000E78000A8B3ED3D0190000C102285231726
:10105000B10397000000E78020B059FD8147A689C1
:1010600063EA970626860C084A8597E00000E78029
:1010700020A581471810B306F700100898083E977E
:101080003E9603470700034606008507318F2380FD
:10109000E600E3E197FE639FA90590080C10228506
:1010A00097000000E78040AB21F981479810B30614
:1010B000F700900818183E973E960347070003462E
:1010C00006008507318F2380E600E391A7FF4109E1
:1010D000C10CB9BD18089000B306F7003E963387DF
:1010E000FC0003470700034606008507318F238075
:1010F000E600B5B798084E97034707001C10CE9737
:101100002380E700850941BF85473546DA85130509
:1011100011022300F10293D9890097E00000E780D3
:10112000209AB3ED3D0190000C1022852317B103E6
:1011300097000000E78040A2E31005EC8147180803
:101140009000B306F7003E963387FC000347070084
:10115000034606008507318F2380E600E391A7FF51
:1011600041460C084A8597E00000E780609581477A
:101170001810B306F700100898083E973E960347EC
:101180000700034606008507318F2380E600E391C0
:10119000A7FF90080C10228597000000E780C09BF5
:1011A0001DD599BD7D5582801713FFFFE70223F2FD
:1011B00001112A842E8593055100328902C002C292
:1011C00002C402C69304740097F0FFFFE780A03DBD
:1011D0001D46A6851305910097E00000E780408E2C
:1011E00010088A854A8597000000E780E09619ED8F
:1011F00093071400180883C60700034607008507F5
:101200000507B18EA38FD7FEE397F4FE0561171390
:10121000FFFF670003EE1713FFFFE702A3E92E8429
:101220008C414111AA89838715003289914463D387
:101230000700A1449757FF1F938707059C43A1C749
:10124000C1CA8D472310F10083C725004A852301B9
:10125000F10083C73500A301F10083C745002302D5
:10126000F10083C75500A302F10083C76500930511
:101270009100A30301002303F1002304010097F070
:10128000FFFFE78040320C404A860A8597F0FFFF57
:10129000E78080330328040083564400A6881D0895
:1012A00081470147E51642868A854E8597000000F2
:1012B000E780408E2A8919E5A685228597B0FFFF31
:1012C000E780E0C14A8541011713FFFF6700C3E1D2
:1012D0004A860A8597F0FFFFE780002F6DB7171346
:1012E000FFFFE70223DD2E848C414111AA89838709
:1012F00015003289914463D30700A1449757FF1F1B
:10130000938787F89C43A1C7C1C68D472310F1007E
:1013100083C725004A852301F10083C73500A30157
:10132000F10083C745002302F10083C75500A302E3
:10133000F10083C7650093059100A3030100230317
:10134000F1002304010097F0FFFFE780C0250C4067
:101350004A860A8597F0FFFFE780002783564400FE
:10136000032804008A85858EC2061D08C1822312C7
:10137000D400A68881470147E51642864E8597002E
:101380000000E78060B041011713FFFF6700C3D57D
:101390004A860A8597F0FFFFE78000234DBF1713A9
:1013A000FFFFE702C3D2B335B000011185052A89DA
:1013B0001315F601336515012308B10093051101DA
:1013C00036843AC632C03EC442C297F0FFFFE7807F
:1013D000801DA2471248425593D68700230BF10087
:1013E0009305910193578800A30AD100A30BF10044
:1013F000230C010197F0FFFFE780E01A3247024615
:1014000003280400B337E000835644009207914458
:1014100011C2A1444A85A68842860C0897F0FFFFB6
:10142000E78040772A8919E5A685228597B0FFFFD6
:10143000E780E0AA4A8505611713FFFF670063CBC9
:101440001713FFFFE70203C701113EC68647B335F6
:10145000B0008505AA891315F6015D8D2308B1003A
:101460009305110136843A89B28442C446C297F08A
:10147000FFFFE780401322489248164593578800A3
:10148000A30AF1009305910193D78800230B010172
:10149000A30BF100230C110197F0FFFFE780A010D0
:1014A0003247104083564400B337E00092070328C8
:1014B0000900914891C0A1480C084E859700000092
:1014C000E780809CAA8401E9835544004A8597B04F
:1014D000FFFFE780C0A0268505611713FFFF6700A7
:1014E000A3C0AA959307F00F17170100130787AC45
:1014F0006317B50013C5F7FF1375F50F8280050557
:101500008346F5FFB58FBA9783C70700D5B7035752
:10151000450014419307F00F17160100130686A922
:10152000369742074183139506014181631BE5000D
:10153000AD8FB29703C50700130515F313351500DA
:101540008280850603C5F6FFA98FB29783C707007F
:10155000D9BF1713FFFFE70283B7B28736842E8601
:10156000BA86AA853E85BA8497F0FFFFE78060526D
:10157000634F0500228597E00000E78060802A869F
:10158000A686A285268597F0FFFFE7808050171377
:10159000FFFF670003B61713FFFFE702A3B15D71FA
:1015A0002A8BAE8A171501001305459E2C00B284C4
:1015B000368ABA893E8997F0FFFFE780C04F2A84B8
:1015C0005DE134104146DA85280097F0FFFFE7809F
:1015D000404C2A8449E98547A303F100A6C293073A
:1015E00071002408BEC4A68685470D462C18281015
:1015F00002DC02DED6C0BEC697F0FFFFE7800044E3
:101600002A8435E183477102A6860D4693F7F707D2
:101610002300FA00C1473EDE2C188947281026DC3B
:10162000A303F10097F0FFFFE78040412A8405ED16
:101630004146A6854E8597D00000E78060488D47DB
:10164000A6860D462C182810A303F10097F0FFFF83
:10165000E780C03E2A8401E94146A6854A8597D0A5
:101660000000E780E045228561611713FFFF6700F6
:10167000A3A71713FFFFE70283A597F7000093873F
:1016800027EF984383C7470079712A89AE841715DD
:101690000100130525900C083AC42306F10097F0C9
:1016A000FFFFE78040412A8405ED14104146CA85BA
:1016B000080897F0FFFFE780C03D2A8415E1140871
:1016C00015462C00081097F0FFFFE780803C2A8425
:1016D00001E921462C08268597D00000E780403E8E
:1016E000228545611713FFFF6700A3A01713FFFFB3
:1016F000E702E39D97F70000938787E79C4779719E
:10170000AA842E8417150100130545890C083EC6CE
:1017100097F0FFFFE780203A0DE914104146A685B7
:10172000080897F0FFFFE780C03605E1140811466E
:101730006C00081097F0FFFFE780A03519E583479C
:10174000F10193F7F7032300F40045611713FFFF3E
:101750006700239A1713FFFFE70263973688A148B3
:1017600081470147E54697F0FFFFE780A042171346
:10177000FFFF670003981713FFFFE70243953688C2
:10178000A14881470147E54697F0FFFFE780C06F1A
:101790001713FFFF6700E3951713FFFFE70223937B
:1017A00001112A842E850C0832C697F0FFFFE780CE
:1017B000803009ED3247970601009386A67C100819
:1017C000C145228597000000E780E0D80561171326
:1017D000FFFF670003921713FFFFE702438F4111DA
:1017E000C1472EC032C48A8509463EC23EC697F024
:1017F000FFFFE780A02441011713FFFF6700638FFD
:101800001713FFFFE702A38C4111AE8613061009E0
:10181000AA850A8502C002C202C402C697F0FFFF71
:10182000E780202741011713FFFF6700838C171300
:10183000FFFFE702C3893287970601009386867609
:101840002E869305000297000000E780C0D0171392
:10185000FFFF6700038A1713FFFFE70243877971D1
:10186000C1472ACC2ED032D42C080D4628003ECEBB
:101870003ED23ED602C402C602C802CA97F0FFFF9B
:10188000E780C01B45611713FFFF670083861713AE
:10189000FFFFE702C3830111AA842E84170501000C
:1018A0001305C5708A8597F0FFFFE780C02015E516
:1018B00014084146A6850A8597F0FFFFE780601D62
:1018C00009ED8347E1010347F101A207D98FCA0758
:1018D000C9836177D98F2310F40005611713FFFFC7
:1018E0006700238115CD1703FFFFE702437E97476B
:1018F000FF1F9387274790439745FF1F9385C54652
:101900001745FF1F1305054297D00000E78000C56B
:101910001745FF1F130505411703FFFF6700637D90
:101920001745FF1F1305054082808DCD1703FFFF6C
:10193000E702E3799747FF1F9387C742944301115A
:101940002E840A869745FF1F9385054297D0000095
:10195000E78040C60A850294014505611703FFFF31
:10196000670023797D5582801703FFFFE702237606
:1019700097D00000E78080D19747FF1F23A4A73EA0
:1019800017F5FFFF1305E5C997B00000E780C074A5
:101990001703FFFF6700E3751747FF1F1307C73ED5
:1019A0009317150008433E95FD572310F5008280DC
:1019B0001703FFFFE702A3712A84084009E5170314
:1019C000FFFF670003731C4158401CC06313E50010
:1019D0005CC08347550023200500F99BA302F50056
:1019E00097A0FFFFE780207CC9BF1703FFFFE70236
:1019F000636C9747FF1F9387273B98432A8411CB3B
:101A00008347350093F7070289C7035505008945C9
:101A100002971305440197B00000E780403B8355CF
:101A200004000355E40097300000E780A00C4858FC
:101A300019C597A0FFFFE7800077232A040213054A
:101A4000840397000000E780E0F68144B149979055
:101A5000FFFFE780C06D63CBA402834734002320DF
:101A6000040493F727FCA301F40000489790FFFFBC
:101A7000E780E06C13161500814522859700FFFF73
:101A8000E780E0671703FFFF67000366B38734034F
:101A90000329040385043E994A8597000000E780E6
:101AA00060F12304090065B78347350093F7070207
:101AB00099E3014582808357E500E39CB7FEC16747
:101AC000FD176316F60005458280054599A81703A2
:101AD000FFFFE702C35F93170601C187B2842A8420
:101AE00001496359F002835705009DCB01456367A7
:101AF000F600034584003E953325A6001375F50FC7
:101B00000DA01C4813171900BA9783D70700E38E5E
:101B100097FA05099790FFFFE7806062E343A9FE0B
:101B200001451703FFFF6700C35C1703FFFFE702D0
:101B30006358AE89AA849790FFFFE78000562A84F5
:101B400097D0FFFFE780A02EAA86014713068401E5
:101B500097050000938585E41745FF1F13050523AE
:101B60009790FFFFE780801C2A8925C98C441304C5
:101B7000C50022859E0593F5050897A0FFFFE78025
:101B8000403CCC4083877400E18163DD070493E52A
:101B90000508228597A0FFFFE780A03A0D469385B0
:101BA0004400228597A0FFFFE780C03683D504005C
:101BB000228597A0FFFFE780E03D83D524002285A2
:101BC00097A0FFFFE780003D03D6490083A50900E9
:101BD000228597A0FFFFE780E0334A851703FFFFC8
:101BE0006700835093F5F5076DB71703FFFFE70212
:101BF000034E01112A84328532C697A0FFFFE78089
:101C0000E0279780FFFFE780603483570400174781
:101C1000FF1F1307E7303246231BF100930700F83C
:101C2000A30DF1001C471843231AA1008983858B5B
:101C3000B307F740B28548083ECE231C0100230DB0
:101C4000010097000000E78080EE05611703FFFFA9
:101C50006700234A1703FFFFE702C3450041014520
:101C60003DC49304C40026853289AE8997A0FFFF46
:101C7000E780C02495452A8A2685035B040197A046
:101C8000FFFFE7802021268597A0FFFFE780603EC9
:101C90008D45AA8A268597A0FFFFE780A01F26858D
:101CA00097A0FFFFE780E03C5C48420A135A0A0114
:101CB000D2975CC423186401814763983A014605B2
:101CC0004D81330625419337160013F5F70F17039F
:101CD000FFFF670063411703FFFFE702C33C896909
:101CE0002A8BAE8B328AB68A81440144314CFD196D
:101CF0009790FFFFE780A04363CDA4009790FFFF7C
:101D0000E780E045018D33B5AA001703FFFF6700A8
:101D1000033D3389840383270B003E9963170A0030
:101D20008347890085043E94E1B703560A00DE85A7
:101D30004A8533F6C90097000000E780E0F16DD1D5
:101D40000545E1B71703FFFFE702633801112A8455
:101D50007C000355E5003ECAB70707003ECC7C0077
:101D60003ECE97200000E78020082A898545480854
:101D700097A0FFFFE78020399945480897A0FFFF0B
:101D8000E780E015AA844A8597200000E780A00834
:101D90002380A4009747FF1F938787189C434166C1
:101DA000130606F09396870113D78701558F93D6B4
:101DB0008700F18E558FA207B706FF00F58FD98FE8
:101DC00011462C00138514003EC497D00000E78014
:101DD00020CF5008A3820400894522859700000087
:101DE000E780E0E019C9AA851305840397A0FFFFE7
:101DF000E780E0313C4085073CC005611703FFFFE9
:101E00006700232F1703FFFFE702632C9790FFFF64
:101E1000E780E0342A8405049790FFFFE7802033B1
:101E20003305A402F14791453305F50297200000E0
:101E3000E78020BA11E565551703FFFF6700632BA4
:101E40009747FF1F23AAA7F49790FFFFE780203151
:101E50002A8405049790FFFFE780602F3305A402D2
:101E60008945060597200000E780A0B669D5974709
:101E7000FF1F23ABA7F09790FFFFE780402E2A8437
:101E800005049790FFFFE780802C3304A402974756
:101E9000FF1F239D87EE9790FFFFE780402C2A8449
:101EA0009790FFFFE780A02A930714003385A702CD
:101EB0009747FF1F239DA7EC970701009387C7D281
:101EC0001747FF1F2328F7EC0145BDB71703FFFF96
:101ED000E702431EAA842E8901449749FF1F938974
:101EE0002904130A80069790FFFFE7804026634786
:101EF000A40001451703FFFF6700031F33054403D8
:101F000083A709024A86A6853E9597000000E780D0
:101F1000E0B919E10504C1BF0545E9BF1703FFFF9B
:101F2000E7026318AA8A2E8BB28B368C3A8A8144D8
:101F300001448149974CFF1F938C8CFE130D800642
:101F40009790FFFFE780A02063C9A40011E08549B6
:101F50004E851703FFFF670083183389A40383A707
:101F60000C025E86D6853E994A8597000000E78080
:101F7000E0B31DC19790FFFFE780601E0544636DCD
:101F80004501D2866286DA851305090397000000B1
:101F9000E780A0D411C1854985045DB71703FFFF11
:101FA000E7024311C16441112A8901449749FF1F87
:101FB000938909F7130A8006FD1436C632C42EC26F
:101FC0009790FFFFE780A01892452246B2466348EB
:101FD000A400014541011703FFFF6700E31033052B
:101FE000440383A709023E9509C683473500C18B88
:101FF0009DC791C68347350093F707028DC36306DB
:1020000099008357E500639C27010357050001CB26
:1020100063E7E50083478500BA97E3CDF5FA050449
:1020200069BF1703FFFFE702E308C1642A8901447F
:102030009749FF1F9389C9EE130A8006FD149790F4
:10204000FFFFE780C0106346A4001703FFFF67008F
:10205000A3093305440383A709023E958357E5008E
:10206000638A970063049900639627019700000034
:10207000E780E0970504E1B71703FFFFE7022302BB
:1020800089692A8AAE8A328BB68B8144174CFF1F2E
:10209000130C0CE9930C8006314DFD199790FFFF4E
:1020A000E780E00A63C6A4001703FFFF6700E302AE
:1020B0003389940383270C028355CA015A863E99BB
:1020C0004A8597000000E780609E31C1814D15A0D0
:1020D0003384AD038327090303D60B00D68533F67B
:1020E000C9003E94228597000000E780E0B609E928
:1020F000850D9790FFFFE7808003E3CBADFC01A83F
:10210000228597000000E780E08A2304040085040C
:1021100071B71703FFFFE70203F94169AA8A014A71
:10212000174BFF1F130BCBDF7D19C14B054C97904D
:10213000FFFFE780C0016346AA001703FFFF6700A7
:1021400003FA93098006B3073A0383290B02BE9969
:1021500083D7E900638E270163842A01639A5701BC
:1021600003A4890301E84E8597000000E780C0BD05
:10217000050A75BF83570401639977099304C40066
:10218000268597A0FFFFE78060D385452A8D2685A9
:10219000835C040197A0FFFFE780C0CF268597A04E
:1021A000FFFFE780A0E762056185635905048D455F
:1021B000268597A0FFFFE780E0CD8945268597A07B
:1021C000FFFFE78020CD8945268597A0FFFFE780A8
:1021D00060CC8545268597A0FFFFE780E0CC83474C
:1021E0000500094793F7F707639AE70099452685A5
:1021F00097A0FFFFE78040CBA30285014848337DCD
:102200002D01231894016A9548C40040A1BF17030B
:10221000FFFFE702C3EB37E404008327041D829726
:102220009747FF1F83C7C7BC1715FF1F1305052F4F
:10223000A300F5008327441C82978327841C8146D2
:102240001306F00F8145014582971703FFFF6700D2
:1022500043EA1747FF1F1307A7A918439745FF1F16
:1022600083C505B99747FF1F938707B78346870341
:10227000034697036397D5009747FF1F238AC7B686
:10228000828083C587010347A7036317B60097477A
:10229000FF1F238FE7B4828003C687016317C7003F
:1022A0009747FF1F2386D7B4828083C68701130711
:1022B00050026319D700930760021747FF1F2309D5
:1022C000F7B2828083C68701130660026315D600C9
:1022D00093077002DDB783C7870155BF9747FF1F7C
:1022E000938787AFD44B0947638DE6081703FFFF39
:1022F000E702E3DD1749FF1F130949AB3E8483471B
:102300000900918B9DCFB7E4040083A7041D829739
:1023100083A7441C1745FF1F1305C5A9829783A7F0
:10232000841C81461746FF1F0346C6AA8145014506
:10233000829721C583470900ED9B1747FF1F23079D
:10234000F7A68347040093F7F70F85CB914717470C
:10235000FF1F232DF7A897000000E78080EB970070
:102360000000E78040EFB7E70400BC4F41469145CD
:102370001745FF1F0345C5A682971703FFFF670098
:1023800043D782801703FFFFE70263D48D474111D3
:102390006306F504C5476308F50285476310F50237
:1023A0009747FF1F2388A7A4B7E70400BC4B9305FA
:1023B00000101745FF1F0345A5A28297410117038F
:1023C000FFFF670003D385471747FF1F2304F7A2CA
:1023D000B7E70400BC4B93050020E1BF9747FF1F00
:1023E0009387879FD44B1147638DE600B7E70400BE
:1023F00083A7071D8297B7E70400BC4B9305000431
:102400004DBF05491747FF1F2322279F83C707009A
:1024100032C62E8493F7F70FD5D3B7E4040083A711
:10242000041D7D141374F40F8297E37689FCB24582
:10243000994703C61500E3F0C7FCFC44090617459D
:10244000FF1F1305659B8297BC489305000817453D
:10245000FF1F0345E598829779BF1703FFFFE70247
:1024600003C71747FF1F130727974047184B1C4008
:102470009746FF1F23A8F6966316E4001747FF1F31
:102480002324F796130584FE9790FFFFE78000AAA8
:10249000035564FF9780FFFFE780807297A0FFFFDE
:1024A000E78060D01703FFFF6700A3C41703FFFF97
:1024B000E702E3C19747FF1F93870792D84BDC479A
:1024C00089C797000000E78080F985471747FF1FFD
:1024D000232EF7909747FF1F938787819C4393058F
:1024E00000021745FF1F0345A58F83C787031747C2
:1024F000FF1F230FF78EB7E70400BC4B829717032B
:10250000FFFF670003BF9747FF1F23A9A78C8280A7
:102510001703FFFFE70203BA37E404007C4CA14530
:102520001745FF1F0345C58B82977C48A14517457A
:10253000FF1F0345E58A9744FF1F9384E489829730
:10254000DC4489EB97000000E78080D91703FFFF88
:10255000670083B903D567FF9780FFFFE780406678
:10256000AA896DD1D84891476310F7027C4C9145F8
:102570001745FF1F0345C58682977C48914517453F
:10258000FF1F0345E585829703A9490103D409018B
:102590008947B7E904001747FF1F2329F78483A75A
:1025A000091D21044204829783C784011715FF1F68
:1025B0001305C5F661191717FF1FA301F7F683A7C7
:1025C000491C418082979747FF1F2385078283A775
:1025D000C91C814609469375F40F4A85829711E913
:1025E0009747FF1F83C7479189C79700FF1FE78061
:1025F000405FB7E70400BC4F2146A1451735FF1FD8
:102600000345057E829799B71703FFFFE70223ACC6
:1026100093F7052001112E8481CF97000000E780F9
:1026200020E91345042005611703FFFF670063AC31
:1026300093F70510A9CF9734FF1F9384E479DC4802
:1026400097000000E78020C11737FF1F1307476A74
:10265000184383C78401034787036318F700DC44EA
:1026600089C797000000E78080DF85471737FF1F85
:10267000232EF776B7E70400BC4B9305000217350D
:10268000FF1F0345E57582971345041069BF93F753
:102690000508BDC79737FF1F83C71776E917194687
:1026A0009735FF1F938565751305D10093F4F70FD8
:1026B0001739FF1F0349497497C00000E780404065
:1026C00093970401C1831737FF1F13076773231DF7
:1026D000F100231CF1009737FF1F9387E76F3ACE75
:1026E0003ACAD8432306010009CBDC43931589017C
:1026F00054080D46E185680082971345040825B704
:1027000093F72500A5C39737FF1F9387E76CD84B36
:1027100089476306F7029737FF1F83C7276913F7B7
:10272000270011EF918B99CFB7E70400BC4F130638
:10273000000A89451735FF1F0345856A82971345AF
:102740002400D5B59737FF1F9387875A9C4383C7CB
:1027500087031737FF1F230DF76897000000E780F6
:1027600060DBF1BF93F7050281CB97000000E780A3
:1027700060DA1345040245BD93F7850081CB9700CD
:102780000000E780E0D21345840071BD93F7150087
:1027900081CB97000000E780A0B41345140061B519
:1027A00093F7450081CB97000000E78060B31345A5
:1027B000440095BD93F7050495C39737FF1F83C762
:1027C000A76191CB97000000E780A0A4914717373D
:1027D000FF1F232DF76013450404B1B593F70501DE
:1027E0000145E38207E49737FF1F9387E75ED84BE5
:1027F00091476310F7049737FF1F9387275B9C432C
:1028000013D727008583D98F858B91E7B7E704001D
:1028100083A7071D8297B7E70400FC4F9145173542
:10282000FF1F0345E55B829785471737FF1F232F5F
:10283000F75A13450401C5BB9737FF1F238EA76ABC
:1028400082801703FFFFE70283889737FF1F23ABC0
:1028500007589737FF1F23A9075885471734FF1FCD
:10286000130404491737FF1F2322F7581C4083C75E
:1028700087031737FF1F230DF7569790FFFFE78059
:10288000409329C59717FF1F23AEA7C81C40170503
:1028900000001305A5D783C787031737FF1F230938
:1028A000F7541717FF1FA30BF7C69737FF1FA38512
:1028B0000752B7E7040083A7070882979737FF1FDF
:1028C0002380A7521703FFFF6700A382B7C7898E33
:1028D000938767ED1717FF1F2326F7C445BF1737E8
:1028E000FF1F0347674F795555E79737FF1F9387BA
:1028F000A74E03C7170005079736FF1FA38EE64CA8
:1029000003C717008D463377D7029736FF1FA3857D
:10291000E64C83C617001737FF1F1307673D1843A0
:1029200093F6F60FA9EE834787031737FF1F23019E
:10293000F74C85471737FF1F2300F74A9737FF1FCC
:102940009387C7469C430145998BA9E717F3FEFF80
:10295000E702E37737E404007C48C1451735FF1FE1
:102960000345054882973C4885451735FF1F0345B9
:1029700025478297014517F3FEFF6700837783C7DA
:10298000170085466395F6008347970379BF834711
:10299000A70361BF82809737FF1F83C7E743A1CF9B
:1029A00017F3FEFFE702A37237E404009737FF1F17
:1029B000238407427C4885451735FF1F0345454260
:1029C00082977C4C91451735FF1F034565418297DF
:1029D0007C4891451735FF1F0345854082973C4849
:1029E000C1451735FF1F0345A53F8297014517F3E2
:1029F000FEFF670003707955828017F3FEFFE70240
:102A0000036D2A84035565FF9780FFFFE780401B15
:102A10009737FF1F9387473CD847BE841DEF979099
:102A2000FFFFE78080779C48232004009DEB9737C9
:102A3000FF1F23AB873A9737FF1F23A5873AB7E7D6
:102A40000400BC4B89451735FF1F03456539829744
:102A5000014517F3FEFF6700C369630A8700184347
:102A600075BF80C39737FF1F23A08738C9BF79552B
:102A7000CDB717F3FEFFE70283659737FF1F9387F4
:102A8000E74788432326050023240500510597A026
:102A90000000E780C03317F3FEFF6700836517F37C
:102AA000FEFFE702C3621734FF1F130424451C40D6
:102AB000411199CF9C472302B5002AC61CC197003B
:102AC0000000E78040FB1C409C4B99C33245829735
:102AD000410117F3FEFF6700C36117F3FEFFE70232
:102AE000035F4111444D328532842EC69790FFFF1B
:102AF000E780C0522AC422859790FFFFE7802054C8
:102B000003A84400630C0800B245835744001840F2
:102B1000224683D54500AA8626850298410117F3EF
:102B2000FEFF6700035D17F3FEFFE702435A404DC7
:102B30001DC808C09705000093856503130544016F
:102B400097A00000E78040169737FF1F9387073B49
:102B50009C43014589E79737FF1F23A1873A17F365
:102B6000FEFF670003597D55DDBF17F3FEFFE70247
:102B70000356011168009305F00F02C602C802CA8D
:102B800002CC02CE97000000E780A0F1056117F3A8
:102B9000FEFF670003569737FF1F938727369C4336
:102BA000D847A1679D076319F70217F3FEFFE702F5
:102BB0000352011132859790FFFFE7802046230AD8
:102BC000A1008145680097000000E78080ED056165
:102BD00017F3FEFF6700E35182809737FF1F93874B
:102BE000E7319C43D847A167938777036319F702BE
:102BF00017F3FEFFE702A34D011132859790FFFF07
